:020000040800F2
:1000000000000110A5B00308C1890308150F0108FD
:10001000A9B10308A9B10308A9B1030800000000B1
:10002000000000000000000000000000099003082C
:1000300005900308000000000190030819C900089A
:10004000A9B10308A9B10308A9B10308A9B103081C
:10005000A9B10308A9B10308E9D4000815D600081E
:10006000D9D500089DD5000861D500085DBC000801
:100070004DBC00083DBC00082DBC00081DBC00089C
:1000800009BC0008F5BB0008A9B10308A9B1030821
:10009000A9B10308A9B10308A9B1030825D500082F
:1000A00031190108A9B10308A9B10308A9B10308CE
:1000B0008119010871190108A9B10308A9B1030840
:1000C000A9B10308A9B10308A9B10308A9B103089C
:1000D000A9B1030885CA0008A9B10308E9C9000845
:1000E000ADD40008A9B1030825900308A9B10308FD
:1000F00041190108A9B1030851190108E1BB000821
:10010000A9B10308A9B1030861190108A9B103083D
:10011000A9B10308A9B10308BDF80108A1F80108B5
:10012000CDBB0008B9BB0008A5BB000891BB000807
:100130007DBB0008A9B10308A9B10308A9B1030850
:10014000A9B10308A9B10308A9B10308C589030827
:1001500069BB000855BB000841BB00084DC9000839
:10016000A9B10308A9B10308A9B10308A9B10308FB
:10017000A9B10308A9B10308A9B10308A9B10308EB
:08018000A9B10308A9B10308AD
:1001880016000800EC240020F424002000000000E1
:100198001006000827000400D0280020D8290020D5
:1001A800000000001806000801010400303000209B
:1001B800AC3E00200000000000000000080209001A
:1001C800263E0020B03E002000000000B3BE00081C
:1001D80002000C00303E0020BC3E00200000000061
:1001E80000000000F7010600203E0020C83E002065
:1001F800000000001C0600080A020A00C0300020A7
:10020800D03E002000000000220600080312330040
:100218006741002034410020000000002C0600083F
:1002280025005A0080400020DA400020000000002D
:1002380000000000F6110C00744000206840002007
:100248000000000060060008012008006442002049
:10025800B0420020000000006C0600081A000800E8
:100268004C420020B842002000000000740600083C
:1002780015007000F8440020484A002000000000E3
:100288000000000003000100F4440020B84A0020E8
:1002980000000000000000002A0060000444002064
:1002A800BC4A002000000000153B020809020100BA
:1002B800AC4B00208C580020000000007C06000891
:1002C80005000600AA5A0020745B00200000000008
:1002D800800600080C002400725A00207C5B002075
:1002E8000000000025EE01080E20EA006A590020EF
:1002F800A05B002000000000D51C020813000400C9
:10030800C05A00208C5C002000000000880600080D
:10031800020103004F590020905C002000000000FB
:100328004DEE0108F511620094580020945C0020FD
:1003380000000000A582000829005000B05F0020DE
:10034800BC63002000000000000000001400020050
:10035800AC5F00200C640020000000008C06000840
:100368000102050034680020A46D00200000000090
:1003780045B902080002050010640020AC6D002099
:1003880000000000000000001E0004002C66002091
:10039800B46D0020000000008E06000822000C004A
:1003A800246D0020B86D00200000000092060008AF
:1003B800FB010100147B0020487B002000000000A6
:1003C8001DFD0008FC010900E07900204C7B00209D
:1003D80000000000E9FC00080A101200B4790020AF
:1003E800587B0020000000009E060008060016004A
:1003F800847600206C7B002000000000F51C0208B9
:1004080034001000F0740020847B002000000000FD
:100418003D3B02080D003400BC740020947B002092
:100428000000000045B8010812100C00A07400205C
:10043800C87B002000000000B00600080C02010084
:100448009C740020D47B002000000000BC0600083B
:1004580002020300B0740020D87B002000000000D6
:1004680000000000FA010200787C00207C7C00205B
:100478000000000075FD0008FD012400047C002038
:10048800807C00200000000035BE0008FE01080046
:10049800F07B0020A47C00200000000059FD00082B
:1004A8001F000E00F07D0020107E002000000000DC
:1004B800BE06000805020100D87D0020207E00202D
:1004C80000000000CC060008030106006A7D002039
:1004D800247E002000000000CE0600081B00F40067
:1004E800347E0020F88000200000000055B9020882
:1004F80026000E00FC810020EC8100200000000096
:10050800E112030810000300888400208C84002076
:1005180000000000D406000828000C007C8400209D
:100528009084002000000000D80600082300100076
:100538006C8400209C84002000000000819B02083D
:100548001900050064840020AC840020000000002D
:10055800E4060008F811010060840020B48400203B
:1005680000000000EA060008000104005C84002086
:10057800B884002000000000EC0600082F001100DD
:1005880048840020BC84002000000000F006000819
:100598000400800014A00020A4A100200000000096
:1005A80000000000F90104002095002024A200208A
:1005B80000000000A5BE000818102C00F0940020D0
:1005C80028A2002000000000AD5503082C001000F0
:1005D80028A4002018A400200000000021530308CC
:1005E8002B0024005CA4002038A400200000000098
:1005F800F15203080B201000D4A600200CA70020FD
:080608000000000002070008D9
:10061000C409000019012828200300001800010067
:10062000000000004A01B400D601000000000000F4
:1006300000000000000000000000000000000000BA
:1006400000000000000000000000000000000000AA
:100650000000000000000000000000000000010099
:10066000000000000000000000000000E80364003B
:10067000040A00017E05EA05B405320013000000FB
:100680002000030001000000080004000300000037
:100690000100C800141E010064002C012800003075
:1006A0000100005A0000000090012C01C800640005
:1006B000000000010005504C554D000001000000F5
:1006C000000000000100000000050000000004011F
:1006D0000100000000010500000000010000000012
:1006E000000000000000280100000400BC01000020
:1006F00000000000000000000000000000000000FA
:1007000000002B21231E64010200000001000A01E9
:020710002900BE
:10071200010100005001000007000000020000007B
:10072200000000000000000001020304060708099F
:1007320001010000C01204083C4B04080000000044
:1007420000000000D0120408D812040800000000C3
:1007520001200000DC120408E4110408000000007B
:1007620001400000E41204082826040800000000EA
:1007720001200000F0120408FC120408000000002E
:100782000400000000130408644204080000000092
:10079200040000000C130408B03D0408000000002F
:1007A20001000000020100000000803F0000803FC5
:1007B200FF0000005D8803081588030865870308A9
:1007C2000000000055840308D985030859860308F0
:1007D200418503080000000000000000498403086E
:1007E2002D84030829840308258403081984030837
:1007F20015840308218403081D8403083D8403082B
:1008020031840308198503082D850308058503082B
:10081200F1840308DD840308F4E6030805080400F4
:1008220000000000D801040874010408E0E603088F
:100832000000000020E7030805080A00000000008D
:10084200D801040874010408FC0104080000000037
:10085200FFFFFFFF0000803F0100000001010100D7
:10086200E04104080F000000457202080000000089
:1008720000000000D0020020A44104080000000093
:100882000000000000000000000000003C4B0408D3
:1008920000000000000000006C07002004000000BF
:1008A200304104080D0000006D8B0208480700204B
:1008B20000000000AC4404080D0000003D8B02085B
:1008C2003C07002000000000C441040808000000AA
:1008D200000000003007002004000000B4410408BA
:1008E2000D000000F98A0208240700200000000021
:1008F2004840040803000000AD8D02080C070020E8
:1009020000000000BC41040803000000AD8D020895
:10091200F4060020000000004C4004080100000022
:1009220000000000000000000000000000000000C5
:100932000E000000000000000000000000000000A7
:10094200A4410408000000000000000000000000B4
:10095200000000003C4B0408000000000000000002
:100962006C07002004000000D440040803000000CB
:1009720049780208DC06002008000000B44104089F
:100982000D000000F98A0208240700200000000080
:100992004840040803000000AD8D02080C07002047
:1009A20000000000BC41040803000000AD8D0208F5
:1009B200F4060020000000004C4004080100000082
:1009C2000000000000000000000000000000000025
:1009D2000E00000000000000000000000000000007
:1009E200CC410408000000000000000000000000EC
:1009F200000000003C4B0408000000000000000062
:100A02006C07002004000000DC4004080300000022
:100A1200AD8D020854070020000000004C4004087D
:100A220001000000000000000000000000000000C3
:100A3200000000000E0000000000000000000000A6
:100A4200000000002D202D2D202D2D2D2D202D2DAF
:100A52002D2D00000000000000000000000000003A
:100A620000000000464B002088130C170100000014
:100A7200484B002088130C17000000002040040897
:100A82000000000000000000000000000000000064
:100A9200304004080800000000000000600300204D
:100AA200040000003C4004080800000000000000B0
:100AB2005403002000000000484004080400000025
:100AC2008178020800000000000000004C40040889
:100AD2000100000000000000000000000000000013
:100AE200000000000E0000000000000000000000F6
:100AF20000000000444B002088130C170100000086
:100B0200424B002088130C170000000084400408A8
:100B12000F0000009D7202080000000000000000AB
:100B22006C030020A34B0020010000009801040880
:100B3200404B002001000000A4010408D47D0020E5
:100B420002000000AC010408DAA00020000000004E
:100B520000000000D8A000200000000000000000FB
:100B6200D6A000200000000000000000D4A0002059
:100B72000000000000000000D2A0002000000000E1
:100B820000000000D0A000200000000000000000D3
:100B9200101E002000000000000000003F4B00205B
:100BA20002000000B80104088C40040800000000A4
:100BB20000000000000000000000000030400408B7
:100BC2000800000000000000F00300200400000004
:100BD2003C4004080800000000000000E40300207C
:100BE2000000000048400408040000007D72020872
:100BF20000000000000000004C400408010000005A
:100C020000000000000000000000000000000000E2
:100C12000E000000000000000000000000000000C4
:100C22009C400408000000000000000000000000DA
:100C320000000000AC4004080D000000958A020884
:100C42002C04002004000000B84004080D0000003D
:100C5200C17202082004002004000000C4400408FD
:100C62000D0000005D8A020814040020000000004C
:100C7200D04004080300000065780208FC0300204D
:100C820008000000DC40040803000000AD8D0208EB
:100C920054070020000000004C400408010000003E
:100CA2000000000000000000000000000000000042
:100CB2000E00000000000000000000000000000024
:100CC200E4400408000000000000000000000000F2
:100CD20000000000EC400408040000009D780208B7
:100CE20000000000000000004C4004080100000069
:100CF20000000000000000000000000000000000F2
:100D02000E000000000000000000000000000000D3
:100D1200384104080000000000000000000000004C
:100D2200000000001C3704080D0000000000000055
:100D32008C04002004000000484104080800000060
:100D42000000000080040020040000005441040858
:100D520008000000000000007404002004000000ED
:100D62005C41040808000000000000006804002044
:100D720004000000644104080800000000000000B4
:100D82005C040020040000006C410408080000001C
:100D92000000000050040020040000007441040818
:100DA20008000000000000004404002004000000CD
:100DB2007C41040808000000000000003804002004
:100DC200040000004C400408010000000000000084
:100DD2000000000000000000000000000E00000003
:100DE2000000000000000000000000008441040830
:100DF2000F0000008D7202080000000000000000D9
:100E0200980400208C4104080F000000000000003C
:100E120000000000000000001005002094410408BA
:100E22000F000000000000000000000000000000B1
:100E3200B0050020A44B002004000000C4010408F7
:100E420088580020E0150C1700000000A14B00207C
:100E52000800000074010408A24B002005000000F5
:100E6200D80104089C4104080F00000000000000A3
:100E72000000000000000000000600202D202D2DA3
:100E8200202D2D2D2D202D2D2D00000000000000E5
:100E920000000000000000000000000020700020A0
:100EA200702D7200EC4904080F00000000000000E1
:100EB20000000000000000002C1B0020FFFFFFFFCD
:100EC200FA00000001000000010000004C4204088A
:100ED20054420408E440040800000000000000003E
:100EE200000000000000000034420408040000007A
:100EF200DB77020800000000000000004C400408FC
:100F020001000000000000000000000000000000DE
:100F1200000000000E0000000000000000000000C1
:100F2200000000006E7F00200100C40900000000E4
:100F32006C7F00200100C409000000006A7F0020CD
:100F42000100C40900000000687F00200100C409FC
:100F520000000000647F00200100C40900000000BE
:100F6200667F00200100C40900000000627F0020AB
:100F72000100C40900000000607F00200100C409D4
:100F820000000000005900200100C800010000001C
:100F9200FE5800203200307532000000FC5800205C
:100FA200055A0500F758002000FF0100FB580020F9
:100FB20001000000BC070020F958002002000000D8
:100FC200F0010408F658002000FF0100FA58002042
:100FD20001000000BC070020F858002002000000B9
:100FE200F0010408984204080F000000000000000D
:100FF2000000000000000000C4070020A87D0020BF
:101002009CFF2C01000000004E0100200A0000009D
:10101200FC0104083C4B0020E0150C170000000006
:101022004D01002008000000740104084C0100205A
:1010320005000000D80104083E4B00200200000019
:1010420014020408B05A00200100FF7F01000000D2
:10105200A85A00200200000020020408585900206B
:10106200030000003002040857590020030000006A
:10107200300204085C5A00200000F4010100000064
:101082005A5A00200000F40101000000585A0020C2
:101092000000F40101000000565A00200000F40193
:1010A20001000000545A002000FF0100705A002085
:1010B200E803D0070A0000006E5A00200064010015
:1010C2000A0000006F5A0020006401000A000000BC
:1010D200685A0020006401000A0000006D5A0020D6
:1010E200006401000A0000006C5A00200064010044
:1010F2000A0000006B5A0020006401000A00000090
:10110200675A002000FF01000A000000665A002012
:1011120000FF01000A000000665900200000F401EF
:1011220001000000645900200000F40101000000E9
:10113200625900200000F401010000006059002003
:101142000000F40101000000635A002000C8010001
:10115200625A002000C80100615A002000C8010044
:10116200605A0020006401000A0000005F5A00205B
:1011720000FF01000A0000009F5A002000C8010081
:101182009E5A002000C801009D5A002000C801009C
:101192009C5A002000C801009B5A002000C8010090
:1011A2009A5A002000C80100995A002000C8010084
:1011B200985A002000C80100975A002000C8010078
:1011C200A04204080000000000000000000000002F
:1011D20000000000B0420408090000000000000006
:1011E2006808002004000000B8420408090000005A
:1011F200000000005C080020040000004C480408C5
:101202000900000000000000500800200400000057
:10121200F01004080900000000000000440800204B
:1012220004000000C04204080900000000000000A1
:101232003808002004000000C84204080900000029
:10124200000000002C08002004000000D042040826
:101252000900000000000000200800200400000037
:10126200D842040809000000000000001408002011
:10127200040000004C4004080100000000000000CF
:101282000000000000000000000000000E0000004E
:10129200000000000000000000000000B04304084D
:1012A200000000000000000000000000000000003C
:1012B200DC11040807000000000000008C08002078
:1012C20000000000C0430408080000000000000005
:1012D2008008002000000000CC4304080800000041
:1012E2000000000074080020000000004C400408C8
:1012F20001000000000000000000000000000000EB
:10130200000000000E0000000000000000000000CD
:1013120000000000D44304080000000000000000A8
:101322000000000000000000E44304080D0000007B
:1013320000000000C808002000000000EC43040880
:101342000D00000000000000BC08002000000000AA
:10135200F44304080700000000000000B408002065
:1013620000000000FC4304080D0000000000000023
:10137200A808002000000000044404080D0000003A
:10138200000000009C080020000000000C4404083B
:101392000700000000000000940800200000000088
:1013A2004C400408010000000000000000000000A2
:1013B20000000000000000000E000000000000001D
:1013C20000000000000000001444040800000000B7
:1013D200000000000000000000000000DC11040812
:1013E2000C00000000000000025900200000000074
:1013F200284404080C0000000000000004590020EA
:1014020000000000384404080C0000000000000046
:101412003A59002000000000484404080C00000073
:10142200000000002E590020000000005C44040867
:101432000C0000000000000006590020000000001F
:10144200684404080C000000000000000859002055
:1014520000000000704404080C00000000000000BE
:101462000A59002000000000844404080C00000017
:10147200000000000C590020000000008C44040809
:101482000C000000000000000E59002000000000C7
:10149200944404080C0000000000000010590020D1
:1014A20000000000A04404080C000000000000003E
:1014B20012590020000000007C3004080C000000DB
:1014C200000000001459002000000000A844040895
:1014D2000C0000000000000016590020000000006F
:1014E200B44404080C000000000000001859002059
:1014F20000000000F41104080C00000000000000CD
:101502001A59002000000000C04404080C0000002A
:10151200000000001C59002000000000CC44040818
:101522000C000000000000001E5900200000000016
:10153200D84404080C0000000000000032590020CA
:1015420000000000E04404080C000000000000005D
:101552003059002000000000E84404080C0000009C
:10156200000000003E59002000000000F44404087E
:101572000C000000000000004059002000000000A4
:10158200004504080C00000000000000465900203D
:1015920000000000101204080C000000000000000F
:1015A2002059002000000000B44104080C00000093
:1015B2000000000028590020000000000C4504082B
:1015C2000C00000000000000225900200000000072
:1015D200184504080C0000000000000024590020F7
:1015E20000000000244504080C0000000000000078
:1015F20026590020000000002C4504080C000000C1
:10160200000000002A590020000000007C34040879
:101612000C0000000000000034590020000000000F
:10162200384504080C000000000000002C5900207E
:1016320000000000681104080C0000000000000017
:101642003C59002000000000444504080C00000042
:101652000000000036590020000000004C4504083C
:101662000C000000000000003859002000000000BB
:10167200544504080C0000000000000042590020FC
:10168200000000005C4504080C000000000000009F
:1016920044590020000000004C40040801000000F2
:1016A2000000000000000000000000000000000038
:1016B2000E0000000000000000000000000000001A
:1016C2006445040800000000000000000000000063
:1016D200000000007445040805000000000000003E
:1016E20056590020000000004C4004080100000090
:1016F20000000000000000000000000000000000E8
:101702000E000000000000000000000000000000C9
:101712007C450408000000000000000000000000FA
:10172200000000003C4B0408000000000000000024
:101732003403002004000000EC1004080D00000037
:101742002178020828090020000000003041040826
:101752000D000000117202081C09002000000000A8
:10176200AC4404080D000000DD71020810090020DD
:1017720000000000C441040808000000000000004E
:101782000409002004000000B44104080D00000018
:10179200C9710208F808002000000000884504080A
:1017A2000900000000000000EC0800200400000016
:1017B2004840040803000000AD8D0208D408002050
:1017C200000000004C40040801000000000000007E
:1017D2000000000000000000000000000E000000F9
:1017E2000000000000000000000000009045040816
:1017F20000000000000000000000000000000000E7
:10180200A04504080D00000000000000400900206F
:1018120000000000A84504080A00000000000000C3
:101822001C5B002000000000B44504080A00000010
:1018320000000000245B002000000000BC450408FA
:101842000A000000000000002C5B002000000000E5
:10185200C44504080800000000000000340900200C
:1018620000000000CC45040804000000F18E0208CC
:1018720000000000000000004C40040801000000CD
:101882000000000000000000000000000000000056
:101892000E00000000000000000000000000000038
:1018A200D84504080000000000000000000000000D
:1018B20000000000EC4504080D00000000000000DC
:1018C2005809002000000000FC4504080400000044
:1018D200F18B02080000000000000000044604082A
:1018E2000D000000000000004C0900200000000074
:1018F2001846040804000000CD8B02080000000016
:10190200000000004C40040801000000000000003C
:101912000000000000000000000000000E000000B7
:101922000000000000000000000000002046040843
:1019320000000000000000000000000000000000A5
:10194200344604080700000000000000940900204B
:1019520000000000404604080800000000000000EB
:1019620088090020000000004C460408080000001E
:10197200000000007C090020000000005846040816
:1019820008000000000000007009002000000000B4
:1019920064460408080000000000000064090020FA
:1019A200000000004C40040801000000000000009C
:1019B2000000000000000000000000000E00000017
:1019C2000000000000000000000000007046040853
:1019D20000000000000000008F070020000000004F
:1019E2007C4604080B00000000000000FC090020F7
:1019F20000000000844604080B0000000000000004
:101A0200F009002000000000904604080B000000CE
:101A120000000000E4090020000000009C460408C9
:101A22000B00000000000000D809002000000000A8
:101A3200A84604080B00000000000000CC090020AA
:101A420000000000B44604080B0000000000000083
:101A5200C009002000000000BC4604080B00000082
:101A620000000000B409002000000000C84604087D
:101A72000B00000000000000A80900200000000088
:101A8200D446040808000000000000009C09002061
:101A9200000000004C4004080100000000000000AB
:101AA2000000000000000000000000000E00000026
:101AB200000000000000000000000000E0460408F2
:101AC2000000000000000000000000000000000014
:101AD200F446040808000000000000002C0A002060
:101AE2000000000000470408080000000000000099
:101AF200200A0020000000000C4704080800000033
:101B020000000000140A002000000000184704082A
:101B12000800000000000000080A00200000000089
:101B22004C4004080100000000000000000000001A
:101B320000000000000000000E0000000000000095
:101B42000000000000000000204704080000000020
:101B5200000000008C07002000000000304704084D
:101B62000B000000000000005C0A002000000000E2
:101B72003C4704080B00000000000000500A00204F
:101B820000000000484704080700000000000000B1
:101B9200480A002000000000544704080700000023
:101BA20000000000400A0020000000006047040816
:101BB2000700000000000000380A002000000000BA
:101BC2004C4004080100000000000000000000007A
:101BD20000000000000000000E00000000000000F5
:101BE20000000000000000006C4704080000000034
:101BF200000000008C070020000000007847040865
:101C02000700000000000000A80A002000000000F9
:101C1200804704080700000000000000A00A00201E
:101C220000000000884704080700000000000000D0
:101C3200980A0020000000009047040807000000F6
:101C420000000000900A00200000000098470408ED
:101C52000700000000000000880A002000000000C9
:101C6200A04704080700000000000000800A0020CE
:101C720000000000A8470408070000000000000060
:101C8200780A002000000000B047040807000000A6
:101C920000000000700A002000000000B84704089D
:101CA2000700000000000000680A00200000000099
:101CB2004C40040801000000000000000000000089
:101CC20000000000000000000E0000000000000004
:101CD2000000000000000000C04704080F000000E0
:101CE200000000004987020800000000B00A00203E
:101CF20054590020170000004002040853590020E4
:101D02000A3201005259002001FA01004E59002006
:101D120000C801004C590020E803D0070100000070
:101D2200504C554D463400009258002000030100EB
:101D32009158002000030100C84704080F0000006A
:101D42006D86020849860208000000008C0B002004
:101D5200D44704080F00000009860208C185020862
:101D620000000000040C0020E04704080F000000FF
:101D7200A98602089186020800000000B80C002023
:101D8200EC4704080F0000005F8702080000000013
:101D92009D8B0208B00F0020F44704080F000000DA
:101DA2002B7102080000000000000000001000205B
:101DB200FC4704080F000000D18E0208AD8902081A
:101DC200A9890208DC100020044804080F00000062
:101DD200858702080000000000000000901100202A
:101DE2000C4804080F00000025880208F587020845
:101DF200000000001C120020144804080F0000001C
:101E0200A1880208E588020800000000BC12002038
:101E1200645A002001030100204804080F0000005A
:101E2200C18702089987020800000000AC13002055
:101E3200284804080F00000055880208158C020883
:101E42000000000038140020344804080F0000008D
:101E5200118902085D8C020800000000D8140020DD
:101E62005E5A0020010301003C4804080000000003
:101E720000000000000000000000000048480408C4
:101E8200080000000000000004160020000000000E
:101E9200504804080700000000000000FC15002064
:101EA2000000000060480408070000000000000075
:101EB200F4150020000000006C4804080700000030
:101EC20000000000EC150020000000007848040823
:101ED2000D00000000000000E015002000000000DE
:101EE2008448040803000000AD8D0208C8150020D4
:101EF200000000004C400408010000000000000047
:101F02000000000000000000000000000E000000C1
:101F12000000000000000000000000008C480408DF
:101F220000000000000000000000000000000000AF
:101F32009C4804080A00000000000000781204080F
:101F420000000000A44804080A000000000000008D
:101F52004412040800000000AC4804080A00000013
:101F620000000000A05A002000000000B44804084D
:101F72000A0000000000000010160020000000000F
:101F82004C400408010000000000000000000000B6
:101F920000000000000000000E0000000000000031
:101FA2000000000000000000BC480408000000001F
:101FB200000000000000000000000000C848040803
:101FC20003000000AD8D020858160020000000003A
:101FD200D847040803000000AD8D02084016002017
:101FE20000000000CC47040803000000AD8D020889
:101FF2002816002000000000D44804080500000054
:10200200000000009058002000000000DC48040896
:102012000700000000000000201600200000000061
:10202200E84804080700000000000000181600201D
:10203200000000004C400408010000000000000005
:102042000000000000000000000000000E00000080
:10205200000000000000000000000000F448040836
:10206200000000000000000000000000000000006E
:102072001C12040803000000AD8D0208A016002007
:10208200000000000849040803000000AD8D0208AA
:102092005001002000000000104904080300000065
:1020A200AD8D0208881600200000000018490408BF
:1020B20003000000AD8D0208701600200000000031
:1020C2004C40040801000000000000000000000075
:1020D20000000000000000000E00000000000000F0
:1020E2000000000000000000244904080000000075
:1020F2000000000000000000000000003049040859
:1021020007000000A98C0208501700200000000000
:102112002845040803000000AD8D0208381700208E
:10212200000000003C49040803000000AD8D0208D5
:1021320020170020000000004449040803000000AA
:10214200AD8D020808170020000000004C49040869
:10215200070000008D8C020800170020000000001C
:102162004C41040803000000AD8D0208E81600206F
:10217200000000005849040803000000AD8D020869
:10218200D01600200000000064490408030000008B
:10219200AD8D0208B8160020000000004C40040873
:1021A200010000000000000000000000000000002C
:1021B200000000000E00000000000000000000000F
:1021C20000000000704904080F00000005870208A3
:1021D200C186020800000000581700207849040850
:1021E2000F0000007D8902080000000000000000CE
:1021F2000C180020844904080F000000A58502087D
:102202008985020800000000981800208C49040803
:102212000F000000000000000000000000000000AD
:102222004C1900209C4904080F000000558902083F
:10223200C58C020800000000D8190020A449040837
:10224200000000000000000000000000000000008C
:10225200B049040803000000AD8D0208141B0020E1
:10226200000000009049040803000000AD8D020840
:10227200FC1A002000000000884904080300000046
:10228200AD8D0208E41A002000000000B8490408DD
:1022920003000000AD8D0208CC1A002000000000EF
:1022A200C449040803000000AD8D0208B41A0020DE
:1022B20000000000CC490408020000003D8F020823
:1022C2000000000000000000D449040802000000E1
:1022D2003D8F02080100000000000000E0490408F0
:1022E200020000003D8F0208020000000000000012
:1022F200000000000E0000000000000000000000CE
:102302000000000001A1020800000000000000001F
:102312000001010101000000E00108000000803F0F
:10232200080001000060024010600240000000004E
:10233200000B000000002000000000000000000070
:10234200006002402860024000000000060C00000D
:1023520000002000000000000000000000600240B9
:102362004060024000000000100D0000000020004C
:1023720000000000000000000060024058600240BF
:1023820000000000160E0000000020000000000007
:102392000000000000600240706002400000000087
:1023A200200F0000000020000000000000000000DC
:1023B2000060024088600240000000002610000019
:1023C2000000200000000000000000000060024049
:1023D200A060024000000000301100000000200058
:1023E200000000000000000000600240B8600240EF
:1023F20000000000362F0000000020000000000056
:10240200000000000064024010640240000000006E
:102412000038000000004000000000000000000042
:1024220000640240286402400000000006390000F7
:1024320000004000000000000000000000640240B4
:102442004064024000000000103A0000000040001A
:1024520000000000000000000064024058640240D6
:1024620000000000163B00000000400000000000D9
:10247200000000000064024070640240000000009E
:10248200203C0000000040000000000000000000AE
:1024920000640240886402400000000026440000FC
:1024A2000000400000000000000000000064024044
:1024B200A06402400000000030450000000040001F
:1024C200000000000000000000640240B864024006
:1024D200000000003646000000004000000000003E
:1024E20000000000000000010000000000000000E9
:1024F2000000000000FFFF0000000000AA550300DA
:102502009FAA5505010000AA550701000001AA551E
:102512000B010000AA5509020000000001000000A2
:10252200C012000000000101FFFF0000A8340408EF
:10253200000000000000000061EE0108A08601001A
:102542000400000000000000000000000000000085
:102552000000000000000000000000000000000079
:1025620028450408D030040800000000FD46010898
:102572007D000000060000000000000000000000D6
:102582000000000000000000000000000000000049
:1025920000000000404B04080000000000000000A2
:1025A20039980308E803000003000000000000005F
:1025B2000000000000000000000000000000000019
:1025C2000000000000000000484B0408000000006A
:1025D20000000000F51D02081027000003000000A3
:1025E20000000000000000000000000000000000E9
:1025F200000000000000000000000000A0430408EA
:1026020000000000B1510308DD950108204E0000D2
:1026120005000000000000000000000000000000B3
:1026220000000000000000000000000000000000A8
:102632001C3604080000000000000000F5920308A8
:102642001027000001000000000000000000000050
:102652000000000000000000000000000000000078
:1026620000000000544B04080000000000000000BD
:10267200B5FC0008E80300000500000000000000AF
:102682000000000000000000000000000000000048
:102692000000000000000000604B04080000000081
:1026A2000000000019F10108204E000003000000A4
:1026B2000000000000000000000000000000000018
:1026C200000000000000000000000000704B040841
:1026D200000000000000000021EF0108204E000071
:1026E20003000000000000000000000000000000E5
:1026F20000000000000000000000000000000000D8
:10270200804B0408000000000000000085900308D0
:10271200400D030003000000000000000000000064
:1027220000000000000000000000000000000000A7
:10273200000000005C3504080000000000000000FA
:10274200CDCF0108102700000100000000000000AA
:102752000000000000000000000000000000000077
:102762000000000000000000EC300408000000003F
:10277200000000000DD10208102700000300000035
:102782000000000000000000000000000000000047
:1027920000000000000000000000000024360408D1
:1027A2000000000000000000B11D0108A00F0000A1
:1027B2000100000000000000000000000000000016
:1027C2000000000000000000000000000000000007
:1027D200904B04080000000000000000E916030806
:1027E20010270000010000000000000000000000AF
:1027F20000000000000000000000000000000000D7
:1028020000000000884904080000000000000000E9
:10281200C5A800081A4100000100000000000000E5
:1028220000000000000000000000000000000000A6
:1028320000000000000000008836040800000000CC
:10284200000000004D0203081027000001000000F4
:102852000000000000000000000000000000000076
:10286200000000000000000000000000C830040862
:102872000000000000000000899002081A410000D8
:102882000100000000000000000000000000000045
:102892000000000000000000000000000000000036
:1028A2009C4B0408000000000000000005A603087D
:1028B200400D0300000000000000000000000000C6
:1028C2000000000000000000000000000000000006
:1028D20000000000A44B04080000000000000000FB
:1028E200C1A50308400D0300000000000000000025
:1028F20000000000000000000000000000000000D6
:102902000000000000000000AC4B040800000000C2
:1029120000000000E1B80108A086010003000000E9
:1029220000000000000000000000000000000000A5
:1029320000000000000000000000000030303030D5
:102942002D30312D30315430303A30303A30300081
:10295200010100000000000001020304010203045F
:1029620006070809040309041201000202020040DA
:1029720083044057000201020301000009024300E0
:10298200020100C032090400000102020100052414
:10299200001001052401000104240202052406009E
:1029A20001070582030800FF09040100020A000072
:1029B20000070501024000000705810240000000F7
:1029C200FF0000004589030885860308E56B0308BC
:1029D20099840308F1880308A9840308C5840308BD
:1029E20089840308798403080000000000000000C5
:1029F2004300000000000000000000000000000092
:102A020000000000000000000000000000000000C4
:102A12004300000000000000000000000000000071
:102A220000000000000000000000000000000000A4
:102A32004300000000000000000000000000000051
:102A42000000000000000000000000000000000084
:102A52004300000000000000000000000000000031
:102A62000000000000000000000000000000000064
:102A72004300000000000000000000000000000011
:102A82000000000000000000000000000000000044
:102A920043000000000000000000000000000000F1
:102AA2000000000000000000000000000000000024
:102AB20043000000000000000000000000000000D1
:102AC2000000000000000000000000000000000004
:102AD20001B7030841B50308000000005350040881
:102AE2002F420408B93F0408B93F0408B93F04085B
:102AF200B93F0408B93F0408B93F0408B93F0408C4
:102B0200B93F0408B93F0408FFFFFFFFFFFFFFFFC3
:102B1200FFFFFFFFFFFF000001004153434949004F
:102B220000000000000000000000000000000000A3
:102B3200000000000000000000004153434949002A
:102B42000000000000000000000000000000000083
:102B520000000000000000000000000050240020DF
:102B62000000000000000000000000000000000063
:102B72000000000000000000000000000000000053
:102B82000000000000000000000000000000000043
:102B92000000000000000000000000000000000033
:102BA2000000000000000000000000000000000023
:102BB2000000000000000000000000000000000013
:042BC200010000000E
:10800000002870B51EDB0928044620DD012303EBA0
:1080100083035B00B0FBF3F2092AF8D87BB10E4E64
:10802000B4FBF3F00928CCBF57223022A6FB03E5AE
:10803000024403FB1044EB0801F8012BF0D10023AC
:108040000B7070BD2D230B7040420131DBE73030E7
:1080500001F8010BF3E700BFCDCCCCCC884230B4A3
:108060004FF001042ED301FB04F4B0FBF4F58D4274
:10807000F9D284B1AAB901E0B0FBF4F5092DCCBF67
:10808000572230222A4404FB150003F8012BB4FBCD
:10809000F1F4002CF0D100221A7030BC7047B0FB14
:1080A000F4F5092DCCBF372230222A4404FB1500F9
:1080B00003F8012BB4FBF1F4002CF0D100221A706C
:1080C00030BC70470546002AEBD1D7E703685A1C3D
:1080D00002601970704700BF2DE9F047089C2578B1
:1080E000002B804689460CBF4FF0200A4FF0300A23
:1080F000661C35B3002A29DD334601E0024698B1FB
:1081000013F8011B501E0029F8D1971E60B13D469F
:10811000013D51464046C8476B1C002BF8DC2578D2
:1081200027EAE770013055B1041B29464046C8478D
:10813000301916F8015B002DF7D1BDE8F087BDE8D6
:10814000F087002A04DC2846BDE8F0870020EBE732
:10815000571EDCE783684268D0ED037A00EB8301A9
:108160000133934281ED040A836004BF00238360DE
:1081700000EB830393ED047A036870EE277A9A424A
:10818000C0ED037A77EEC77AC0ED037A0CDA0133DB
:1081900007EE103AF8EEC76AB7EE007A87EEA60A45
:1081A000036030EE070A704707EE102AB8EEC77A70
:1081B00087EE870A704700BF90ED057A90ED004A80
:1081C000D0ED066AD0ED014AD0ED047A90ED035A65
:1081D000D0ED025AA4EE007AB0EE406AB0EE470A43
:1081E000B0EE667AA6EE247A67EEC07AA0EE457A03
:1081F000E6EE257A80ED057AC0ED067A704700BF7D
:10820000D0ED057A90ED013AD0ED003AD0ED064A76
:1082100090ED024A90ED077A90ED035A90ED086ACE
:10822000D0ED045AC0ED067AF0EE406A27EE830ADC
:10823000C0ED056AA3EEA60A80ED087AA4EE240A32
:10824000A5EE470AA5EEC60A80ED070A704700BFF3
:10825000D0ED007A90ED017A30EE670AE7EE007A11
:10826000B0EE670AC0ED007A704700BF704700BFEC
:108270000A44914214D030B40139551E41F2210212
:1082800011F8014F082380EA042004044CBF82EA5D
:1082900040004000013B80B2F7D18D42F0D130BCAC
:1082A000704700BFF0B540F6280340F62C0240F6B8
:1082B000360540F6210440F64D1140F66A1740F6A7
:1082C000E1060380428040F6791340F68112458131
:1082D000848140F6611540F6DA04C18140F633012D
:1082E0000782468240F6F70740F6A7168382C282CD
:1082F00040F6C71340F6E7120583448340F6411564
:1083000040F65914818340F64911C783068440F62C
:108310004C0740F601064384828440F6011340F680
:108320002112C584048540F6410540F62F1441858D
:1083300040F62E118785468640F60A1740F68816C5
:108340008386C28640F6C80340F652020586C4877B
:1083500040F68A0540F63714818740F61711A0F8D9
:10836000447006878380C380038140F6530CC28526
:1083700014234FF0013E4FF0011745874FF00126BF
:10838000A0F846200125A0F84040A0F842100B4C70
:108390000B49A0F848C02822C0F84AE0C0F84E7047
:1083A000C0F8526080F85B50C465C0F8561080F881
:1083B000612080F85A3080F86030F0BD000A010A70
:1083C000980864004FF480538382704750F8043C4F
:1083D000012280F84520103803B11847704700BFCC
:1083E000BFF34F8F0549064BCA6802F4E06213439E
:1083F000CB60BFF34F8F00BFFDE700BF00ED00E093
:108400000400FA0570B4037B04681F2B08D9203BD5
:108410002021626801FA03F31A421CD170BC704734
:108420002021226801FA03F31A42F7D04269144965
:10843000582000FB021251685689CD6808682968E7
:1084400021F001012960828992B222EA060282812A
:10845000A36070BC704742690949582000FB0212B2
:1084600051685689CD680868296821F001012960A2
:10847000828992B222EA06028281E36070BC704770
:10848000AC76002030B4094B1C786CB1084A00254A
:1084900002EBC404116893884D6288890832034353
:1084A0009BB2A2428B81F5D130BC70476C79002021
:1084B0007079002010B4037B01681F2B09D9203B81
:1084C00020224C6802FA03F31C4214D15DF8044BDD
:1084D000704720220C6802FA03F31C42F6D00C4AC3
:1084E00040680024147002685DF8044B22F0010219
:1084F00002608B607047064A40680024147002686E
:108500005DF8044B22F001020260CB60704700BFAF
:10851000377F002070B5044682B00830656A0623B4
:108520006A463B21A847A8B19DF804009DF8006069
:108530009DF801109DF802509DF803209DF805302C
:1085400041EA062143EA002342EA0522E18222832E
:108550006383012002B070BD2DE9F0410446164D41
:10856000084616460F4632F0BFF82A6802301168F6
:108570009072D4723B4610464F6922460221B8479A
:1085800028680E4B0268C472152181725769142144
:108590002246B847304632F0A7F8296816300D68F1
:1085A0008872CC7222466C6933460846A44616216E
:1085B000BDE8F041604700BFB42400200810040863
:1085C000014B186804F020BB78A7002038B5054699
:1085D00000BF084C2368986804F006FF236829460A
:1085E000586805F08DF82368986804F003FF00BF11
:1085F00038BD00BF687C0020F0B5044690F85900F3
:1086000083B0002840F0AA806A4E3779002F43D00B
:1086100004F114054FF48071A06905F0A9F894F8ED
:1086200052201A21284603F057FC012004F07CF860
:108630000421A06905F09CF828460623E56D6A46EA
:108640004321A847D8B19DF802609DF803309DF8FA
:1086500000509DF801109DF804009DF8052043EAA4
:1086600006231BB2E3875BB241EA052142EA0022FE
:108670000133A187A4F8402006D003B0F0BDB4F9BF
:108680003E305BB20133F8D194F93C300133F4D180
:10869000062003F0ADFDF0E704F114054FF48071FE
:1086A000A06905F065F880226B21284603F014FCD0
:1086B000962004F093F803226821284603F00CFC6E
:1086C000962004F08BF803226B21284603F004FC6B
:1086D0000F2004F029F810226A21284603F0FCFB41
:1086E0000F2004F021F83A466C21284603F0F4FBF1
:1086F0000F2004F019F894F854201921284603F0AB
:10870000EBFB0F2004F010F818221B21284603F081
:10871000E3FB0F2004F008F810221C21284603F088
:10872000DBFB0F2004F000F810223721284603F06D
:10873000D3FB0F2003F0F8FF01223821284603F075
:10874000CBFB0F2003F0F0FF0421A06905F010F827
:10875000012003F0E9FF012333715BE704F0FAFB2A
:108760000546D8B1202300218371C17104F084FD36
:108770002146114B41F8103F284631F039FDAB88B6
:10878000B3FA83F3C3F11F03012212FA03F33FF498
:108790003BAF0A490A6813430B6035E7014604F012
:1087A0006BFD2146044B41F8103F284631F020FD77
:1087B0002AE700BFB4240020CD830008003C01401C
:1087C000F8B5057B466903681F2D29D9A5F120045A
:1087D0005F682021A1400F422A4613D01022A240F8
:1087E000D960DA605A68E240D10703D5012202FA63
:1087F00004F4DC600446304604F092F9227B2368DE
:108800001F2A20D9A2F1200008215A688140114274
:1088100000D0D9600422596882400A4221D1F8BDB3
:1088200020211C68A9400C422A460CD01022AA40E4
:1088300099609A601A68EA40D207DBD5012202FAF1
:1088400005F59D60D6E7082118689140014200D0E7
:1088500099600421186801FA02F2024203D09A607A
:10886000F8BDDA60F8BDF8BD70B582B0044669465F
:10887000143031F02BFDB0B19DF805009DF801607A
:108880009DF802109DF803509DF804209DF80630D5
:1088900041EA062143EA002342EA0522A187E28752
:1088A000A4F84030012002B070BDF8B5174D2B7808
:1088B000A32B28D16B78BE2B25D1022229464FF657
:1088C000FF70FFF7D5FC124FAC1C22884AB1A618E6
:1088D000BE4218D2052A16D92146FFF7C9FC3446F4
:1088E000F3E721460222FFF7C3FC0222A118FFF79B
:1088F000BFFC0634074B641B1C8041F60F53C31AA0
:1089000058425841F8BD0020F8BD00BF00400008A3
:1089100000800008E83E00202DE9F04FDFF84C9180
:108920004D4F8BB00326A7EB09071822002104A89E
:1089300035F02FF9494BCDF8109005971A69002AA8
:1089400004DA474A5A6002F188325A6001228DF8EF
:108950002420F322DA60434B434C1B88ADF80030EF
:108960000222694604A805F0C3F9022269464FF6BF
:10897000FF70FFF77DFCDFF8F8A080464FF0000B9A
:10898000544539D30AAC002524F8245D022221463F
:1089900004A805F0ADF9022221464046FFF768FC25
:1089A00040BAC043ADF80800022202A904A805F0AD
:1089B0009FF9079878B106ABC0F104022946184424
:1089C00035F0E7F8089818B9069904A805F0F2F808
:1089D0000023089007939DF82430089A23B11F497B
:1089E0000B6943F000430B61013E2DD0002A9CD15E
:1089F000FFF75BFF50B32CE065888DF80DB0C5F331
:108A00000B05AB1DADF808302388C3F30B02ADF89E
:108A10000A201B0B062202A904A88DF80C3005F0D1
:108A200067F9062202A94046FFF722FC61688046EA
:108A30002A4604A805F05CF9616840462A46FFF71B
:108A400017FC143480469BE7002AD1D0052003F0A0
:108A5000CFFB0BB0BDE8F08F00800008003C024067
:108A600023016745FCDC030888010008004000087A
:108A7000100600080378202B024600F10100F9D00F
:108A8000092BF7D02D2B2CD02B2B03BF5378B7EE0F
:108A9000000A0246B7EE000AA3F13001C8B2092865
:108AA0009FED467A10D8F2EE046A07EE901AF8EEBF
:108AB000E77A12F8013FE7EE267AA3F13001C8B257
:108AC0000928B0EE677AF0D92E2B4CD003F0DF03E3
:108AD000452B0BD0F7EE007A67EE276A20EE260AC8
:108AE00070475378BFEE000A0246D5E710B45178BC
:108AF0002D2959D02B290ABF9178501C901C002495
:108B0000A1F13003092B53D8002303EB830301EBBE
:108B1000430310F8011FA1F13002092AA3F1300329
:108B2000F3D9B3F59A7F28BF4FF49A73072B42D934
:108B3000DFED236A1A46F7EE007A083A072A67EE55
:108B4000A67AFAD803F007032BB1F2EE046A013BD0
:108B500067EEA67AFBD124B3C7EE276A5DF8044B13
:108B600020EE260A70475378A3F13001C8B20928D5
:108B700002F10102AAD8F2EE046AF0EE665A07EE9C
:108B8000901AF8EEE77A12F8013F87EEA66AA3F191
:108B90003001C8B2092866EEA56A37EE067AEED92A
:108BA00094E767EE276AD9E7901C91780124A7E73C
:108BB000F7EE007ACFE7F7EE007AC5E70000000095
:108BC00020BCBE4CB5EEC00ADFED317AF1EE10FAF2
:108BD000CCBF30EE270A30EE670ADFED2E7A20EEAA
:108BE000270A30B5FDEEC07A87B017EE904A0546E9
:108BF00084EAE470002303A9A0EBE47001930093DE
:108C0000029326F0BDFC002CACBF20232D2303A82B
:108C10008DF8003031F068FD012803A924D0022826
:108C20002DD0032805BF3023684668468DF80130F3
:108C300034F0D5FF684631F057FD0338C4B2224600
:108C40006946284635F029F800232B55284631F08F
:108C50004BFD2E22431C2A540DEB0401E81834F07E
:108C6000DBFF284607B030BD302368468DF8013061
:108C70008DF802308DF8033034F0B1FFDAE730239D
:108C800068468DF801308DF8023034F0A8FFD1E746
:108C90006F12033A00007A442DE9F041064615466A
:108CA0000846B6FBF2F43CB905FB1464124B1B5D9D
:108CB00000F8013BBDE8F081B4FBF2F767B90E4B59
:108CC00005FB174705FB1464DA5D00F8012B1B5DFB
:108CD00000F8013BBDE8F081B7FBF2F8B8F1000FF6
:108CE00002D04046FFF7D8FF05FB1878024B13F877
:108CF000082000F8012BE3E70C10040830B40268E8
:108D00001146531C036011F8024B0160D31C5178CB
:108D100003609378151D05601B0443EA0123D07896
:108D2000234343EA006030BC704700BF0368591C0E
:108D30001A46016012F8021B0260587841EA0020CE
:108D4000704700BF03685A1C02601878704700BF64
:108D500038B504460068154632F004FC22682A44FF
:108D6000226038BD036810B40A0E5C1C04601A70DF
:108D700003680A0C5C1C04601A7003680A0A5C1C15
:108D800004601A7003685A1C026019705DF8044B85
:108D9000704700BF036810B40A0A5C1C04601A70B4
:108DA00003685A1C026019705DF8044B704700BFDD
:108DB00003685A1C026010B4197003680A0A5C1C2C
:108DC00004601A7003680A0C5C1C04601A70036863
:108DD000090E5A1C026019705DF8044B704700BF01
:108DE00003685A1C026019700368090A5A1C026061
:108DF000197070472DE9F047002488B080460F466F
:108E00001E46A14605AD531C0393117839B325299D
:108E100033D1931CCDF810900393507830284ED066
:108E20004FF0000AA0F13003DBB2092B42D96C28C5
:108E300019D0642800F0938024D825281CD063D949
:108E4000582876D063281BD131784046B847039A1A
:108E5000531C03931178043601340029D7D12046DE
:108E600008B0BDE8F087039B5A1C03921B78642B63
:108E70007CD02AD8252B54D1252140460134B8472F
:108E8000039AC0E7732833D044D975284FD106F12F
:108E9000040E30682B4600220A217646FFF7DEF8E2
:108EA000049A0095534639464046FFF715F9039A50
:108EB0000444A8E704AA03A926F03EFBB7E7D31CA5
:108EC000039390784FF0010AACE7732B10D05BD975
:108ED000752B3AD0782B96D1A3F15802B2FA82F2D0
:108EE000306852092B4610210436FFF7B7F8D7E750
:108EF0003368049A0093394600234046FFF7ECF8A4
:108F000004360444039A7EE70028B9D1204608B00D
:108F1000BDE8F0876E28B3D1039A336804361C602D
:108F200071E72AD9582BD7D0632B8DD06BE77828DF
:108F3000A6D1A0F15802B2FA82F2306852092B464B
:108F40001021FFF78BF80436AAE706F1040E30680B
:108F50002B4600220A217646FFF780F8A0E7331D52
:108F6000306829461E46FFF74BF899E7331D3068F5
:108F700029461E46FFF744F892E7002B7FF443AFE3
:108F8000204608B0BDE8F0876E2BC6D03BE700BF97
:108F90000EB400B584B005AB019053F8042B06491C
:108FA000039301A8FFF726FF019B00221A7004B06B
:108FB0005DF804EB03B07047CD8000080FB430B506
:108FC00083B006AB0A490B4853F8042B09680068C4
:108FD0000193FFF70FFF084C0546206803F000FEE1
:108FE0000028FAD0284603B0BDE8304004B07047EE
:108FF000FC3D0020003E002078A70020DFED2B7A0A
:10900000B4EEE70AF1EE10FA4ADDDFED296A9FEDD2
:10901000297A01E0B0EE670AB4EEC70AF1EE10FA61
:1090200070EE667AF6DC9FED247AF4EEC77AF1EE04
:1090300010FA38D5DFED1E6A9FED207A01E0F0EEE0
:10904000407AF4EEC77AF1EE10FA37EEA60AF6D4BB
:10905000DFED1B7AB4EEE70AF1EE10FA14DDDFED76
:10906000137A37EEC00A60EE006A9FED166A9FED34
:10907000167ADFED167AA6EE867A20EE266AE6EEFE
:10908000877AA6EE270A7047DFED117AB4EEE70A79
:10909000F1EE10FA44BFDFED087A37EEC00AE2E7DE
:1090A000F0EE407ABFE7B0EE670AD1E7DB0F494048
:1090B000DB0FC940E4CB1641DB0F49C0E4CB16C13E
:1090C000DB0FC93F92E741B99730083C15A82ABE8B
:1090D000DB0FC9BF09B909E0194690FBF1F301FBA9
:1090E00013030846002BF7D1084670470146FBE7FB
:1090F000F0EEC07AB0EEE07AB4EEE77AF1EE10FA74
:10910000B4BFB0EE676AB0EE476AB5EE406AF1EE02
:1091100010FA46D0B4EEE77AF1EE10FA8CBFF0EE1A
:10912000675AF0EE475AC5EE866A9FED1F3A9FEDEB
:109130001F6A9FED1F4A9FED1F5ADFED1F3ADFEDBB
:109140001F4ADFED1F5AA6EEC36AE6EEA34AA6EE5B
:10915000864AB7EE006AA6EE845AA6EEA46AE6EE48
:10916000855AC5EE866AB4EEE77AF1EE10FA48BF8A
:10917000DFED147AF5EEC00A48BF77EEE66AF1EE4D
:1091800010FA48BFDFED107AB5EEC00A48BF77EE9F
:10919000E66AF1EE10FA48BFF1EE666AB0EE660AD2
:1091A0007047DFED076ADEE739094E3DE3B59E3EC5
:1091B00088FA163E45FE7F3F99FB243F69A2163E82
:1091C000A7DFA834DB0FC93FDB0F4940DFED317A61
:1091D00030EE277AFDEEC76A16EE903A2033402B28
:1091E00002D99FED2D0A7047B4EEE70AF1EE10FAAE
:1091F0004DDD9FED2A6ADFED2A6A01E0B0EE677A65
:10920000B4EEE67AF1EE10FA77EE467AF6DC9FEDF0
:10921000257AF4EEC77AF1EE10FA35D5DFED1F6A44
:109220009FED217A01E0F0EE407AF4EEC77AF1EE9C
:1092300010FA37EEA60AF6D4DFED167AB4EEE70A96
:10924000F1EE10FA1BDCDFED197AB4EEE70AF1EE6D
:1092500010FA44BFDFED137A37EEC00A60EE006A01
:109260009FED136A9FED137ADFED137AA6EE867AEF
:1092700020EE266AE6EE877AA6EE270A7047DFED33
:109280000F7A37EEC00AE9E7B0EE670AD4E7F0EEEE
:10929000477ABCE7DB0FC93F00000000DB0FC94085
:1092A000E4CB1641DB0F49C0E4CB16C1DB0FC9BFCD
:1092B00092E741B99730083C15A82ABEDB0F494018
:1092C000FDEEC07A17EE903A2033402B51D8DFEDF7
:1092D0002D7AB4EEE70AF1EE10FA50DDDFED2A6ADE
:1092E0009FED2A7A01E0B0EE670AB4EEC70AF1EE0C
:1092F00010FA70EE667AF6DC9FED257AF4EEC77A06
:10930000F1EE10FA38D5DFED206A9FED227A01E008
:10931000F0EE407AF4EEC77AF1EE10FA37EEA60AD4
:10932000F6D4DFED1D7AB4EEE70AF1EE10FA1BDC9D
:10933000DFED1A7AB4EEE70AF1EE10FA44BFDFED82
:10934000147A37EEC00A60EE006A9FED156A9FED51
:10935000157ADFED157AA6EE867A20EE266AE6EE1D
:10936000877AA6EE270A7047DFED067A37EEC00A45
:10937000E9E79FED0E0A7047B0EE670AD1E7F0EE1D
:10938000407AB9E7DB0F4940DB0FC940E4CB164117
:10939000DB0F49C0E4CB16C1DB0FC93FDB0FC9BFF0
:1093A00092E741B99730083C15A82ABE000000009A
:1093B00010B507EE901A2DED028BB8EE678ADFED3F
:1093C000217A28EE008A044628EE278AB0EE480A61
:1093D00032F01EFBF0EE408AB0EE480A32F07AFA24
:1093E000F7EE007A9FED187AF0EE675AE8EE875AAA
:1093F0000023A361B0EE676AC7EEA56A63612362CA
:10940000E361A8EEC76ABDEC028B77EEC07AB6EED8
:10941000007AF8EE005A27EE877A20EE250A27EE2A
:10942000267A26EE266A67EEA67A20EE260A84EDD4
:10943000046AC4ED017A84ED007A84ED027A84ED49
:10944000030A10BD27D4D236F304353F10B44C09BB
:10945000012250F8243001F01F0102FA01F10B4300
:1094600040F824305DF8044B704700BF4B0901F011
:109470001F0150F82320012303FA01F1114214BF08
:1094800018460020704700BFAA4B33F81020110582
:1094900013D52DE9F043A8490446400904F01F05FF
:1094A00051F820000121A940014291B006D0A34902
:1094B000097819B111B0BDE8F083704702F01F07B9
:1094C000C2F34415242CF5D8DFE814F0430055000E
:1094D0009000A2005201960196019B044A036A0380
:1094E0007002A002BA02C502D802E302F402FD0231
:1094F000C901CB04BD040A05D9010D020D023702D2
:109500004A024A028E03EF03FC030D041E048F047B
:10951000510480042500DFF85482D8F820200AB1D5
:10952000B2F90820864908AE3046FFF731FD3046D3
:1095300031F0DAF8D8F800403844A0722068E572BB
:109540002A463346456939462046A84711B0BDE84A
:10955000F0837C4B7C491A88DFF81082642303FB7C
:1095600002F39B1208AE632BA8BF6323304601228F
:10957000FFF70EFDDBE7754B754A1B781088022B51
:1095800000F00785734B744C5A781978247802EBF5
:109590008202520000EB800301EB81015B0093FB30
:1095A000F4F39B1AC3EBC303C2EB410293FBF2F348
:1095B000062BA8BF062323EAE373C3F19603DBB2AD
:1095C000664A8DF82030A2FB0032D20802EB8203FB
:1095D000A0EB4303624906209BB200900DF12100ED
:1095E000FFF7D6FC08AEDFF88481A0E7DFF87C81C6
:1095F000D8F8000003681B69984710AEB0F5F07FFB
:10960000584B46F8203D0CBF072506250D278EE751
:1096100093F86120544993F86060B1F9000002EBBF
:10962000820253005F4206EB8606B8424FEA4606C6
:1096300003DB8342A8BF03461F46B1F902307542DF
:10964000AB4203DBB342A8BF33461D46DFF81C81A3
:10965000D8F8000003681B699847B0F5F07F05EB68
:10966000850518BF0224BB0048BF3F3305EB8505C5
:1096700095FBF6F6293EC6EBA313512B40F22A8642
:1096800007EB4705002D2B46B8BF05F13F03C6EB9E
:10969000A313512B40F20186ED1B002D2B46B8BFC2
:1096A00005F13F03C6EBA313512B40F2D985ED1B07
:1096B000002D2B46B8BF05F13F03C6EBA313512B7A
:1096C00040F28A85ED1B002D2B46B8BF05F13F0304
:1096D000C6EBA313512B40F2E184ED1B002D2B466A
:1096E000B8BF05F13F03C6EBA313512B40F2B98479
:1096F000ED1B002D2B46B8BF05F13F03C6EBA313AE
:10970000512B40F29184ED1B002D2B46B8BF05F183
:109710003F03C6EBA313512B40F26984ED1B48BFF6
:109720003F35C6EBA516512E40F2FA840420FFF710
:10973000ABFEBFE694580020206600200000002009
:1097400084100408887F002054100408907F0020B3
:10975000E87D0020D4A60020FE7D0020CDCCCCCC1E
:109760005C100408267E2700CCA60020B42400202C
:10977000DFF8E883D8F8000003681B699847B0F564
:10978000F07F0CBF0727062707F1040614BF032448
:1097900004240825D8F800000368C4728572D3F841
:1097A0001890224613230721C847D8F80000162234
:1097B0000368C472827222460134D3F818901521CE
:1097C0001323E4B2C847A642E4D1D8F80000092226
:1097D0000368C77282729C693A4603230821A04736
:1097E000D8F8000015220368C77282729C693A4655
:1097F00002231421A0475DE603EB4403B3F8523083
:1098000013F00F0200F0DC83022A8CBF20219C2180
:10981000012AC3F303148DF8201000F0D685C0F0A0
:10982000D483022A00F0BE850023DFF830831A4675
:109830001846012C40F0B083A74EA84CA849A6FBBF
:109840000060400BA4FB00646409642606FB14005E
:1098500000900DF12100FFF79BFB08AE67E6A14BDE
:10986000A14A1868A149047A83790194C0790090CB
:1098700008AE3046FFF78CFBDFF8E08257E69C4BE2
:109880009C4A1B8812789C4903EB8303022A0978BF
:109890004FEA430393FBF1F300F07983974A517841
:1098A000127801EB8101490002EB82005A1AC2EBE7
:1098B000C202C1EB400192FBF1F2062AA8BF0622C8
:1098C00022EAE272C2F19602D2B284488DF82020D8
:1098D00080FB0320DA17C2EB60126424884906205B
:1098E00004FB123379E6874A874B8849DFF86C829C
:1098F00092E84100182C08BF064683FB06234FEA76
:10990000E672C2EBA35203A814BF602364238DF850
:109910002030FFF73DFB32467C4905A8FFF738FBB6
:1099200003A830F0E1FE05AB034403AA78490DF12A
:109930002100FFF72DFB08AEF9E576487649B0F92E
:109940000230B0F90020B0F90640B0F904000090F0
:1099500008AE01943046FFF71BFBDFF80082E6E516
:109960006E4B6F486F49DFF8F4811A2C0CBFB3F9C6
:109970000220B3F9002080FB0230D317C3EBA00410
:1099800004EB8400A2EB400383EAE370002AA0EB1F
:10999000E37008AE84EAE4730090ACBF20222D226D
:1099A000A3EBE4733046FFF7F3FAC0E55E4E31688F
:1099B00000248DF80B408DF80C40002900F02D8517
:1099C0000A68D269002A00F00A8503A90DF10B008C
:1099D000904731688DF8144031B10B68196A19B19C
:1099E00005A888479DF814109DF80C404F489DF835
:1099F0000B204F4B825C009108AE53F824304D4948
:109A0000DFF858813046FFF7C3FA90E54A4B3348F8
:109A10001B684A49DFF8448183EAE37EAEEBE37ECC
:109A200080FB0E304FEAEE72C2EB601208AE64208B
:109A30009A2400FB12E300943046FFF7A9FA76E57A
:109A40003D4B3F499A68DFF8148108AE3046072342
:109A5000FFF79EFA6BE52B4B3A4ADB893A49DFF870
:109A6000FC8003EBC3039B0082FB030208AEDB1701
:109A7000C3EBA2123046FFF78BFA58E5214B33496E
:109A80001B7DDFF8D88008AE30461F22FFF780FA32
:109A90004DE593F85B302E49DFF8C080002B0CBFFA
:109AA0000F220C2208AE0023009230461A46FFF720
:109AB0006FFA3CE50B4B274A18680C498478037809
:109AC00001944078D3E6074B234A18680749447944
:109AD000C37801940079CAE65917B7D11F85EB51B5
:109AE000B01004085C590020F0100408DC100408D1
:109AF000E87D0020907F0020FE7D0020D4A600207D
:109B00003C110408F0A600206BCA5F6B84100408A7
:109B100088100408087D002048110408CCA6002005
:109B2000676666665C110408A84B00206C01040897
:109B300074010408CC100408B4A4002068100408C0
:109B400074100408D34D62107C10040854100408EB
:109B500098100408D8100408EC100408B42400205D
:109B6000C54B1A78002A00F0B6825C1E03F10F087C
:109B70000DF11F09667831F0D5FC30443246437848
:109B800003F00303022B14F8013F08BFA6F12002E3
:109B900009F8012F002B00F08480A045EAD180E075
:109BA000B64BB74AB3F90630B649DFF81C83B3F5B4
:109BB000FA6FA8BF4FF4FA63B3F57A7FB8BF4FF4DA
:109BC0007A73A3F57A7382FB0302DB17C3EBA2025D
:109BD000042405230DF122008DF820408DF821305A
:109BE00008AEFFF7D5F9A2E4A74BA84A1B899268F3
:109BF000A7499A1A9A42A8BF1A4622EAE27207EEC9
:109C0000902AA1FB0313DB08B8EEE77A07EE903A3F
:109C1000F8EEE77AC7EE276A16EE900A30F0D0FE2B
:109C200041EC100B31F07CFD51EC100B31F0B6F92A
:109C30008A23C0B28DF82030002840F09E818D2309
:109C40008DF821308D238DF82230022800F26B81AF
:109C50008D238DF823308D238DF824308D238DF8BE
:109C600025308D238DF826308D238DF827308D23D8
:109C70008DF828308D238DF829308D238DF82A30EA
:109C80008D238DF82B30431E8F22092B8DF82C202D
:109C900004D810AB18448E2300F81F3C00238DF825
:109CA0002D3008AEDFF8208241E47A4B1B78DB07C9
:109CB0003FF500AC08AE30467749DFF80C82FFF77D
:109CC00067F934E4754B1B7803F00303032B00F0B2
:109CD00019832D238DF8203000238DF8213008AE14
:109CE000DFF8E48123E46D4A127802F00302032ACC
:109CF00000F03B832D2200238DF820208DF82130A9
:109D000008AEDFF8C48112E4654B5D4AB3F9043054
:109D100064486549DFF8B08182FB0342DB17C3EB7F
:109D2000A2031BB2162404EB430480FB0462161941
:109D3000E217C2EB66224FF4347606FB124280FB38
:109D400002401044D217C2EB6012D2B2C2F1180224
:109D5000504200F00F0002F00F0258BF4242603242
:109D600008AED2B23046FFF713F9FFF7E0BB4C4B19
:109D7000434CB3F904304B484C49DFF84C8184FB29
:109D80000324DA17C2EBA4021623022412FB0432C6
:109D900080FB02439C18D317C3EB64234FF4347445
:109DA00004FB132380FB03021A44DB17C3EB62138B
:109DB00051FA83F308AE186859681C7A334603C316
:109DC00000221C708DF82920FFF7B1BBDFF8F88066
:109DD000D8F820200AB192F90120354908AE304662
:109DE0000E23FFF7D5F8FFF7A2BB08AE00233046DD
:109DF000009368222F49DFF8D080FFF7C9F8FFF7FA
:109E000096BB2D4B1B68DC0040F1CE802B4B032210
:109E10002B490988480500F18380CE0700F1BF82F5
:109E200001F00201274800291CBF032203462649EE
:109E300008683A4404688272C57239462A466469E1
:109E4000A047FFF737BB214A214953781278DFF842
:109E5000788008AE013301323046FFF799F8FFF7FA
:109E600066BB1C4A094B10881B681B4A1B49DFF85C
:109E7000588003FB00F3F7E548840020607F002052
:109E80006766666684100408D4A60020B4A4002087
:109E9000A38B2EBA747D002068110408ECA6002064
:109EA000CCA60020B7600BB67411040800DD0308CF
:109EB000901004087C110408208400203410040849
:109EC0008A7F002050100408B4240020A0740020D1
:109ED000FC100408E87D0020D34D6210F410040843
:109EE0000021CC48FFF7C2FA002840F03281CA4B6B
:109EF0001B7813F0020FC94B1B7802D1002B00F026
:109F00007882012B00F00381022B40F0F28008AE32
:109F10003046C349DFF84483FFF73AF8FFF707BB41
:109F20000422C04B83E78B2303288DF823307FF670
:109F300092AE04288DF824307FF690AE05288DF877
:109F400025307FF68EAE06288DF826307FF68CAE53
:109F500007288DF827307FF68AAE08288DF828303C
:109F60007FF688AE09288DF829307FF686AE0A285C
:109F70008DF82A303FF685AE82E68B2301288DF8D6
:109F8000213018BF8DF822307FF45FAE5AE6972259
:109F90009BE49723FFF714BBA3490DF12100FEF7C3
:109FA000F7FF08AEFFF7C3BAA04AA1491268A14B58
:109FB00002F48002002A0ABF0B460322042227E78C
:109FC0009B22C3F303148DF8202002F061FB9A4B0F
:109FD0009A4ADFF88882A3FB00139B0C82FB0312D2
:109FE0001A445211C2EB0211A3EB810321E49449FC
:109FF000D8F8000081FB0321DA17C2EB610204EB01
:10A00000020E02EBC2015B1A5FFA8EF20168C272A5
:10A010004FF0120E80F80AE0803BD1F81890DBB2C6
:10A020001121C847FFF77ABB8549D8F8000081FBAA
:10A030000321DA17C2EB610204EB020E02EBC2014C
:10A040005B1A5FFA8EF20168C2724FF0110E80F84F
:10A050000AE0803BD1F81890DBB21021C847FFF727
:10A0600052BB7749D8F8000081FB0321DA17C2EB15
:10A07000610204EB020E02EBC2015B1A5FFA8EF280
:10A080000168C2724FF0100E80F80AE0803BD1F8F0
:10A090001890DBB20F21C847FFF72ABB6849D8F8F0
:10A0A000000081FB0321DA17C2EB610204EB020E10
:10A0B00002EBC2015B1A5FFA8EF20168C2724FF0C6
:10A0C0000F0E80F80AE0803BD1F81890DBB20E2129
:10A0D000C847FFF702BB5B4BDFF8808193E80700BE
:10A0E00008AE334603C323F8022B120C1A70FFF795
:10A0F0001EBADFF8688198F81C30002B3FF4DAA90B
:10A1000008AE30465049FEF743FFFFF710BA08AEDD
:10A1100030464E49DFF84481FEF73AFFFFF707BAB1
:10A12000474AD8F8000082FB0632F317C3EB6203FC
:10A13000E21803EBC3031324D2B2F61A0168C27209
:10A14000A6F1800384728C69DBB21221A047FFF76D
:10A15000EDBA3F4B1B88002B3FF4C9AEDC0700F182
:10A160006081C3F340025ABB580700F1748119079C
:10A1700000F16F81DA0600F16A819E0600F16581C7
:10A180005C0600F16081180600F15B81D90500F1E1
:10A1900056819A0500F151815E0500F14C811C0544
:10A1A00000F14781D80400F14281990400F13D811A
:10A1B0005A0400F13881DB0B18BF0F223FF471AD58
:10A1C000244B254953F82220DFF8908008AE304612
:10A1D000FEF7DEFEFFF7ABB91949D8F8000081FBA6
:10A1E0000321DA17C2EB610204EB020E02EBC2019B
:10A1F0005B1A5FFA8EF20168C2724FF00E0E80F8A1
:10A200000AE0803BD1F81890DBB20D21C847FFF778
:10A2100059BA00BF20840020747D0020907F002068
:10A220002411040840100408A4100408D879002060
:10A23000381004083410040883DE1B43898888889A
:10A24000398EE338C01004083011040818110408CE
:10A25000B87F002090E7030804110408B42400200C
:10A260007E49D8F8000081FB0321DA17C2EB6102B6
:10A2700004EB020E02EBC2015B1A5FFA8EF2016878
:10A28000C2724FF00D0E80F80AE0803BD1F81890B2
:10A29000DBB20C21C847FFF70ABA7049D8F80000B2
:10A2A00081FB0321DA17C2EB610204EB020E02EB21
:10A2B000C2015B1A5FFA8EF20168C2724FF00C0E97
:10A2C00080F80AE0803BD1F81890DBB20B21C84738
:10A2D000FFF7E2B96149D8F8000081FB0321DA17E2
:10A2E000C2EB6102A51802EBC2015B1AEAB2016877
:10A2F000C2720B25803B85728D69DBB20A21A847AB
:10A30000FFF7BEB9564B1B88002B6CD0554B5648F7
:10A31000B3F90430554A5649B2F9002080FB034096
:10A32000DB17C3EBA0031BB2D21A5200163281FB1B
:10A3300002039818D317C3EB60234FF4347000FB6B
:10A34000132381FB03121A44DB17C3EB6213DBB246
:10A35000C3F118035A4202F00F0203F00F0358BF73
:10A36000534260338DF82030B6E43D4A93F85B30B9
:10A370001288002B3BD14FF4A4733E4903FB02F239
:10A3800081FB0213D217C2EB63120F2308AE3046D3
:10A390003949DFF80481FEF7FBFDFFF7C8B8374BFA
:10A3A000042244E5DFF8F0803549D8F81800354A32
:10A3B000A1FB0031890C82FB01320A445211C2EB2D
:10A3C0000213A1EB8303FFF734BADFF8CC802C4BE8
:10A3D000D8F808002B4AA3FB0013990CEBE78DF883
:10A3E0001420FFF7FABA05238DF8203074E40C230B
:10A3F000CCE7254A254B2649927B1B88097893FB9D
:10A40000F1F39A427FF675AE08AE30462149DFF887
:10A410008880FEF7BDFDFFF78AB88DF81410FFF7AE
:10A42000E3BA0022CCE60E22CAE60D22C8E60C22D0
:10A43000C6E60B22C4E60A22C2E60922C0E60822CA
:10A44000BEE60722BCE60622BAE60522B8E60422EA
:10A45000B6E60322B4E60222B2E600BF398EE33844
:10A46000D46C0020CCA6002067666666D66C0020FF
:10A47000B7600BB61F85EB51901004084810040814
:10A4800083DE1B4389888888D4A60020E87D0020CD
:10A49000FE7D002008110408B4240020074A084B60
:10A4A00010781B78074A834296BFC31AC3F1800312
:10A4B0000020126818441044704700BF98820020A2
:10A4C00014820020A85F0020064A074B10781B78F2
:10A4D00083428ABFC3F18003C01AC018C0F17F0055
:10A4E000704700BF988200201482002030B5144CC1
:10A4F000237883B01BB90120237003B030BD05223F
:10A5000000238DF800208DF8013000BF0D4D2B6821
:10A51000986802F069FF2B6801AA694658682FF015
:10A52000E5FC2B68986802F065FF00BF9DF80530D8
:10A5300003F0010383F00100237003B030BD00BFBE
:10A540007A7C0020687C002070B5064C06462568A1
:10A5500003E023685B1BB34203D8FFF7C7FF002863
:10A56000F7D070BD607C00202DE9F04F89B0B2F1CA
:10A57000000A02900491039340F3B0800B4600223E
:10A5800001EB8A0153F8040B8B420244FAD1039B7E
:10A590000592002B00F09A80059B002B6AD0544B4B
:10A5A000059A1B68DFF85C9100920099DAB25118A5
:10A5B000B1F5807F8CBFC2F58072009A01924D4A3E
:10A5C00092689A426DD9190C1A0A4FF002040620BB
:10A5D0008DF81F308DF81E208DF81D108DF81C4051
:10A5E000FFF7B2FF0620FDF7F1FF434A0123137086
:10A5F00000BFD9F80030986802F0F6FED9F80030B4
:10A6000007A9586800222FF023FC0024049D029E15
:10A61000019FA34629684FEA840800220B460134B3
:10A6200071B1B9422AD2D9F800003168406803F00C
:10A63000CBF82A68336813443360BF1AC5F800B0FA
:10A64000A24505F1040506F10406E3D1D9F800306E
:10A65000986802F0CFFE00BF254B019900981B6857
:10A66000421A0092224A0B441360039A32B3009AB2
:10A67000002A9AD1059809B0BDE8F08F029CD9F85C
:10A68000003054F80810586800223B4603F09CF84C
:10A6900054F808202B683A44DF1B44F808202F6048
:10A6A000D4E70598009C1549154A001B05900598AC
:10A6B00000230B70137009B0BDE8F08F059B009A62
:10A6C0009B1A0593059809B0BDE8F08FFFF70EFFC0
:10A6D00000287FF461AF039B0593CBE7039C1CB973
:10A6E000FFF704FF0594C5E700230593C2E700BF09
:10A6F000A85F0020D41D00207A7C002098820020D2
:10A7000014820020687C002070B5104D104E2B780C
:10A7100031788B4284B016D00E4A03921A440292CA
:10A720008CBF0C46CA1A04A98CBFC3F18002002456
:10A73000012341F8102D02A802220194FFF714FF13
:10A74000002333702B7004B070BD00BF1482002052
:10A75000988200201882002070B5194C194D23787A
:10A760002978994284B027D0174A03921A4402925A
:10A7700034BF0E46CA1A04A934BFC3F180020026B2
:10A78000002341F8102D02A802220196FFF7ECFEEB
:10A7900023781844C0B203062B7848BF80F08000AD
:10A7A0008342207002D0002004B070BD002301203D
:10A7B0002B70237004B070BD012004B070BD00BFC9
:10A7C00014820020988200201882002008B545F2EB
:10A7D0000820FFF7B9FE0620FDF7F8FE064B012220
:10A7E000C7201A70FDF7F2FE04480549054A002308
:10A7F00003700B70136008BD7A7C002098820020E3
:10A8000014820020A85F00202DE9F04182B00346A9
:10A81000060C050A032406208DF8073088461746E3
:10A820008DF805608DF806508DF80440FFF78CFE1A
:10A83000C0B100BF0D4C2368986802F0D5FD2368B5
:10A8400001A9586800222FF003FB2368424600212B
:10A8500058683B4602F0B8FF2368986802F0CAFDCA
:10A8600000BF384602B0BDE8F08100BF687C002020
:10A87000F0B5124B9D6885B00DB905B0F0BDED0A7D
:10A8800014D0002704AE7C196410E002102269463F
:10A89000FFF7BAFF0F2809DD6B4653F8042B01328E
:10A8A0000AD1B342F9D12546AF42ECDBFFF72CFFCA
:10A8B000034BED021D60E0E7671CF5E7D41D0020A7
:10A8C000A85F00202DE9F04F744B754C1B788DB0BC
:10A8D00005460BB101232377626A724BA3FB021377
:10A8E0009B0803EB8303511CD31A616240F0B980CB
:10A8F000DFF8E4B194F828109BF8007007F0010726
:10A90000B94200F09781002F40F0EE80D4F800802B
:10A91000654ED8F8003040469B6898472068FF2372
:10A9200088F80D300122036888F80C2011210222DA
:10A930008172C272D3F814805C4B1146C04796F8FE
:10A940005230002B40F0A38309230693082305937C
:10A950000623049305234FF00A084FF0070A0393D8
:10A960004FF00409032796F85330002B40F03F8343
:10A9700096F84A30DFF8648123B198F800309B07DD
:10A9800000F14C8496F85430CBB196F85B30B4F9B2
:10A990001620002B00F0C9830C23454909A8FEF7B7
:10A9A000F7FA384609AA4349FDF7D6FD049BCDF8CE
:10A9B00010A0DDF814A04F46DDF80C90039396F834
:10A9C0004B30002B40F0BB8296F85130DFF810A1DD
:10A9D000002B40F0EE8296F84C30002B40F0D282F3
:10A9E000354B9B79002B40F04782DFF8F89096F8C2
:10A9F0004F30002B40F0688296F85030CBB12F4B8F
:10AA00009B783BB3032B25D0012B00F06B840022F5
:10AA1000114609ABB2FBF1F2184692B228490793EE
:10AA2000FEF7B6FA7B1C3846079A2649DFB2FDF7D7
:10AA300093FD96F855306BB1204B9B7853B1032BA7
:10AA400008D009A9002024F09BFD09AA38461E4918
:10AA5000FDF782FD1D4A1E4E2A4400233260A36189
:10AA600069E020680368DB689847236863B193F95D
:10AA70000E30002B08DD174A138843F480439BB245
:10AA800013800DB0BDE8F08F124A138823F4804381
:10AA90009BB213800DB0BDE8F08F00BF387F00205F
:10AAA000B4240020CDCCCCCC9458002090110408C4
:10AAB00090100408AC110408D4A60020AA5A002063
:10AAC000341204081C120408281204080087930397
:10AAD00028660020B87F0020747D0020ECA60020AE
:10AAE000E87D0020B4A40020266863613068A3617B
:10AAF0004FF0FA714FF4C6028368E160304622617C
:10AB000098472068DFF86083DFF860A3DFF8609380
:10AB1000FF237373012203683273112107228172AC
:10AB2000C2725F69C04BC14E0C21B84705F5F422D3
:10AB300002F5907232609BF8001001F0010184F878
:10AB40002810BB4BDFF82CE3DB89BA4803EBC303C7
:10AB50009B008EFB03CEDB170788B4F90C00C3EB18
:10AB6000AE131BB29842B8BFA381B4F90E00BAF875
:10AB700000309842C8BFE381AF48D9F800304FF0A9
:10AB8000640E80FB03C0DB170EFB07F7C3EB6013FB
:10AB9000B4F910E01BB29E45B8BF2382B4F912305D
:10ABA000C7F38727BB42B4F91430C8BF6782002BB4
:10ABB000BCBF0023A38298F8003084F8297003F00A
:10ABC0000303032B2ED039B1E36AA068A169EB1A05
:10ABD00018440B44A060A361E5626AB1AA1A002A76
:10ABE00031DB27683B6838469B6898470121FF2284
:10ABF000002339737A7333609049914F914A3B68CF
:10AC0000AD09A1FB0515C5F3801515701D0100F1F7
:10AC10000581236853B393F90E20002A26DD002214
:10AC2000227723E7884BB4F916001B889842B8BFF7
:10AC3000E382C8E77D4EDFF830823268DFF82CA26D
:10AC4000DFF82C927DE7814AB2F9061040F2D66314
:10AC5000994203DCB2F902209A4201DD00233360FD
:10AC6000206803681B6A98472368D8E7784E94F8F1
:10AC7000293096F85A209A4240F22181754D2B686E
:10AC800043F00103744A1278002A40F0138123F440
:10AC9000C00323F0020398F80020900700F1078119
:10ACA00043F48043B6F85C802B6008F00F02012A61
:10ACB00000F0B282C0F0AC82022A00F04382002091
:10ACC000664A4FEA182802FB08F2002A00F06A825E
:10ACD000824200F2678243F02003B6F85E802B6068
:10ACE00008F00F02012A00F09182C0F06382022A6C
:10ACF00040F05E82A069594A4FEA182802FB08F228
:10AD0000002A00F04C82824200F2498243F0400364
:10AD1000D9F80820B6F856109142B6F85820D4BF9A
:10AD200043F0102323F01023002A00F03E8223F486
:10AD3000004326682B60336830469B6898470122A1
:10AD4000FF233273737313214548FEF78FFB0028EE
:10AD500086D1444D2B68990700F1AD820120FEF7A2
:10AD600093FB0020FEF790FB0220FEF78DFB0520F1
:10AD7000FEF78AFB0620FEF787FB0720FEF784FB21
:10AD80000920FEF781FB0A20FEF77EFB0B20FEF771
:10AD90007BFB0C20FEF778FB0820FEF775FB0F20ED
:10ADA000FEF772FB1020FEF76FFB1120FEF76CFB25
:10ADB0001220FEF769FB1320FEF766FB1420FEF756
:10ADC00063FB1520FEF760FB1620FEF75DFB1920E4
:10ADD000FEF75AFB1A20FEF757FB1B20FEF754FB29
:10ADE0001C20FEF751FB1D20FEF74EFB2020FEF736
:10ADF0004BFB2120FEF748FB2220FEF745FB2B688A
:10AE00009A0600F145823B681B017FF529AF23209C
:10AE1000FEF73AFB2420FEF737FB21E7FF2026F060
:10AE20005BF92062F5E600BF88110408286600205F
:10AE3000F0A60020887F00201F85EB51632D3E0582
:10AE4000D879002000000020D46C0020607F002012
:10AE50009458002020660020907F002000879303F4
:10AE600020840020E8A60020ECA60020E87D002039
:10AE7000B4A40020D34D621096F84D30002B40F062
:10AE8000E48196F84E30DFF87C93002B3FF4AFADB1
:10AE9000D9F80820C94909A80723FEF779F87B1CCF
:10AEA000384609AAC649DFB2FDF756FB9FE523F4F1
:10AEB0008043F7E643F4C00343F00203EBE6C14DE1
:10AEC0002B6823F00103DDE696F85B10B4F914E07B
:10AED000002940F039810EEB8E000EEBC00EBA4A0D
:10AEE000BA4B4FEACE004FEAE07E82FB00C2CEEBC7
:10AEF0002232002A83FB00C0B8BF5242DEEB601E44
:10AF000000F1DD8183FB0E314FEAEE73C3EB611379
:10AF10006420AF4900FB13E381FB0301DB17C3EBA4
:10AF2000A1030F21009109A8AA49FEF731F87B1C63
:10AF3000384609AAA849DFB2FDF70EFB5CE5B4F973
:10AF40000E30A34AA54982FB0302D817C0EBA20228
:10AF500002EB82004FF0060EA3EB40031BB212B2CD
:10AF6000CDF800E009A8FEF713F8384609AA9C4975
:10AF7000FDF7F2FA049BCDF810A04F46DDF80C90D7
:10AF8000039321E509AA1146B4F91200049224F0B2
:10AF9000F7FA049A10462FF0A7FB924B049A1B88ED
:10AFA000135291493846FDF7D7FA4F46DDF80C9019
:10AFB00016E5BAF800308D4A8849A2FB0302D20890
:10AFC00002EB82004FF0060EA3EB40039BB2CDF8DC
:10AFD00000E009A8FDF7DCFF384609AA8449FDF71F
:10AFE000BBFA049B4F46DDF80C900393F3E4B6F8EC
:10AFF0005E3003F00F02012AC3F30313079300F03E
:10B00000C980C0F06B81022A40F06481D4F818E056
:10B01000784B794AA3FB0E139B0C82FB03121A4454
:10B020005211C2EB0211A3EB81030799012940F0F1
:10B030002881DFF8D4C165487049ACFB0ECE4FEAD9
:10B040005E3EA0FB0EC040094FF0640C0CFB10EEFE
:10B05000CDF800E009A80790FDF79AFFB6F85E303A
:10B060006749079A03F00F03384651F82310FDF79C
:10B0700073FA049BCDF810A04F46DDF80C900393B3
:10B08000069BDDF814A0CDF81880059370E4B6F89F
:10B090005C3003F00F02012AC3F303187DD0C0F027
:10B0A0001681022A40F00F81A069524B524AA3FB3D
:10B0B00000139B0C82FB03121A445211C2EB0217BD
:10B0C000A3EB8703B8F1010F40F0D480DFF838E13B
:10B0D0003E4F4A49AEFB00E0400BA7FB00E77F096B
:10B0E0004FF0640E0EFB170009AF0090384607972B
:10B0F000FDF74EFFB6F85C304149079A03F00F03A5
:10B10000032051F82310FDF727FA0A230693092399
:10B1100005930723049306234FF00B084FF0080A0A
:10B1200003934FF0050904271DE402EB820302EBB1
:10B13000C3022649D30081FB0321DA17C2EB611257
:10B140000F232AE4A069BBE5204A4FEAEE7382FB95
:10B150000E02C3EB6212002AB8BF5242BEF1000FCA
:10B16000C0F2AF80DFF864C08CFB0E0CC3EB6C1335
:10B1700017484FF0640C0CFB13E380FB03E0DB1774
:10B18000C3EBA003002BB8BF5B4200290CBF0F210B
:10B190000C21C7E6D4F808E03AE7A06885E723F079
:10B1A0004003B5E523F0200397E543F40043C0E5F1
:10B1B0000020A0E501F06CFA2B689CE590100408D3
:10B1C000F411040820660020AD8BDB681F85EB516D
:10B1D00067666666001204080C1204085C10040816
:10B1E000BC110408D4110408D8110408CDCCCCCC6F
:10B1F000C811040883DE1B4389888888B0100408BE
:10B20000F0010408B4A400205917B7D1A06872E572
:10B2100001F03EFA2B6853E5A06851E509A9B4F99D
:10B220000C0024F0ADF9384609AA3949FDF794F924
:10B23000049BCDF810A04F46DDF80C900393069BBD
:10B24000DDF814A00593FFF79DBB09AA1146B4F9D8
:10B250001000039224F094F9039A10462FF044FA58
:10B260002C4B039A1B8813522B493846FDF774F96F
:10B270004F4606E609A9079108462849FDF788FECA
:10B2800038E709A9079108462449FDF781FEE5E65C
:10B290000E20FEF7F9F80D20FEF7F6F81820FEF75D
:10B2A000F3F81720FEF7F0F81F20FEF7EDF81E2048
:10B2B000FEF7EAF8A7E50320FEF7E6F84EE54FEAC9
:10B2C000EE7352424EE73B463A463846FAE601F004
:10B2D000DFF9EAE600231A469E46A6E601F0D8F911
:10B2E000864695E6FFF702F938B909AB18460C49CE
:10B2F0000793FDF74DFEFFF795BB0A4B9968890A46
:10B30000FFF7CCF86423820A03FB02F2FFF781BB4C
:10B31000A0110408E4110408E8110408A4100408AA
:10B320003C120408D41D00202DE9F043314A324E6E
:10B3300013683060042B89B004D0304C591C44F899
:10B34000230011602E4B2F4A1B78002103F00103CC
:10B350001160516086F82830012702F0B9F9A02366
:10B360000424FDB203E00134E4B21C2C13D0FF2B03
:10B37000F9DC306802688472C572611E0134D2F84B
:10B38000188003F10109C9B2DBB22A46E4B2C04712
:10B390001C2C4B46EBD10137052FE1D168461A4AE8
:10B3A0001A49FDF7F5FD6B4606221421306802F0BC
:10B3B0006BF9174B30680822072102F065F9154B2D
:10B3C000306809220B2102F05FF9134B30680A2222
:10B3D0000B2102F059F9306802F052F901F058F9E6
:10B3E0000E4B00F5741000F51060186009B0BDE850
:10B3F000F08300BF385B0020B42400203C5B0020B9
:10B40000747D002020660020441204084C120408B9
:10B4100050120408601204086C1204082866002008
:10B420002DE9F84FDFF8A890DFF8A880D9F80000E0
:10B43000DFF8A4A0234E012388F8003001F0D4FFE8
:10B4400005202EF0A1FD00202EF09EFD06202EF0FE
:10B450009BFD00202EF098FD9AF80040042044F057
:10B4600001042EF091FD20462EF08EFD33888BB125
:10B47000154D164F002415F804B007202EF084FD5A
:10B4800058462EF081FD2A5D33883A550134A4B226
:10B49000A342F0D807202EF077FDFF202EF074FD98
:10B4A0009AF8004004202EF06FFD20462EF06CFD2F
:10B4B000D9F8000001F09EFF002388F80030BDE8B5
:10B4C000F88F00BF081C0020186400204868002086
:10B4D0009474002030680020396800202DE9F04184
:10B4E000474E306801F080FF464B1B78012B78D027
:10B4F0005FD3022B0AD1DFF82C81082388F80030B3
:10B500000D254FF4C373404F3B8010E0DFF81481EA
:10B510003D4F98F8003003F04003002B14BF4FF468
:10B52000F0734FF4C3733B8014BF10250D25002426
:10B5300004F11000C0B22EF027FD013401202EF0DE
:10B5400023FDA3B2AB42F3D398F800402F4D002067
:10B550002EF01AFD20462EF017FD2D4B1C780220F0
:10B560002EF012FD20462EF00FFD2A4B1C780320F2
:10B570002EF00AFD20462EF007FD274B1C780420F4
:10B5800004432EF001FD20462EF0FEFC306801F051
:10B5900031FF3A882148002132F0FBFA6B7833B151
:10B5A0001F4B1B7833B300236B70BDE8F081BDE8FF
:10B5B000F081A0202EF0E8FC00202EF0E5FC00F049
:10B5C0000603022BDFF85C8007D000F0050001289D
:10B5D00003D1482388F8003008E0082388F80030B9
:10B5E0008EE7DFF84080482388F8003010254FF4BC
:10B5F000F07388E7FFF714FF00236B70BDE8F0815C
:10B6000094740020AC740020081C0020000000206E
:10B61000B3740020B474002039680020486800200A
:10B62000306800200A1C00200C4B984213D0A3F570
:10B63000806398420FD003F5804398420BD003F506
:10B640008063984207D003F58063984203D0044B8F
:10B65000186840087047024B1868704700040140A2
:10B66000C0750020F0B5774B774A87B019689142D2
:10B6700000AF00F0DB800023744A3B607B601368FE
:10B6800043F48033136003E03B68B3F5A04F09D067
:10B69000136803F400337B603B6801333B607B68D5
:10B6A000002BF1D0694B1B6813F4003318BF012342
:10B6B0007B607B68012B7BD0654D644B654AEA60FB
:10B6C0006549586F654A0860AA605E6B644C654ABC
:10B6D000654826F080065E635E6F46F080765E67A2
:10B6E000196B0C431C63596B5963996B9963196C03
:10B6F00041F05B5141F47B1141F41F6141F00F01B6
:10B700001964596C07F118040A4348F2FF715A642E
:10B7100044F8101D002621460123FB733E737E73FF
:10B72000BE732BF0DFFC21464FF6FF734F48BB6022
:10B730002BF0D8FC4FF6FF7321464D48BB602BF031
:10B74000D1FC21464B482BF0CDFC21464A482BF03A
:10B75000C9FC214649482BF0C5FC214648482BF03E
:10B76000C1FC214647482BF0BDFC214646482BF042
:10B77000B9FC20462BF0A8FE444B454C1B68BA6828
:10B7800044484549A4FB03439B09A0FB0202013B3B
:10B79000920CB3F1807F0A6007D2404AF020072163
:10B7A000536085F82300966011601C37BD46F0BDDC
:10B7B000264B3B4C1A6C3B4942F080521A6420687D
:10B7C0008A684D68C96840F4404020609868986075
:10B7D0009868120640F40040986042EA8512986822
:10B7E00042F48002490842F00802013942EA01426B
:10B7F00040F4A05098605A601A6842F080721A6053
:10B800001A689201FCD52849104A40F20570086078
:10B81000996821F003019960996841F002019960EB
:10B82000936803F00C03082BFAD145E700221A6055
:10B8300062B61E4B1B6883F308881D4B1B68984734
:10B84000FEE700BFFCFF0120EFBEADDE0038024086
:10B8500000ED00E00005FA051C950020000000083E
:10B86000FF916700335F07000000024000040240C0
:10B8700000080240000C0240001002400014024088
:10B8800000180240001C024000200240C075002049
:10B89000D34D621083DE1B43647C002010E000E087
:10B8A0000070004000000020003C02400000FF1F2C
:10B8B0000400FF1F08B5054B1B6803B19847044BF4
:10B8C000044A1A6072B6FCF78BFD00BF10600020BE
:10B8D000FCFF0120EFBEADDE08B5034B1B6803B1D2
:10B8E000984772B6FCF77CFD10600020084B10B53D
:10B8F00007281B68C8BF143818440C46007E01F0A6
:10B9000029FB20B12146BDE8104001F079BD10BDF2
:10B91000007C002038B50C4B07281B68CCBFA0F179
:10B920001404044623440546187E01F013FB50B16D
:10B9300001342722C47182712EF0F6FB28460021C3
:10B94000BDE83840D2E738BD007C002070B50F4C10
:10B950000F4DC0EBC00004EB8004286B2669304318
:10B96000286382B09209667BA1600025012101A8AD
:10B9700063618DF804608DF805208DF806508DF810
:10B98000071024F025FE02B070BD00BF141C00207B
:10B9900000380240074BC0EBC00030B403EB80001E
:10B9A000054C0569236B2B4323630176427630BC3B
:10B9B000704700BF141C0020003802402DE9F04FF2
:10B9C0005B4C54F8204083B0002C00F0AC80E66D56
:10B9D000002E00F0AA809046564A356922609946AA
:10B9E00004F2622204F162036361A2614FF4007306
:10B9F0007268A1600746E36023616265A246B5B143
:10BA00004D4B00205A68954203F11C0376D001305B
:10BA10001028F7D100207A1CD2B20C21FFF7BAFF10
:10BA2000636DB168326922630433A1632365F068F2
:10BA3000E8B1414B00215A68904203F11C035BD0EE
:10BA400001311029F7D100257A1CD2B20B212846EA
:10BA5000FFF7A0FF2346F27F38492846FFF776FF1D
:10BA6000636DB168F26862630433E163E36494F880
:10BA7000610001F06FFA054694F8600001F06AFA7F
:10BA80008346307F00284BD119F0080F38D118F0C9
:10BA9000020F09D045B10B227B1CAA71EB7128461D
:10BAA000727F222101F01CFB18F0010F15D1A36B4E
:10BAB0007BB996F82020B17F8DF8063001A8930954
:10BAC00001228DF805308DF804108DF8072024F040
:10BAD0007FFD504603B0BDE8F08FBBF1000FE6D00C
:10BAE00001370C238BF807708BF806305846727FAD
:10BAF000222101F0F5FADAE7CDB2A5E7C0B28AE774
:10BB00000137FFB215B10B23EF71AB7119F0100FB4
:10BB1000284614BF02211221727F01F0E1FAC6E724
:10BB20002EF0E4FAB0E7A246D3E7B246D1E700BF71
:10BB3000083E002018DD0308141C0020C1870008FF
:10BB40000348D0F8AC3113B100F5D27018477047F4
:10BB5000141C00200348D0F8903113B100F5C470D4
:10BB600018477047141C00200348D0F8743113B1F3
:10BB700000F5B67018477047141C00200348D0F831
:10BB8000583113B100F5A87018477047141C0020F5
:10BB90000348D0F83C3113B100F59A70184770474C
:10BBA000141C00200348D0F8203113B100F58C702C
:10BBB00018477047141C00200348D0F804310BB11B
:10BBC000FC301847704700BF141C00200348D0F811
:10BBD000E8300BB1E0301847704700BF141C00205C
:10BBE0000348D0F8CC300BB1C4301847704700BFC1
:10BBF000141C00200348D0F8B0300BB1A83018470F
:10BC0000704700BF141C00200348D0F894300BB1DB
:10BC10008C301847704700BF141C00200248836F07
:10BC20000BB1703018477047141C00200248C36DD8
:10BC30000BB1543018477047141C00200248036CA5
:10BC40000BB1383018477047141C00200248436A73
:10BC50000BB11C3018477047141C00200248836841
:10BC600003B11847704700BF141C00201549164B3C
:10BC700016484A6810B4CC681549B2FBF4F203FBCD
:10BC800002F30360D1F88820124B134C42F4700287
:10BC9000C1F888201A68002042F001021A609860FA
:10BCA0001A6822F0847222F480321A605C601A688A
:10BCB0004FF0006422F480221A60D8608C605DF836
:10BCC000044B70470000002040420F00C075002068
:10BCD00000ED00E00038024010300024044B4FF427
:10BCE000F07002210A225860D9609A60FFF7BEBF47
:10BCF00000000020436A8269D154436A0169426BA3
:10BD000001338B4228BF00234362002A2FD0EFF378
:10BD10001182502383F31288436B1968C9072CD40E
:10BD200070B45E686EB9456A816A8D4217D08469C5
:10BD30000C44DC600ED9691A59608562002180F8D4
:10BD40005810196841F00101D2B2196082F31188CC
:10BD500070BC70470469611A59608662EEE701237E
:10BD600080F85830D2B282F3118870BC7047426DAF
:10BD7000D36843F08003D3607047D2B282F3118856
:10BD8000704700BF026B10B462B1836CC268446933
:10BD9000D11A013B615C5DF8044B08BF1346836414
:10BDA000C8B27047016A4369C4685B5C0131A14253
:10BDB00028BF114601625DF8044BD8B2704700BF3E
:10BDC000436B13B190F858007047836A406A181AA1
:10BDD000B0FA80F040097047416A836A99420AD3F9
:10BDE000CB1A416B026961B14968501E0B44834212
:10BDF0000AD2C01A704702691144CB1A416B00295C
:10BE0000F2D1501EC01A704700207047036B43B137
:10BE1000826C5B6893422FBF981AC0689B1AC01847
:10BE20007047C269036A9A422FBFD01AC06880184F
:10BE3000C01A70470A4B30B503F1140493F900207F
:10BE40005D78072AC8BF143A811804330D7313F8BC
:10BE5000025C855413F8012C0A76A342EED130BD62
:10BE600040DD030803682DE9F041DF691FB13B465F
:10BE7000BDE8F0411847002A164611DD04460D467C
:10BE80000E4400E023689B68204698470028F9D0BC
:10BE9000236815F8011B1B6820469847AE42F1D174
:10BEA000BDE8F08100232422027043708370C370C8
:10BEB000704710B5074B03F10C0193F900205C7833
:10BEC000845402449C78D470DC78947104338B429F
:10BED000F3D110BD54DD030830B4846814B1236875
:10BEE000A5885D83436840F2E93001E0002833D043
:10BEF0001D89013815F0020F80B2F7D089B29981FF
:10BF000040F2E93101E0002950D01889013910F0E0
:10BF1000010F89B2F7D0998940F2E93101E0002997
:10BF20002FD01889013910F0020F89B2F7D092B2E0
:10BF30009A8140F2E93201E0002A4BD01989013A96
:10BF400011F0010F92B2F7D09B8914B12368A28837
:10BF50001A83012030BC70472C498B4208D0A1F5D0
:10BF600078418B424CD001F580618B42D4D10220C4
:10BF7000274901EB00104189013189B24181418992
:10BF8000CAE7224A934208D0A2F57842934235D0BC
:10BF900002F580629342D8D102211D4B03EB0111BF
:10BFA0004B8901339BB24B814B89CEE717488342C3
:10BFB00007D018498B4227D001F580618B42ABD165
:10BFC0000221134800EB01114889013080B24881F9
:10BFD0004989A1E70D498B4207D00E4A934211D0FF
:10BFE00002F580629342B0D10222094B03EB0212A8
:10BFF000538901339BB253815389A6E70121CCE7D2
:10C000000120B5E70122F0E70121DAE70030014025
:10C01000F8A700200038004030B50446406D61713B
:10C020008389A26823F400531B041B0C838185B011
:10C03000A379009213F0040230D04FF4805213F031
:10C040000203ADF8042056D1ADF806304FF48063FA
:10C050000022ADF8083011F00103ADF80C2028D112
:10C06000ADF80A3008238D07694648BFADF80A309D
:10C0700024F0E6FAA279636DD10724D412F0080FF8
:10C080009A8A1BD122F008021204120C9A829A8911
:10C0900092B242F400529A8105B030BD13F002030F
:10C0A000ADF8042024D04FF400551346ADF80650E7
:10C0B000CEE70423ADF80A300C23D4E792B242F065
:10C0C00008029A82E3E70D498B420FD0A1F548415F
:10C0D0008B4209D00A498B42D0D105200121FFF7BC
:10C0E00005FCA279636DC9E70220F7E70020F5E7B8
:10C0F000ADF80630ACE74FF40053A5E7001001405F
:10C100000014014010B50446406DA160838923F4FA
:10C1100000531B041B0C8381A37984B013F0040229
:10C12000009135D04FF4805213F00203ADF8042093
:10C1300056D1ADF806304FF480636279ADF808301F
:10C14000D1074FF00003ADF80A30ADF80C3045BF11
:10C150000423ADF80A3008230C236946920748BF30
:10C16000ADF80A3024F06CFAA279636DD1071FD4C0
:10C1700012F0080F9A8A16D122F008021204120C4B
:10C180009A829A8992B242F400529A8104B010BD08
:10C1900013F00203ADF804201FD04FF400511346F2
:10C1A000ADF80610C9E792B242F008029A82E8E7B9
:10C1B0000D498B420FD0A1F548418B4209D00B4964
:10C1C0008B42D5D105200121FFF790FBA279636D49
:10C1D000CEE70220F7E70020F5E7ADF80630ACE740
:10C1E0004FF40053A5E700BF0010014000140140C8
:10C1F0002DE98048013085B0C3B203938A4D8B4F3F
:10C200008B4C8C4E0A230293DFF82C9223F008F813
:10C210004FF4FA7A4FF0100C4FF47A70D9F80430DA
:10C22000C3F30803002B40F0C180EFF31183002B10
:10C2300040F0BC802968A26800BF2B689942F9D100
:10C24000D7F800E000FB0EF39B1AB3FBFEF300FBF4
:10C2500001314FF0010E0191D9F80430C3F3080306
:10C26000002B40F08780EFF31183002B40F0828099
:10C270002B68A16800BF2A689342F9D1D7F800B0B3
:10C2800000FB0BF2521AB2FBFBF200FB0323019AF4
:10C290009B1AB3F57A7FDFD3BAF1010ABED1039BB3
:10C2A000002B40F0BD804FF47A7ADFF88C91504635
:10C2B0004FF0100CD9F80430C3F30803002B40F002
:10C2C0009280EFF31183002B40F08D802968A268E3
:10C2D00000BF2B689942F9D1D7F800E000FB0EF3BC
:10C2E0009B1AB3FBFEF300FB01314FF0010E0191ED
:10C2F000D9F80430C3F3080303BBEFF31183EBB9A0
:10C300002B68A16800BF2A689342F9D1D7F800B022
:10C3100000FB0BF2521AB2FBFBF200FB0323019A63
:10C320009B1AB3F57A7FE3D3BAF1010AC2D1029B1B
:10C33000013B02937FF468AFFFF7BCFAEFF311887B
:10C340008CF31288A1682368DB0344BFC6F800E0C1
:10C35000A1682B6832685FFA88F888F31188D7F8EB
:10C3600000801A4400FB08F35B1AB3FBF8F300FBF0
:10C370000233D4E7EFF311888CF31288A1682368A5
:10C38000DB0344BFC6F800E0A1682B6832685FFA9F
:10C3900088F888F31188D7F800801A4400FB08F366
:10C3A0005B1AB3FBF8F300FB023370E7EFF3118283
:10C3B0008CF31288D4F808E02368D90303D501234D
:10C3C0003360D4F808E02B683168D2B282F3118868
:10C3D0003A68194400FB02F3A3EB0E03B3FBF2F33C
:10C3E00000FB013135E7EFF311828CF31288D4F8AA
:10C3F00008E02368D90303D501233360D4F808E0AB
:10C400002B683168D2B282F311883A68194400FB74
:10C4100002F3A3EB0E03B3FBF2F300FB013164E77D
:10C42000184622F06BFD3EE7607C0020647C002013
:10C4300010E000E05C7C002000ED00E02DE9F04F12
:10C44000013085B0C3B203930B4602918B4C8C4EE6
:10C45000002B00F099808B4D8B4FDFF8309222F04B
:10C46000DFFE4FF4FA7A4FF0100C4FF47A70D9F8DF
:10C470000430C3F30803002B40F0DE80EFF3118398
:10C48000002B40F0D9802968A26800BF2B68994230
:10C49000F9D1D7F800E000FB0EF39B1AB3FBFEF3D3
:10C4A00000FB01314FF0010E0191D9F80430C3F3C4
:10C4B0000803002B40F08780EFF31183002B40F03E
:10C4C00082802B68A16800BF2A689342F9D1D7F80F
:10C4D00000B000FB0BF2521AB2FBFBF200FB03238D
:10C4E000019A9B1AB3F57A7FDFD3BAF1010ABED164
:10C4F000039B002B40F0BD804FF47A7ADFF88C91DB
:10C5000050464FF0100CD9F80430C3F30803002B49
:10C5100075D1EFF31183002B71D12968A26800BF98
:10C520002B689942F9D1D7F800E000FB0EF39B1A73
:10C53000B3FBFEF300FB01314FF0010E0191D9F87E
:10C540000430C3F3080313BBEFF31183FBB92B686B
:10C55000A16800BF2A689342F9D1D7F800B000FB68
:10C560000BF2521AB2FBFBF200FB0323019A9B1A57
:10C57000B3F57A7FE3D3BAF1010AC4D1029B013B40
:10C580000293002B7FF467AF05B0BDE8F08FEFF3A7
:10C5900011888CF31288A1682368DB0344BFC6F8B6
:10C5A00000E0A1682B6832685FFA88F888F3118888
:10C5B000D7F800801A4400FB08F35B1AB3FBF8F3CA
:10C5C00000FB0233D2E7EFF311888CF31288A168E5
:10C5D0002368DB0344BFC6F800E0A1682B6832681B
:10C5E0005FFA88F888F31188D7F800801A4400FBB6
:10C5F00008F35B1AB3FBF8F300FB023370E7EFF3C9
:10C6000011828CF31288D4F808E02368D90303D58B
:10C6100001233360D4F808E02B683168D2B282F38A
:10C6200011883A68194400FB02F3A3EB0E03B3FB35
:10C63000F2F300FB01317FE7EFF311828CF31288F4
:10C64000D4F808E02368D90303D501233360D4F874
:10C6500008E02B683168D2B282F311883A68194435
:10C6600000FB02F3A3EB0E03B3FBF2F300FB01317B
:10C6700018E7184622F042FC3EE700BF10E000E059
:10C680005C7C0020607C0020647C002000ED00E0E9
:10C69000204B5B68C3F3080330B4BBB9EFF31183DD
:10C6A000A3B91D4B1D4C1868A16800BF1A689042C1
:10C6B000F9D11B4B1C684FF47A7202FB04F3591A30
:10C6C000B1FBF4F130BC02FB00107047EFF31182B4
:10C6D000102383F3128811498C680B6813F4803F90
:10C6E000104B02D0012018608C680B49D2B20D6843
:10C6F000186882F311880A4B19684FF47A7228443B
:10C7000002FB01F31B1B30BCB3FBF1F302FB003057
:10C71000704700BF00ED00E0607C002010E000E00A
:10C72000647C00205C7C00202DE9F84F8046FFF7F8
:10C73000AFFF254E2549DFF8A0E0254A254D844668
:10C7400010274FF47A740120DEF80430C3F3080395
:10C75000D3B9EFF31183BBB90B68D2F808A000BFBF
:10C76000D1F800904B45F7D1D6F800B004FB0BF997
:10C77000A9EB0A09B9FBFBF904FB0393A3EB0C0338
:10C780004345E1D3BDE8F88FEFF3118A87F31288B0
:10C79000D2F808B01368DB0344BF2860D2F808B0B1
:10C7A0000B68D5F800905FFA8AFA8AF31188D6F8F8
:10C7B00000A0994404FB0AF3A3EB0B03B3FBFAF3C9
:10C7C00004FB0933DAE700BF647C0020607C0020B2
:10C7D00010E000E05C7C002000ED00E02DE9F04F6F
:10C7E000DFF830C1474A4849484E494D8046102736
:10C7F00018F1FF38C0F08480DCF80430C3F308037C
:10C80000002B5CD1EFF31183002B58D10B68946897
:10C8100000BF08688342F9D1D6F800904FF47A70CF
:10C8200000FB09FEAEEB040EBEFBF9FE00FB03EEBF
:10C83000DCF80430C3F308034FF47A740120FBB929
:10C84000EFF31183E3B90B68D2F808A000BFD1F869
:10C8500000904B45F7D1D6F800B004FB0BF9A9EBDB
:10C860000A09B9FBFBF904FB0393A3EB0E03B3F531
:10C870007A7FBDD2DCF80430C3F30803002BDFD08D
:10C88000EFF3118A87F31288D2F808B01368DB033C
:10C8900044BF2860D2F808B00B68D5F800905FFA62
:10C8A0008AFA8AF31188D6F800A0994404FB0AF3A7
:10C8B000A3EB0B03B3FBFAF304FB0933D5E7EFF368
:10C8C000118487F31288D2F808901368D80303D52F
:10C8D00001232B60D2F808900B682868E4B284F337
:10C8E0001188D6F800A04FF47A7400EB030E04FB15
:10C8F0000AF3A3EB0903B3FBFAF304FB0E3E97E73D
:10C90000BDE8F08F10E000E0607C0020647C002037
:10C910005C7C002000ED00E030B4EFF311831022C6
:10C9200082F312880649074C0A680748013200253D
:10C930000A602560DBB2026883F3118830BC70475F
:10C94000607C00205C7C002010E000E038B5254BC6
:10C950005C69236B73B1636D626BCAB1998A1A8883
:10C96000C90592B201D5D20700D438BD4FF6F7728F
:10C970001A8038BD636D99891A88890692B2EBD501
:10C980009206E9D5E26ACAB1988880B29047E2E798
:10C9900099891A880D0692B2E0D51006DED5A26AF2
:10C9A000616A8A4219D0A1692569885C9880013240
:10C9B000B2FBF5F105FB1122A262CFE79B88E26989
:10C9C0006169DBB28B54E269E068636D0132B2FBEE
:10C9D000F0F100FB1122E261BEE7DA6822F080028A
:10C9E000DA60BBE7083E002038B5254B9C68236B16
:10C9F00073B1636D626BCAB1998A1A88C90592B224
:10CA000001D5D20700D438BD4FF6F7721A8038BD71
:10CA1000636D99891A88890692B2EBD59206E9D599
:10CA2000E26ACAB1988880B29047E2E799891A8889
:10CA30000D0692B2E0D51006DED5A26A616A8A427E
:10CA400019D0A1692569885C98800132B2FBF5F1A3
:10CA500005FB1122A262CFE79B88E2696169DBB224
:10CA60008B54E269E068636D0132B2FBF0F100FBC8
:10CA70001122E261BEE7DA6822F08002DA60BBE7E9
:10CA8000083E002038B5254B1C68236B73B1636DDD
:10CA9000626BCAB1998A1A88C90592B201D5D207C8
:10CAA00000D438BD4FF6F7721A8038BD636D99898E
:10CAB0001A88890692B2EBD59206E9D5E26ACAB124
:10CAC000988880B29047E2E799891A880D0692B259
:10CAD000E0D51006DED5A26A616A8A4219D0A16942
:10CAE0002569885C98800132B2FBF5F105FB1122C3
:10CAF000A262CFE79B88E2696169DBB28B54E2698D
:10CB0000E068636D0132B2FBF0F100FB1122E261DB
:10CB1000BEE7DA6822F08002DA60BBE7083E002058
:10CB200070B4EFF31186502383F31288436B1A68B5
:10CB3000D20720D45D686DB9446A826A944217D0E6
:10CB400081691144D9600ED9A21A5A608462002208
:10CB500080F858201A6842F00102F1B21A6081F39D
:10CB6000118870BC704701698A1A5A608562EEE7C5
:10CB7000012380F85830F3B283F3118870BC7047FA
:10CB800003685B6A03B11847704700BF03681B6AFC
:10CB900003B11847704700BF03682DE9F041DF6912
:10CBA0001FB13B46BDE8F0411847002A164611DD8B
:10CBB00004460D460E4400E023689B6820469847D3
:10CBC0000028F9D0236815F8011B1B6820469847F8
:10CBD000AE42F1D1BDE8F08103689B69184700BF00
:10CBE00003685B69184700BF03681B69184700BFEB
:10CBF0000368DB68184700BF03689B68184700BFDD
:10CC000003685B68184700BF03681B68184700BFCC
:10CC100038B50C46097849B1054601342B682846D9
:10CC20001B68984714F8011B0029F7D138BD00BFD5
:10CC3000064B53F820302BB11A689B8851690B4280
:10CC400001D1138370475383704700BF2C7C0020B1
:10CC500003682DE9F04F03F13F4404F57E04604E74
:10CC6000A40A0125345D04F01F066409032C05FAAB
:10CC700006F500F0AF80042C00F0A780022C54D001
:10CC80008588B5FA85F0C0F11F0080B2C40803EBB7
:10CC9000840400F00700266A80000F27874026EAF8
:10CCA00007062662276A01F0030602FA00F0721EE8
:10CCB0003843012AC1F3810CC1F300182062C1F38B
:10CCC000411137D90024224601274FF0030E03E01B
:10CCD000102A04F1020426D007FA02F0A84302F158
:10CCE0000102F5D1D3F800C00EFA04F0C04300EA07
:10CCF0000C0CC3F800C0D3F8008006FA04FC4CEA20
:10CD0000080CC3F800C0D3F80CC000EA0C00D860CF
:10CD1000D3F80CC001FA04F040EA0C00102AD860E5
:10CD200004F10204D8D1BDE8F08F2E4C666C354377
:10CD30006564A5E7002002464FF0010E4FF003099D
:10CD400004E00132102A00F102003CD00EFA02F792
:10CD500037EA0504F5D1D3F800A009FA00F4E4435A
:10CD60000AEA040AC3F800A0D3F800B006FA00FAF1
:10CD70004AEA0B0AC3F800A0D3F808A004EA0A0A9A
:10CD8000C3F808A0D3F808B00CFA00FA4AEA0B0A74
:10CD9000C3F808A0D3F804A02AEA07075F60D3F815
:10CDA00004A008FA02F747EA0A075F60DF683C4020
:10CDB000DC60DF6801FA00F401323C43102ADC60D9
:10CDC00000F10200C2D1BDE8F08F064C266B35435E
:10CDD000256355E7034C266C3543256450E700BFB7
:10CDE000D40F040800380240026802F13F4303F503
:10CDF0007E032DE9F04F9B0A544DEB5C03F01F05B9
:10CE00005B090124032B04FA05F400F09980042B3C
:10CE100000F09180022B3ED001F00306731E012B1F
:10CE2000C1F3810CC1F300188588C1F3411137D9D2
:10CE30000024234601274FF0030E03E0102B04F1DA
:10CE4000020426D007FA03F0A84303F10103F5D149
:10CE5000D2F800C00EFA04F0C04300EA0C0CC2F88D
:10CE600000C0D2F8008006FA04FC4CEA080CC2F8B4
:10CE700000C0D2F80CC000EA0C00D060D2F80CC0A0
:10CE800001FA04F040EA0C00102BD06004F1020417
:10CE9000D8D1BDE8F08F2E4B5D6C2C435C64BBE7B2
:10CEA000002003464FF0010E4FF0030904E0013368
:10CEB000102B00F102003CD00EFA03F737EA05040C
:10CEC000F5D1D2F800A009FA00F4E4430AEA040A12
:10CED000C2F800A0D2F800B006FA00FA4AEA0B0A3B
:10CEE000C2F800A0D2F808A004EA0A0AC2F808A012
:10CEF000D2F808B00CFA00FA4AEA0B0AC2F808A005
:10CF0000D2F804A02AEA07075760D2F804A008FA6A
:10CF100003F747EA0A075760D7683C40D460D768F0
:10CF200001FA00F401333C43102BD46000F10200FD
:10CF3000C2D1BDE8F08F064B1D6B2C431C636BE721
:10CF4000034B1D6C2C431C6466E700BFD40F040820
:10CF50000038024010B50409013C032C17D80D4BD2
:10CF600033F8142000F00F0042FA00F313F001032D
:10CF70000DD0012303FA00F0013810402EF07EF8A6
:10CF8000054A064B125D104403EBC00010BD0020A3
:10CF900010BD00BF00100408FC0F040810B00020F2
:10CFA0002DE9F04F4A484B494B4B4C4C4FF0010A8E
:10CFB0004FF002094FF004084FF0080C4FF0100E2C
:10CFC00020274026802530F8022B12F0010F03D0D5
:10CFD0001960A3F804A0083312F0020F03D01960FF
:10CFE000A3F80490083312F0040F03D01960A3F8DB
:10CFF0000480083312F0080F03D01960A3F804C0AE
:10D00000083312F0100F03D01960A3F804E00833BE
:10D0100012F0200F02D019609F80083312F0400FE9
:10D0200002D019609E80083312F0800F02D0196080
:10D030009D80083312F4807F05D04FF4807B196007
:10D04000A3F804B0083312F4007F05D04FF4007B3E
:10D050001960A3F804B0083312F4806F05D04FF4C0
:10D06000806B1960A3F804B0083312F4006F05D088
:10D070004FF4006B1960A3F804B0083312F4805F1A
:10D0800005D04FF4805B1960A3F804B0083312F4A4
:10D09000005F05D04FF4005B1960A3F804B00833BB
:10D0A00012F4804F05D04FF4804B1960A3F804B000
:10D0B0000833D20B04D04FF4004219609A80083331
:10D0C00001F58061A1427FF47EAFBDE8F08F00BF23
:10D0D000001004080000024010B0002000100240C0
:10D0E00000286AD003682DE9F04F03F13F4404F5AE
:10D0F0007E045F4EA40A0125345D04F01F06640916
:10D10000032C05FA06F559D0042C00F0AC80022C53
:10D1100059D08588B5FA85F0C0F11F0080B2C408E7
:10D1200003EB840400F00700266A80000F27874085
:10D1300026EA07062662276A01F003068240701E6F
:10D140003A430128C1F3810CC1F300182262C1F3F4
:10D1500041113DD90024224601274FF0030E03E080
:10D16000102A04F1020426D007FA02F0A84302F1C3
:10D170000102F5D1D3F800C00EFA04F0C04300EA72
:10D180000C0CC3F800C0D3F8008006FA04FC4CEA8B
:10D19000080CC3F800C0D3F80CC000EA0C00D8603B
:10D1A000D3F80CC001FA04F040EA0C00102AD86051
:10D1B00004F10204D8D1BDE8F08F70472D4C266CE5
:10D1C00035432564A5E72B4C666C35436564A0E7C1
:10D1D000002002464FF0010E4FF0030904E0013237
:10D1E000102A00F102003CD00EFA02F737EA0504DB
:10D1F000F5D1D3F800A009FA00F4E4430AEA040ADE
:10D20000C3F800A0D3F800B006FA00FA4AEA0B0A05
:10D21000C3F800A0D3F808A004EA0A0AC3F808A0DB
:10D22000D3F808B00CFA00FA4AEA0B0AC3F808A0CF
:10D23000D3F804A02AEA07075F60D3F804A008FA2D
:10D2400002F747EA0A075F60DF683C40DC60DF689E
:10D2500001FA00F401323C43102ADC6000F10200C4
:10D26000C2D1BDE8F08F034C266B3543256350E7F0
:10D27000D40F040800380240002855D0026802F19B
:10D280003F4303F57E032DE9F04F9B0A544DEB5CC1
:10D2900003F01F055B090124032B04FA05F444D0B5
:10D2A000042B00F09780022B44D001F00306731E7C
:10D2B000012BC1F3810CC1F300188588C1F3411122
:10D2C0003DD90024234601274FF0030E03E0102B25
:10D2D00004F1020426D007FA03F0A84303F1010386
:10D2E000F5D1D2F800C00EFA04F0C04300EA0C0CED
:10D2F000C2F800C0D2F8008006FA04FC4CEA080C20
:10D30000C2F800C0D2F80CC000EA0C00D060D2F81D
:10D310000CC001FA04F040EA0C00102BD06004F1BC
:10D320000204D8D1BDE8F08F70472E4B1D6C2C4302
:10D330001C64BAE72B4B5D6C2C435C64B5E70020A2
:10D3400003464FF0010E4FF0030904E00133102BA8
:10D3500000F102003CD00EFA03F737EA0504F5D1DC
:10D36000D2F800A009FA00F4E4430AEA040AC2F879
:10D3700000A0D2F800B006FA00FA4AEA0B0AC2F896
:10D3800000A0D2F808A004EA0A0AC2F808A0D2F85D
:10D3900008B00CFA00FA4AEA0B0AC2F808A0D2F860
:10D3A00004A02AEA07075760D2F804A008FA03F796
:10D3B00047EA0A075760D7683C40D460D76801FA4B
:10D3C00000F401333C43102BD46000F10200C2D1C1
:10D3D000BDE8F08F034B1D6B2C431C6365E700BF5A
:10D3E000D40F04080038024010B1036882885A83C1
:10D3F000704700BF10B1036882881A83704700BF6E
:10D4000018B10368828809B95A8370471A83704734
:10D410000E4B1B8801463BB90D4B0E4A1B7810681A
:10D420000BB981F00101EBE70B4B5A691AB118B93E
:10D430001A68106058747047084A18681188084ABA
:10D4400092FBF1F20121026059747047387C002090
:10D450003A7C00203C7C0020407C0020587C00204E
:10D4600020A1070010B40A4B0A4A1C78012383400C
:10D47000234052F8200029B9B3FA83F149095DF835
:10D48000044BBDE7191C18BF01215DF8044BB7E739
:10D49000287C00202C7C002030B1036882881B6926
:10D4A0001A4214BF01200020704700BF2DE9F0414F
:10D4B0000B4E346873691C400FD0DFF828800127B9
:10D4C000B4FA84F3C3F11F0307FA03F558F82300F5
:10D4D00003689847AC437561F2D1BDE8F08100BFA5
:10D4E000003C014098B100202DE9F0410B4E34681A
:10D4F00073691C400FD0DFF828800127B4FA84F349
:10D50000C3F11F0307FA03F558F82300036898478F
:10D51000AC437561F2D1BDE8F08100BF003C014031
:10D5200098B100202DE9F0410B4E346873691C401E
:10D530000FD0DFF828800127B4FA84F3C3F11F036A
:10D5400007FA03F558F8230003689847AC43756160
:10D55000F2D1BDE8F08100BF003C014098B100204D
:10D560002DE9F0410B4E346873691C400FD0DFF891
:10D5700028800127B4FA84F3C3F11F0307FA03F5E7
:10D5800058F8230003689847AC437561F2D1BDE8B1
:10D59000F08100BF003C014098B100202DE9F0412E
:10D5A0000B4E346873691C400FD0DFF828800127C8
:10D5B000B4FA84F3C3F11F0307FA03F558F8230004
:10D5C00003689847AC437561F2D1BDE8F08100BFB4
:10D5D000003C014098B100202DE9F0410B4E346829
:10D5E00073691C400FD0DFF828800127B4FA84F358
:10D5F000C3F11F0307FA03F558F82300036898479F
:10D60000AC437561F2D1BDE8F08100BF003C014040
:10D6100098B100202DE9F0410B4E346873691C402D
:10D620000FD0DFF828800127B4FA84F3C3F11F0379
:10D6300007FA03F558F8230003689847AC4375616F
:10D64000F2D1BDE8F08100BF003C014098B100205C
:10D65000084A094808B5536C43F4804353640021D9
:10D66000402230F096FA054B4FF0FF321A60C3F8B3
:10D67000032008BD0038024098B10020D8B1002036
:10D6800003685B6A184700BF2DE9F041044618465D
:10D690000D46164698462DF027F82768E67228446E
:10D6A000A07229467D69434632462046AC46BDE815
:10D6B000F0416047036810B504461B68984723682B
:10D6C00020469B689847A37B0133A37310BD00BF1E
:10D6D00010B5036804469B689847FF2301226373D3
:10D6E000227310BD08B5FFF735FC38B12C228271CA
:10D6F0000022C2712021BDE80840BDE508BD00BF81
:10D7000040F2E93300E0A3B10289013B12F0020FBD
:10D710009BB2F8D089B2818140F2E93300E043B195
:10D720000289013B12F0010F9BB2F8D08089C0B290
:10D7300070470C4A904209D00B4B984210D003F529
:10D740008063984201D0FF2070470223074A02EB12
:10D7500003135A89013292B25A815889C0B2704774
:10D760000123F3E70030014000380040F8A7002013
:10D77000144B984224D003F58063984220D002884D
:10D7800022F040021204120C0280028822F03803B8
:10D790001B041B0C59B141F48071002991FAA1F2CC
:10D7A000B2FA82F108BF4FF0FF310139C9000B43D3
:10D7B0009BB2038003889BB243F040030380704711
:10D7C0004908DCE700380040F0B484894FF6FF7662
:10D7D0004FF47A7463B300293CD00F78013101E033
:10D7E000B4421AD00589013C15F00205A4B2F7D065
:10D7F000BCB284814FF47A7402E0BCB2B4420CD063
:10D80000058915F0010504F1FF37F6D08589ADB221
:10D810000AB115700132013BDCE7104B98420BD086
:10D82000A3F57843984217D003F58063984202D05D
:10D830000120F0BC70470225094B03EB05156B89ED
:10D8400001339BB26B81688980B2003018BF012020
:10D85000F0BC7047FF27C5E70125EDE70030014028
:10D86000F8A7002070B50546806810B1046880886C
:10D87000608341F08001686840F2E93400E0E4B17F
:10D880000689013C16F0020FA4B2F8D089B281815A
:10D8900040F2E93100E029B30489013914F0010FA5
:10D8A00089B2F8D081890021FFF78EFFAB6813B1F0
:10D8B0001A689B881383012070BD1649884208D0DE
:10D8C000A1F57841884221D001F580618842EAD1F2
:10D8D0000224114901EB04146189013189B261818B
:10D8E0006189E0E70B4CA04207D00C4988420FD079
:10D8F00001F580618842D6D10221074C04EB011169
:10D900004C890134A4B24C814989CCE70124E0E779
:10D910000121F2E700300140F8A700200038004064
:10D92000F8B5654C0601A7190546387A2CF0DEFBE0
:10D930003B7A03F01F015B090122032B02FA01F27B
:10D940006DD0042B66D0022B5CD0A3190135187959
:10D95000FFF700FBEDB2074610B11223C5718371CA
:10D96000A3195879FFF7F6FA10B11323C571837123
:10D97000A3199879FFF7EEFA10B11423C5718371DA
:10D98000A5190A21EA793846FFF7AAFB6879FFF75B
:10D99000E1FAEA790A21FFF7A3FBA879FFF7DAFA9F
:10D9A000EA790A21FFF79CFBA359444A934247D0E6
:10D9B000434A934250D0434A934259D0424A9342F9
:10D9C00062D0424A93426BD0414A93422CD03444B5
:10D9D000227BE2B901200222198801F4415141F46D
:10D9E00045710A4302431A809A8B22F400621204A2
:10D9F000120C07219A8319821A8892B242F04002CF
:10DA00001A80F8BD334B596A0A435A629DE70020D9
:10DA10000246E1E72F4B19690A431A6195E72D4B3E
:10DA2000196A0A431A6290E702F564424FF4001043
:10DA3000536A43F40013536229F088FCA359C6E7E4
:10DA400002F584324FF48050536A43F4805353629A
:10DA500029F07CFCA359BAE702F500324FF480406C
:10DA6000136A43F48043136229F078FCA359AEE7AC
:10DA700002F5FE324FF40040136A43F40043136290
:10DA800029F06CFCA359A2E702F582324FF4005052
:10DA9000536A43F40053536229F058FCA35996E7A4
:10DAA00002F568424FF48010536A43F480135362C6
:10DAB00029F04CFCA3598AE7F8A700200030014068
:10DAC00000380040003C004000340140005001405C
:10DAD0000054014000380240427A02B9704710B544
:10DAE00004460368406804F10A0198470023637202
:10DAF00010BD00BF437A5A1C0344D2B242729972DD
:10DB0000037A934200D802B9704710B504460368FF
:10DB1000406804F10A0198470023637210BD00BFFA
:10DB2000302828D0312828D0322828D0332828D0AF
:10DB3000342828D0352828D0202828D0212828D0BB
:10DB4000102828D0112828D0122828D0132828D00F
:10DB5000142828D0152828D0162805D0172808BF43
:10DB60000F2202D0002070470E22114B03EB42031C
:10DB700093F8210070470022F7E70122F5E702221F
:10DB8000F3E70322F1E70422EFE70522EDE706229F
:10DB9000EBE70722E9E70822E7E70922E5E70A229F
:10DBA000E3E70B22E1E70C22DFE70D22DDE700BF10
:10DBB00040DD0308F8B50468C4F30D0405460E46BD
:10DBC00004B32F6829F0C8FC092840F08780454C31
:10DBD000236923F440732361236943F400732361B1
:10DBE000236943F0010323613E6029F0B5FC2369FA
:10DBF000092823F00103236170D12B6804332B60C3
:10DC00000020F8BD384B394A93422AD902F58042A8
:10DC1000934225D902F58042934229D902F58042E8
:10DC2000934227D902F58032934225D902F500327A
:10DC3000934223D902F50032934221D902F50032F2
:10DC400093421FD902F5003293421DD902F580227A
:10DC500093421BD9B3F1016F1AD30520FEF7C8FA1E
:10DC6000082429F079FC092814D04FF0FF30F8BDC2
:10DC70001024F6E71824F4E72024F2E72824F0E73C
:10DC80003024EEE73824ECE74024EAE74824E8E7CC
:10DC90005824E6E7134F3B6923F440733B613B692B
:10DCA00043F400733B613B6923F0F8033B613B693C
:10DCB00043F002031C433C613B6943F480333B6106
:10DCC00029F04AFC3B6923F002033B613B690928C8
:10DCD00023F0F8033B613FF474AFC6E76FF0010037
:10DCE000F8BD00BF003C024000400008FF3F0008B4
:10DCF000F8B504460D468E180027B54201D12069BB
:10DD0000F8BDE368591CE160234415F8012B1A7231
:10DD10000429F2D1206918B9A1682046FFF74AFF0B
:10DD20002061E760E9E770B5448806460D46C4F314
:10DD30000B042246002128462FF02BFF33690A4AA4
:10DD4000934209D3094A934206D2224628461946ED
:10DD5000BDE870402DF006BC23B121462846BDE841
:10DD60007040184770BD00BF100600081207000879
:10DD7000064B07498B4202D30023184670471A8886
:10DD8000C2F30B029042F8D01433F3E78801000885
:10DD900010060008024A136823EA0000106070476A
:10DDA000C05A00202DE9F04F9DB0B0F908500D8108
:10DDB000EDB2442D00AF0C46904600F0CC820646F2
:10DDC00043D9812D00F0048200F29980542D00F097
:10DDD000CE8040F2E9816E2D00F08B82802D40F0E4
:10DDE0001981BF4B93F800A00AF1020A1AF0FF0A4A
:10DDF00000F09980BB4BDFF82483BB4EDFF820B3E3
:10DE00009A4403F101090A2516E0322D00F0D4826C
:10DE1000A5F13C00C0B2132840F2D482002322684E
:10DE2000511C216015702268D14502F10101216069
:10DE3000137078D019F8015B0A2DE6D1BBF80030D9
:10DE4000FF2BA8BFFF23DBB2E9E7052D00F07182AD
:10DE500020D8022D00F0838040F29381032D00F042
:10DE60003E82042D40F0D6802A46A0492046FAF78B
:10DE70006FFF00212046FAF7B3FF22680221531CEE
:10DE80000125236028462B46743711706381BD46F7
:10DE9000BDE8F08F242D60D040F20481282D00F0E1
:10DEA000E081382D40F0B6800A68914B0125511C65
:10DEB00021601570226805215019206011702268B8
:10DEC0000A21501920601170226800215019206029
:10DED00011702268197850192060117022685978E1
:10DEE00050192060117022689978531923602B46CD
:10DEF0001170284674376381BD46BDE8F08FA02DB0
:10DF000019D040F21381B82D00F0E781FE2D40F0CA
:10DF10008180784D05F1080635F8021B2046FAF796
:10DF20005FFFB542F8D101252B462846743763813F
:10DF3000BD46BDE8F08F704B08461968FAF738FF08
:10DF40006E4B20461968FAF733FF6D4B196820466F
:10DF50000125FAF72DFF2B46E7E76A4BF6E7042287
:10DF6000694920460125FAF7F3FE2B46C1E70B6805
:10DF7000664ADFF8B081581C1121206019702368AF
:10DF80001278591C21601A70236898F85B20591C7C
:10DF900021601A70236898F85A20591C21601A7061
:10DFA000B8F856102046FAF71BFF00212046FAF772
:10DFB00017FFB8F858102046FAF712FFA8F102052B
:10DFC00008F1480635F8021F2046FAF709FFB54266
:10DFD000F8D122684E4B0C21501C20605D18117046
:10DFE000226813F8011F501C9D4220601170F7D168
:10DFF00023680222591C21601A70B8F85C10204670
:10E00000FAF7EEFE0125B8F85E102046FAF7E8FEB2
:10E010002B466EE72146284601F01AFF03460028EA
:10E0200081D1742D00F0C680772D0DD132687168D2
:10E0300091421EBF531C33601178364A08BF1946FF
:10E0400020462BF097FE6EE7F52D01F0AF83762D7D
:10E0500000F08981472D00F074823268392D114615
:10E0600000F05B8300F20882212D01F05F83292DEF
:10E0700040F07083531C336013780A2B01F0428404
:10E08000502B40F076853046FAF750FEDFF8988046
:10E09000A8F800003046FAF749FE0125A8F802006A
:10E0A0002B4626E7202DB5D10B681B4D591C6A78ED
:10E0B00021601A7023682A78591C21601A7023681D
:10E0C000AA78591C21601A7029892046FAF788FE1F
:10E0D00023686A79591C21601A702268A979CEE6F2
:10E0E000E57C002080DD030848300020A674002075
:10E0F0004F590020087D0020107AFF1F147AFF1F5F
:10E10000187AFF1FC05A002078120408B07400204B
:10E11000DD58002079900308D4A600206766666663
:10E12000703000209458002030300020822D7FF481
:10E1300071AF0B68BB4ABC4D1178BC4A581C2060BB
:10E14000197011892046FAF74BFEB94B22681B88DB
:10E15000FF2B02F10101A8BFFF2321601370A96802
:10E1600081F3100189B22046FAF73AFE296801F3DB
:10E170000F0189B22046FAF733FEAE4B22681978B8
:10E180007DE6012D7FF446AF0B680022591C21600B
:10E190001A7023685A1C22601D7022682421531CA7
:10E1A00023602B461170A4E6522D7FF433AF226812
:10E1B000002164E63268716891421EBF531C3360CF
:10E1C00011789D4A08BF194620462BF0D3FDAAE6D8
:10E1D0009A4B1E78033616F0FF063FF4A4AE984B18
:10E1E000DFF88C821E4403F1010A4FF00A0920E097
:10E1F000B9F1500F00F0DE80B9F1320F00F0F78076
:10E20000A9F13C00C0B2132840F2F4800025294651
:10E2100023685A1C2260204683F80090FAF7E0FD3C
:10E2200029462046FAF7DCFD56453FF47CAE1AF845
:10E23000019BB9F10A0FDBD1824B9D68196805EB90
:10E2400085054FF6FF736D009D42A8BF1D4699429C
:10E25000A8BF194625EAE57521EAE171ADB289B298
:10E26000D6E70B68DFF80C92774E591C022221602A
:10E270001A7023684FF006085A1C226083F8008049
:10E2800023680A22591C21601A70236801255A1933
:10E2900022601D70B9F800102046FAF7A1FDB9F808
:10E2A00002102046FAF79CFD23685A19226083F871
:10E2B000008023685022591921601A7023680022B7
:10E2C000591921601A7031882046FAF789FD718842
:10E2D0002046FAF785FD2B460BE65C4B36E60B68CD
:10E2E0005A1C0A601D700B680222591C21601A70AA
:10E2F0005DE74F4B0A681B884B4DFF2BA8BFFF23E0
:10E30000511C21601370A96881F3100189B2204665
:10E31000FAF766FD4E4B20461988FAF761FD296829
:10E3200001F30F0189B220460125FAF759FD2B466A
:10E33000DFE50B2247492046FAF70AFD0822464945
:10E340002046FAF705FD0125072244492046FAF741
:10E35000FFFC2B46CDE5002A3FF4E5AD404B1360B2
:10E3600001252B46C5E53268511C31601278002A20
:10E3700001F0CF82102A07BF3A4B93E822001D46D6
:10E3800029462368581C20601A702046FAF710FDB1
:10E3900029462046FAF70CFD334B20465968FAF718
:10E3A00007FD20460021FAF71BFD00212046FAF761
:10E3B00017FDFCE62D4B40E73388FF2BA8BFFF235A
:10E3C000DBB22CE522F088FE00283FF427AD03786D
:10E3D0000A2B25D8B0F9023088FB0312DB17C3EBF8
:10E3E000A2039BB2FF2BA8BFFF23DBB217E598E87F
:10E3F000220024E722F070FE00283FF407AF0378E4
:10E400000A2B3FF603AFB0F90430B0F9061003EB66
:10E41000830383F3500521EAE171ADB289B2F7E6D7
:10E420000023E2E7FE7D0020B4A40020D4A6002053
:10E43000E87D0020907F0020219C0308E57C0020DF
:10E4400090DD0308FC2F00203030002074400020B5
:10E45000887F0020801204088C1204089812040897
:10E4600081FD0008C42A0020E4240020343000206C
:10E47000403000205C840020552D00F02781572D6E
:10E4800040F06881531C336012F8378B07F12F017D
:10E490000133336013F8010C01F8010F9342F7D1F7
:10E4A000DFF8A4A29AF80050002DFDD1DFF89CB24D
:10E4B0000126DBF800008AF80060FEF795FF9F4B0D
:10E4C00028461E702BF060FD28462BF05DFD0920CC
:10E4D0002BF05AFD40462BF057FD07F1300845461A
:10E4E00007F16609A5EB0806F6B20A202BF04CFDF1
:10E4F00030462BF049FD15F8016B0B202BF044FD45
:10E5000030462BF041FD0020FEF792FB4D45E9D14E
:10E5100008202BF039FDA0202BF036FDA0202BF099
:10E5200033FD00202BF030FD10F02000F6D1064620
:10E530000125DBF80000FEF75DFF8AF800602B463E
:10E54000D7E4726835687B623046551BFAF7D6FB14
:10E55000052D38627B6A01F2C8818026B346012509
:10E5600094E80600521A103A9642C8BF1FFA82FB7E
:10E57000734A396A92683A61521A9345396A7B62E2
:10E580002046FA6088BF1FFA82FBFAF711FC7B6A0B
:10E59000002B01F08981002D41F065812368C7F8C7
:10E5A00000D05D71C0B00533C7F804D0FB61BBF18A
:10E5B000000F01F07D823B6A3A69934281F0D38279
:10E5C0003E6A7D62AA46A846BC608025FB68A3EB34
:10E5D00008085B4BB8F5807F9B6828BF4FF48078B4
:10E5E00006EB08029A4288BFA3EB0608FCF78CF8FA
:10E5F0007C68424621463046FCF706F9F969B86165
:10E6000004EB000C0B787B6164452ED2DFF840915F
:10E610000CF1FF3C04F1FF3E1EF8013F09EB8302C1
:10E6200019F823405688ECB100234FF4004204F15E
:10E63000FF3816424FEA520202D008782843087089
:10E640006D0806D10AF1010A4D701FFA8AFA0131EC
:10E650008025D34503D8E64532D3984530DC0133D5
:10E660009C42E6D1E645D7D1F9617B6ABA69134489
:10E670009BB2D3457B6206D97B6A3A6A9846D61824
:10E680003B699E42A2D3BC68802D1CBF0AF10103E6
:10E690001FFA83FA0AF1020189B22046FAF7A0FBB9
:10E6A0002368796A01255A19226020461D70FAF7FD
:10E6B00097FB2368534423602B46D7F800D018E417
:10E6C000FB69BC681A463B7D1370DDE7531C336061
:10E6D00092F80080B8F1FF0F01F0B881B8F1FE0F99
:10E6E00001F060813046FAF721FB96E80C009B1A96
:10E6F000002B07DD531C336013781BB9B8F10B0FE7
:10E7000041F28881B8F1240F00F2C9850D4B012533
:10E7100023F818002B46FFF7ECBB531C336013782B
:10E720000A2B01F0FB803046FAF70CFB3046FAF773
:10E7300009FB3046FAF706FBFFF7F5BB3A68002005
:10E74000D41D0020945800203068002094740020CC
:10E75000A0DD030870680B3D831AEF2D00F29F8542
:10E760000FF2040E5EF825F0C9F400089FF20008CD
:10E770009FF200089FF200089FF200089FF2000835
:10E780009FF200089FF200089FF200089FF2000825
:10E790009FF200089FF200089FF200089FF2000815
:10E7A0009FF200089FF200089FF200089FF2000805
:10E7B0009FF200089FF200089FF200089FF20008F5
:10E7C0009FF200089FF200083FF400089FF2000843
:10E7D0001DF400089FF20008F3F300089FF2000800
:10E7E0009FF200089FF20008CBF300089FF2000898
:10E7F0004BF300089FF2000819F300089FF200088D
:10E80000A5F300089FF200083FF200089FF20008FD
:10E81000A9F200089FF2000851F200089FF20008D8
:10E820009FF200089FF200089FF2000827DF00080F
:10E830009FF20008FDF200089FF200089FF2000816
:10E8400043F000089FF2000829EB00089FF200083F
:10E850009FF200089FF200089FF20008EBF000080A
:10E860009FF200089FF200089FF20008ABF000083A
:10E870009FF200085DF000089FF200089FF2000878
:10E88000FDF100089FF200089FF200089FF20008C7
:10E890009FF200089FF200089FF200089FF2000814
:10E8A00029F100089FF20008CFEF00089FF200084E
:10E8B0005DEF00089FF20008A9EE00089FF2000833
:10E8C00081EE00081BEE00089FF200089FF200088E
:10E8D0009FF200089FF200089FF200089FF20008D4
:10E8E0009FF200089FF200089FF200089FF20008C4
:10E8F0009FF200089FF200089FF200089FF20008B4
:10E900009FF200089FF200089FF200089FF20008A3
:10E910009FF200089FF200089FF200089FF2000893
:10E920009FF200089FF200089FF200089FF2000883
:10E930009FF200089FF200089FF200089FF2000873
:10E940009FF200089FF200089FF200089FF2000863
:10E950009FF200089FF200089FF200089FF2000853
:10E960009FF200089FF200089FF200089FF2000843
:10E970009FF200089FF200089FF200089FF2000833
:10E980009FF200089FF200089FF200089FF2000823
:10E990009FF200089FF200089FF200089FF2000813
:10E9A0009FF200089FF200089FF200089FF2000803
:10E9B0009FF200089FF200089FF200089FF20008F3
:10E9C0009FF200089FF200089FF200089FF20008E3
:10E9D0009FF200089FF200089FF200089FF20008D3
:10E9E0009FF200089FF200089FF200089FF20008C3
:10E9F0009FF200089FF200089FF200089FF20008B3
:10EA00009FF200089FF200089FF200089FF20008A2
:10EA10009FF200089FF20008F1ED00089FF2000845
:10EA200041EF00089FF200089FF200089FF20008E3
:10EA30009FF200089FF200089FF200089FF2000872
:10EA40009FF200089FF200089FF200089FF2000862
:10EA50009FF200089FF200089FF2000893ED000863
:10EA600041ED000809ED00089FF2000867EC00087E
:10EA70004DEC000831EC00089FF2000817EC00088C
:10EA8000ABEB000883EB000879EB0008CDF600083B
:10EA90009FF200089DF600089FF200089FF2000810
:10EAA00073F6000845F6000831F6000809F600087C
:10EAB000E9F50008BFF5000893F500089FF200088B
:10EAC0009FF200089FF200089FF200089FF20008E2
:10EAD0009FF200089FF200089FF200089FF20008D2
:10EAE0009FF200089FF200089FF200089FF20008C2
:10EAF0009FF200089FF2000873F500089FF20008DB
:10EB00009FF2000819F500089FF200089FF2000824
:10EB10009FF200089FF200089FF200089FF2000891
:10EB20009FF20008FFF40008531C3360C24B1278B8
:10EB3000DFF844831A700023C8F800303046FAF733
:10EB4000DDF83368D8F80020BC49BD4D10435A1C8D
:10EB5000C8F8000032601B780B723046FAF7E6F80E
:10EB600028603046FAF7E2F868603046FAF7DEF8D7
:10EB7000A8603046FAF7DAF83046FAF7D7F8FFF728
:10EB8000D2B9531C33601078060601F16380AD4B97
:10EB90001B78DD073FF5C7A9032828BF0020012502
:10EBA00002F0D2F92B46FFF7A4B9531C336030466C
:10EBB00092F800A0FAF7A2F881463046FAF79EF8DC
:10EBC00005463046FAF79AF880463046FAF7AEF82E
:10EBD0003046FAF7ABF83046FAF7B4F8BAF1000F5E
:10EBE00001F02180BAF1100F7FF49DA9964BC3F874
:10EBF00000905D60B8F1000F02D0944BC3F8048020
:10EC00009349944B0222081F01251A7018F086FEC2
:10EC10002B46FFF76EB98B4B1B78D8073FF583A9BE
:10EC2000012502F041FC02F05DFA2B46FFF761B9C5
:10EC3000844B1B78DA073FF576A9874A13780125BC
:10EC400043F0040313702B46FFF753B97D4B1B7839
:10EC5000D9073FF568A9814B4FF4C87201251A8086
:10EC60002B46FFF746B9092B40F31983DFF80C82D6
:10EC70001346511CD8F80050316013F8021B29705C
:10EC800033605378AB70D31C33609378642B02F1FC
:10EC90000401A8BF64236B713160D378642B02F147
:10ECA0000501A8BF6423AB7131601379EB71931D2B
:10ECB00033605379642B02F10701A8BF64232B72E0
:10ECC00031609379EB7002F108033360D3792B71D3
:10ECD0003046FAF72BF8726833686881D11A002938
:10ECE0000CDD591CD8F800003160521A002A19783E
:10ECF000417203DD9A1C32605B784370012517F086
:10ED0000D1FF2B46FFF7F5B8554B1868D31C0146C9
:10ED100021329D1E356013F8035C0D705D1E356059
:10ED200013F8025C4D70336013F8015C8D7003338F
:10ED30009A4201F10301ECD116F0FEFAFFF7F3B8A5
:10ED4000531C336013784449002B00F08E870B78F6
:10ED500043F00203901C0B70424D306053782B75CA
:10ED60003046F9F7CBFF28603046F9F7C7FF6860F7
:10ED70003046F9F7DBFF28813046F9F7D7FF3A4AEA
:10ED8000E8811378012543F0020313702B46FFF747
:10ED9000B0B8C3F34705122D00F28182C5B107F167
:10EDA000700307F12E0A03EB4508D146A8F142088B
:10EDB0003046F9F7BBFF29F8020FC845F8D12B4BB5
:10EDC0003AF8022F23F8022FD145F9D1112D09D895
:10EDD000274A6B00023B13440021223223F8021F12
:10EDE0009A42FBD1234A01231D461370FFF781B8D5
:10EDF0001346511C316013F8025B3360D31C50780A
:10EE000033609178002D00F0FD86012D7FF48BA8F2
:10EE100010F062FD2B46FFF76CB80A4B1B7813F01D
:10EE2000010140F03C82531C33601078012510F042
:10EE300095FC2B46FFF75DB8AC5F0020F0940020F6
:10EE4000303E0020747D0020C42A0020E4240020ED
:10EE5000C82A0020906C0020ECA60020E2B100201F
:10EE60005C590020F0A600208E6C00208AA20020B1
:10EE70008CA20020B0A20020C05A00201C4B002011
:10EE80001346511C31609C4913F8020BC870336063
:10EE90009A4953784B71D31C3360994B9278DA704E
:10EEA00001252B46FFF725B83046F9F73FFF3046DE
:10EEB000F9F73CFF3046F9F739FF3046F9F742FFE2
:10EEC0003368904D1946581C2A68306011F8020BBF
:10EED00082F82C003160597882F83610D91C3160E4
:10EEE0009B7882F837303046F9F72CFF3046F9F737
:10EEF00029FF3046F9F726FF3046D5F80080F9F7AC
:10EF000015FFA8F83A003046D5F80080F9F70EFF53
:10EF100096E80C00991A0129A8F838000ADD511C5E
:10EF20002B683160127883F82E203046F9F70AFFFB
:10EF300096E80C009B1A032B00F39C862868FBE6DE
:10EF4000DFF8DC8100233046C8F80030F9F7D6FE40
:10EF50000125C8F800002B46FEF7CBBF531C3360D9
:10EF6000684DDFF8C081137888F805303046D5F851
:10EF70000090F9F7DBFEA9F820003046D5F80090A4
:10EF8000F9F7D4FE96E80C00991A0729A9F81E0093
:10EF900000F31C86991A032900F30A869B1A002B9A
:10EFA00005DD511C2B683160127883F8262001F0B2
:10EFB000F1FF1FF0BFF9544B1B68002B00F02886AF
:10EFC0002868012515F05EFE2B46FEF792BF13461A
:10EFD000511C3160DFF84C8113F8021B88F80210D5
:10EFE00033604A4953780B70D31C3360484D937893
:10EFF0002B71131D3360D378092BA8BF092330462A
:10F00000AB70F9F793FE96E80C00991A0129288055
:10F0100005DD3046F9F78AFE96E80C00E881934258
:10F0200040F0BC8501F0B6FF336872689A423EF446
:10F030007AAF5A1C32601B78EB7001252B46FEF725
:10F0400058BF344B03F10801501C3060127803F8AC
:10F05000012F99423EF467AF3268F5E7531C3360E5
:10F0600092F80080B8F1110F00F21981931C3360FF
:10F07000294D537805F818303046F9F757FE40F619
:10F08000CA039842A8BF184640F2EE23984205EB07
:10F090004801B8BF18460125A0F2EE222B461920E0
:10F0A00092FBF0F24A70FEF724BF1346511C1B4D31
:10F0B000316013F8021B2971336053786B7130464D
:10F0C000F9F734FE336828805A1C32601B78AB7124
:10F0D0003046F9F72BFE336868805A1C32601B7883
:10F0E000EB7101252B46FEF704BF0125FBF76EFBF4
:10F0F0002B46FEF7FEBE00BF6C840020FC81002082
:10F100007C8400205C590020A45F002060840020E3
:10F1100084760020EF9400205CA40020644200204C
:10F1200074400020B47900203046F9F7FFFD054611
:10F1300018F002FDFF283EF4F6AE3F2D00F21785D1
:10F1400007F17008002308F8403D4FEAD509414611
:10F1500007F12F0087F82F3009F1010918F0CCFCD6
:10F1600097F82F305FFA89F905F007054B4505F14F
:10F17000010503D197F83030AB4203D02946484609
:10F1800018F0C6FC33687268D21A012A7EF7CBAE3B
:10F190005A1C07F17000326000221D7800F8412DE2
:10F1A00018F09EFC97F82F30AB420AD0B94B1B6881
:10F1B0003BB19A79AA4204D31B681B690BB128465C
:10F1C000984733685A1C3260404600221D7887F801
:10F1D000302018F079FC97F83030AB423EF4A3AE03
:10F1E000AC4B1B68002B3EF49EAE1B685B69002B8A
:10F1F0003EF499AE28469847FEF795BEA64B1B787D
:10F20000012B3EF690AE1146531C3360DFF8AC8202
:10F2100011F8023B88F802303160D31C92F801E00B
:10F220003360C31A012B917840F391843046F9F78B
:10F230007DFD0125A8F800002B46FEF75ABE531CA1
:10F240003360964B12785A7501252B46FEF751BE56
:10F250000722B3FBF2F2C2EBC2055B1B1FD1D2B295
:10F2600002F1FF395FFA89F9002A3EF45CAEDFF85B
:10F2700030A209F101091D464B1C336091F90010C1
:10F28000874B4FF0000893F902208A4203F10803EC
:10F2900000F09B8308F10108B8F1060FF3D14FF09D
:10F2A000FF352B46FEF725BE531C336013780E2B1B
:10F2B000F5D8911C31605578032DF0D87948062196
:10F2C00001FB03F1431802F1030E5D71C6F800E083
:10F2D00095784554111D3160D1785970511D3160B8
:10F2E00011799970911D31605179D970D11D3160BA
:10F2F00092791A7101252B46FEF7FBBD1346511C6E
:10F300003160694913F8020B8870336053784B7091
:10F3100001252B46FEF7EDBD644D05F14008304652
:10F32000F9F704FD3368A5F88000591C1A463160CE
:10F3300012F8021B85F8821032605B7885F8833002
:10F340000435A845EBD1FEF7EEBD531C534D336099
:10F3500013782B723046F9F7E9FCA8833046F9F7A9
:10F36000E5FC28833046F9F7E1FC336868835A1CD2
:10F3700032601B78EB7473689A1A032A00F3C8830F
:10F380003268991A052900F3B3839B1A002B7EF784
:10F39000CAAD531C3360137885F8213001252B4604
:10F3A000FEF7A7BD511C316015781F2D3FF677AFD2
:10F3B000052B7FF474AF3046F9F7A0FC3B4B43F8C4
:10F3C00025001DF051F9FEF7AEBD531C33603849DE
:10F3D00015780D70C31A002B7EF7A5AD931C336012
:10F3E0005378003318BF012301254B702B46FEF7DD
:10F3F00080BD3046F9F79AFCDFF8C480C8F80000F9
:10F400003046F9F793FCC8F804003046F9F78EFC53
:10F410000125C8F808002B46FEF76BBDDFF8A48075
:10F420000023C8F800303046F9F768FCD8F80030FF
:10F4300001250343C8F800302B46FEF75ABD531C84
:10F4400033601578132D3FF62AAF931C3360507844
:10F450007A622AF0C9FC00283FF421AF7A6A154B82
:10F46000017803F82510D11C316003EB85039178F6
:10F470005970111D3160D0789870501D30600E4960
:10F480001279DA700868012517F09AFB2B46FEF70F
:10F4900030BD00BFA84B0020A75A0020F0940020E8
:10F4A000BC7400208040002088840020347E00202E
:10F4B000AC5F0020B05F00205C590020AA5A0020F9
:10F4C000303E0020C05A0020A84A102B4FF0000107
:10F4D00028BF1023116051609160D1601174002B1E
:10F4E0003EF421AD3168013A0B440131316011F82D
:10F4F000010C02F8010F9942F7D1FEF714BD9C4BA5
:10F500001B78DB073FF5CBAE012501F039FD01F09B
:10F51000E9FD2B46FEF7EDBC531C336013780F2B2F
:10F520003FF6BDAE911C3160C3EBC30391495078E7
:10F53000C854D01C30600B4491785970111D316053
:10F54000D1789970511D31601179D970911D316058
:10F5500051791971D11D31609179597102F1080108
:10F560003160D2799A71012515F0F8FA2B46FEF731
:10F57000C0BC3046F9F7DAFBDFF80482A8F80E00C9
:10F580003046F9F7D3FB0125A8F80C002B46FEF70F
:10F59000B0BC1146531C3360774B11F8020B187046
:10F5A000316051785970D11C316091789970111D7A
:10F5B0003160D278DA7001252B46FEF79ABC3046CE
:10F5C000F9F7B4FBDFF8D481A8F810003046F9F75A
:10F5D000ADFBA8F812003046F9F7A8FB0125A8F802
:10F5E00014002B46FEF785BC1346511C316013F8FE
:10F5F000020B3360D31C51783360927823F0B4F857
:10F6000000287EF490AC4AE61346511C31605B49F9
:10F6100013F8020B08703360594953788B70D31C70
:10F620003360584B92789A7001252B46FEF761BCE7
:10F63000554B564918684E2201252BF093FF2B4657
:10F64000FEF757BC1146531C3360514B11F8020BA7
:10F650001870316051785970D11C316092789A706D
:10F660003046F9F763FB4B4B0125D8802B46FEF75C
:10F6700040BC3046F9F75AFBDFF81881A8F80000C3
:10F680003046F9F753FBA8F802003046F9F74EFB75
:10F690000125A8F804002B46FEF72BBCDFF80091EB
:10F6A00099F80030002B3EF43EACDFF8F8800025DE
:10F6B0003046F9F73BFB13F0F1FC99F80030A8EC69
:10F6C000010A01359D42F3DBFEF72DBC0D2B7FF4C3
:10F6D000E6AD531C33601578072D3FF6E0ADDFF83B
:10F6E000C89030464FF00C08F9F720FB08FB05F8EE
:10F6F00009EB0805A8803046F9F718FBE88030468A
:10F70000F9F714FB336828811A46591C316012F846
:10F71000021BA97232605B78EB723046F9F7EEFAA1
:10F72000012549F808002B46FEF7E3BB1346511CA0
:10F730003160194D13F8021B6970336053782B70D8
:10F74000D31C33609378AB703046F9F7EFFA336827
:10F750002881591C1A46316012F8021B6971326007
:10F760005B78AB7101252B46FEF7C3BB48840020B4
:10F77000747D0020F84400202C660020B47900201D
:10F780006C8400207C8400205C590020E4F803088D
:10F79000648400204C420020D4A6002084760020FF
:10F7A000E57C0020A44100200444002033687268F6
:10F7B0009A4240F0C480C14BFF221A704FF0000AF9
:10F7C000BF4D0FF0BDFD51462022BE4885F800A078
:10F7D0002EF0DFF987F830A097F83030072B00F2D1
:10F7E0005781DFF80493B74E524697F8303003EB59
:10F7F000430309EBC3035B7CE3B197F8303003EBC1
:10F80000430309EBC30320215B699BB197F83030B8
:10F8100003EB430309EBC303586946F82200FDF7E5
:10F820002BFD2B7856F82300FDF7E4FD2A780132F2
:10F83000D2B22A7097F830300133DBB287F830301B
:10F8400097F83030072BD0D92368591C21601A70E3
:10F85000B8F1000F3EF467AB9B4BC8F800300125B0
:10F860002B46FEF746BB994B3A6A9B68D4F800904A
:10F870005A449A4200F2D980FAF746FF5A4649465E
:10F88000386AFAF7C1FF23680344236086427EF793
:10F890004AAB002100E0236801305A1C86422260F6
:10F8A0001970F8D1FEF73FBB002DDCD15946204638
:10F8B000F9F796FA23685A1C22601D70834B26685C
:10F8C0009D683B6A0BEB0302954280F0E3803B6A44
:10F8D000ED1AFAF719FF2A463146386AFAF794FF0B
:10F8E000236803442360FEF71EBB3046F9F71EFA77
:10F8F000326871687B6A9142834649D106461D464B
:10F90000FEF72EBE3046F9F711FADFF8E081FEF778
:10F91000BFBB6F4B93E82200FEF733BD931C3360EF
:10F920006C4B51781970D11C316091785970111D50
:10F930003160D2789A7001252B46FEF7DABA5A1C4C
:10F94000194632605D4811F8022B027031605B7815
:10F950004370042A03D9FF2A7EF429AC2EE75E49BE
:10F960000978994205D8022A7EF421ACFF2B7EF457
:10F970001EAC236801255A1922601D70B8F1000FD2
:10F980003EF4D1AA554BC8F800302B46FEF7B1BA69
:10F99000511C316012781D46131C064618BF012306
:10F9A000FEF7DEBD931C33605578022D3FF677AC31
:10F9B0003046F9F7BBF94A4B03EB45034FF0FF35EF
:10F9C000A3F85C002B46FEF794BA0AEBC80B30464E
:10F9D0008BF80210F9F7AAF933682AF838001A46AA
:10F9E000591C316012F8021B8BF8031032605A78F0
:10F9F0008BF80420DA1C32609A788BF80620191DE7
:10FA000031600135DB788BF80530A9457FF434ACE3
:10FA1000FEF789BA324B0030984418BF0120012507
:10FA200088F84A002B46FEF764BA3A6AA3EB02084C
:10FA3000FAF76AFE42464946386AFAF7E5FE236855
:10FA400003442360002D3EF46EAA1FE7931C33602D
:10FA5000244B51781970D31C3360DFF8848093787D
:10FA600088F85B30131D3360D37888F85A303046FD
:10FA7000F9F75CF9A8F856003046F9F757F930461F
:10FA8000F9F754F90125A8F858002B46FEF731BACA
:10FA90005246D9E6FAF738FE5A463146386AFAF73E
:10FAA000B3FE23680125034423602B46FEF721BAE9
:10FAB000DA46C7F824B0FEF7EDBD00BFE42400200D
:10FAC000DF42002088A30020913D0208D41D0020C1
:10FAD000846C00204F590020E57C00208DFD00083B
:10FAE00094580020B0740020C47500205C8400206D
:10FAF000531C33601378EB723046F9F7FFF8336824
:10FB0000E8605A1C32601B782B7496E80C003CE4C9
:10FB10003046F9F70BF9A8843046F9F707F996E86B
:10FB20000C00991A0329E8847FF72BAC1346511C6B
:10FB3000316013F8021BA9773360537885F82030C1
:10FB40003046F9F7F3F896E80C00688419E4504B56
:10FB50001A88012512FB0EF22B4692FBF1F2A8F84F
:10FB60000020FEF7C6B97D62AA46FEF793BD07F1F5
:10FB70003008404617F09CFF3B8EAB423FF402AB8F
:10FB8000444B1B68002B3FF4FDAA1B689B69002BAC
:10FB90003FF4F8AA28469847FFF7F4BA531C33609D
:10FBA0001378003318BF012388F80730FFF73ABAFB
:10FBB0003046F9F7BBF8A8F80E003046F9F7B6F86A
:10FBC00096E80C00A8F81000FFF7E8B93046F9F7FE
:10FBD000ADF8A8F80A003046F9F7A8F8A8F80C0024
:10FBE0003046D5F80090F9F7A1F8A9F82200304680
:10FBF000D5F80090F9F79AF896E80C00A9F82400D7
:10FC0000FFF7C8B9012515F005FA2B46FEF771B9C3
:10FC100021482249224A234B036001250B601360CF
:10FC20002B46FEF766B9204B1020C3F800905D60AC
:10FC30000DF0B6FA1D4A137843F001031370B8F1C2
:10FC4000000F3EF470A91A4B0125C3F804802B461F
:10FC5000FEF74FB900F07F00032828BF00200125E0
:10FC60000FF056FE2B46FEF744B90B7803F0FD0368
:10FC7000FFF770B83046D5F80080F9F757F8A8F8C4
:10FC8000320030462E68F9F751F8B086FFF756B9C2
:10FC9000AC820020A84B002070450020C445002005
:10FCA000C44900206D820008846C0020ECA600206E
:10FCB000E424002038B50B4C23688BB15A68821AB3
:10FCC000002A054604DA0CE05A68AA1A002A07DB63
:10FCD0009A68226018461A6890472368002BF3D16F
:10FCE00038BD38BDC85E00200B4B002210B4027234
:10FCF00003F58474042102E0072A09DC9979890755
:10FD000002D51979815401329C4203F11803F3D1D1
:10FD10005DF8044B704700BFAC05040810B40D4CEF
:10FD200004232146002200E08B7913F0010301F146
:10FD3000180106D101320C2AF6D103705DF8044B8C
:10FD4000704702EB420204EBC2025DF8044B1379E8
:10FD500003707047AC050408012310B4332131242B
:10FD6000322244704171C2700370037183705DF878
:10FD7000044B70471F22032302704370704700BF7B
:10FD800008B513F00DFAFBF7A7FD00BF024A034BBD
:10FD90001278197817F0DCBEE4240020E524002056
:10FDA000038A2DE9F0478589ADB21D4029D00F4661
:10FDB00006464FF000484FF00009B5FA85F328FADF
:10FDC00003F2D24391B21B3B15403182042B16D86B
:10FDD000DFE803F03129211903007B6A002B32D0C0
:10FDE00003F1FF3A1FFA8AFAC7F824903C6A34B14B
:10FDF00023682046514698476468002CF8D1002DAE
:10FE0000DBD1BDE8F0873868716B036889B2984729
:10FE1000002DD2D1F5E77868B16B036889B29847B5
:10FE2000002DCAD1EDE7B868F16B036889B2984735
:10FE3000002DC2D1E5E7F868316C036889B29847B4
:10FE4000002DBAD1DDE7F36A1FFA83FACEE700BFCF
:10FE50002DE9F04F2DED028BA0F10A0389B00C467D
:10FE6000E72B00F21187DFE813F01C010F070F07E3
:10FE70000F070F070F070F070F070F070F070F07D2
:10FE80000F070F070F070F070F070F070F070F07C2
:10FE90000F070F070F070F070F0790050F070F0733
:10FEA0000F0780050F070F070F0779050F071905C3
:10FEB0000F0700050F07F4040F07EC040F07C70432
:10FEC0000F07B3040F070F070F07AD04A6040F07B2
:10FED00099040F070F07E6010F07BE010F070F0771
:10FEE0000F07A2010F070F070F070F0783010F0767
:10FEF000FC000F07E60593060F070F070F070F0714
:10FF00000F070F070F0781030F0753030F071F0387
:10FF10000F0767020F071E020F070F070F070F07D4
:10FF2000FC02BB02F502ED01E800C2037E06660694
:10FF30008F040F0758043C040F070F070F070F0724
:10FF400031040F070F0710040F070F070F070104F5
:10FF5000F70651060E060F070F070F07FE05B70637
:10FF60000F0764010F070F070F070F070F070F0792
:10FF70000F070F070F070F070F070F070F070F07D1
:10FF80000F07FC020F070F070F070F070F070F07D9
:10FF90000F070F070F070F070F070F070F072D0199
:10FFA0000F070F070F070F070F070F070F070F07A1
:10FFB0000F070F070F070F070F070F070F070F0791
:10FFC0000F070F070F070F070F070F070F070F0781
:10FFD0000F070F070F070F070F070F070F070F0771
:10FFE0000F070F070F070F070F070F070F070F0761
:10FFF0000F070F070F070F070F070F070F070F0751
:020000040801F1
:100000000F070F070F070F070F070F070F070F0740
:100010000F070F070F070F070F070F070F070F0730
:100020000F070F070F070F070F070F070F070F0720
:100030000F070F070F07DA05AF05A54E337853B149
:10004000A44F002537F8021F2046F8F7C9FE337881
:100050000135AB42F6DC012009B0BDEC028BBDE8F6
:10006000F08F9B4E3378002BF5D09B4F0025B84680
:10007000236817F81520591C21601A7098F8011090
:1000800001EB810101EB810101F2EE2189B22046F1
:10009000F8F7A6FE33780135AB4208F10208E7DC39
:1000A000D9E78E4D28462AF01FFB0028D3DD2B46CA
:1000B0000544226813F8011B501C9D4220601170FA
:1000C000F7D1C8E70B68DFF868C2591C9CF800201C
:1000D00021601A709CF80030002BBCD0804E814DFE
:1000E000814882490023226816F8017F02F1010E3F
:1000F000C4F800E01770226815F8017F02F1010EC4
:10010000C4F800E01770226810F8017F02F1010EB8
:10011000C4F800E01770226811F8017F02F1010EA7
:10012000C4F800E017709CF8002001339A42DADC32
:1001300091E70B686E4F591C3A7821601A703B7832
:10014000002B88D00025EEB2304620F0C5FF236892
:100150004278591C216030461A7020F0BDFF018999
:100160002046F8F73DFE3B780135AB42EBDC72E709
:100170000B68604D591C2A7921601A7023686A79CE
:10018000591C21601A7029882046F8F729FE236837
:10019000AA79591C21601A7069882046F8F720FE58
:1001A0002368EA79591C216001201A7054E7FAF794
:1001B0009DF92368504D002803F101010CBF022274
:1001C000032221601A7029882046F8F7F1FDA968FA
:1001D0002046F8F7EDFDFAF761F901462046F8F7F9
:1001E000E7FD012038E70B68444A454D1178454A40
:1001F000581C2060197011682046F8F7D9FD236853
:10020000414A591C127A21601A7029882046F8F751
:10021000E7FDA9882046F8F7E3FD29892046F8F78D
:10022000DFFD00212046F8F7DBFD20460021F8F72E
:10023000D7FD012010E7084608223349F8F788FD6A
:10024000012009E7314D324E9FED328ADFF8E4801C
:10025000DFED318A05F120070EE0FCEEE77ACDED07
:10026000017ABDF8041020460435F8F7B9FDAF4215
:1002700006F118063FF4EFAE717C0029F3D0274B4E
:10028000D5ED007A1B78012BE7D1254B1B68DB04E9
:1002900040F1B885F5EE407AF1EE10FA40F0E585D0
:1002A00040F2DC51DFE70B681E4A1F49D0781F4A35
:1002B0005D1C2560187023684979581C20601970EE
:1002C0002368D278591C216001201A70C4E600BF4F
:1002D0007CA200205E7F00205CA4002048840020D7
:1002E000476600205766002077660020676600207A
:1002F000E57C002064420020D41D0020AC5F00207B
:10030000303E0020C05A0020F0940020805F002082
:10031000C47500200000404200E08244A87600201E
:10032000D87900206C840020FC8100207C8400208F
:1003300045660020DB9B914100212046F8F750FDE7
:1003400000212046F8F74CFD00212046F8F748FD33
:100350002368B94D00265A1C22601E7023682A6843
:10036000591C92F82C2021601A7023682A68591CA5
:1003700092F8362021601A7023682A68591C92F876
:10038000372021601A7023685A1C22601E7023686F
:100390005A1C22601E7023685A1C22601E702B6833
:1003A0002046598FF8F71CFD2B682046198FF8F767
:1003B00017FD23682A68591C92F82E2021601A70B4
:1003C00023685A1C22601E702B682046598EF8F74D
:1003D00007FD2B682046998EF8F702FD01203BE6C9
:1003E000964B9B8AB3F5006F00F21585B3F5806FCD
:1003F00000F23885B3F5007F34BF01270227904D06
:1004000005F10C0655F8041B91FBF7F1204689B263
:10041000F8F7E6FCB542F5D18A4D8B4F05F10C0695
:10042000B5EC010AD7ED087A80EE270A2BF0A4FA82
:1004300081B22046F8F7D4FCAE42F1D1834D05F1EC
:100440000C0655F8041B204689B2F8F7C9FCAE42E9
:10045000F7D100E6084610227D49F8F779FC012023
:10046000FAE500258146DFF8FC81DFF8FCB105954F
:1004700004950695079501214FF6FF7A05E00135B1
:100480000B2D00F0218418F9011F4F1C4AFA05F3C7
:10049000F5D0DE07F3D5BBF800302B41D807EED5F9
:1004A00006A8F8F7D3FFEAE76A4E0B687279624D47
:1004B000591C21601A702B682046198CF8F790FCA3
:1004C0002B682046D98BF8F78BFC71892046F8F70A
:1004D00087FCB1892046F8F783FC2B682046598CAD
:1004E000F8F77EFC2B682046998CF8F779FCF189A7
:1004F0002046F8F775FC318A2046F8F771FC2A6827
:10050000236892F82620591C216001201A70A3E567
:10051000504EF378002B00F081840B680822591CA0
:1005200021601A7023680122991821601A702368CB
:10053000494D591C2A7921601A702368AA78591CE0
:1005400021601A7029882046F8F74AFCE98920467C
:10055000F8F746FC2368F279591C21601A70236869
:10056000EA78591C216001201A7075E517F0E4FA49
:10057000FF28064600F05F8408A9002501F8125DF7
:100580000DF10D008DF80D5017F0B6FA08A800F81F
:10059000115D17F0A5FA08A800F8105D17F094FA9D
:1005A00008A820F8085D17F083FA23685A1C226017
:1005B0001E7023689DF80D20591C21601A70236855
:1005C0009DF80E20591C21601A7023689DF80F2099
:1005D000591C21601A7023689DF81020591C216055
:1005E0001A702046BDF81810F8F7FAFB33E51B4BDC
:1005F0000A681B781A4D511C03F002032160137026
:1006000023682A7D591C21601A7029682046F8F752
:10061000CFFB69682046F8F7CBFB29892046F8F71D
:10062000DFFBE9892046F8F7DBFB2046298AF8F74B
:10063000D7FB012010E500BF5C5900207CA60020FC
:10064000B4A60020CC79002028A80020C0420020B9
:10065000705F0020B479002084760020ECA6002092
:10066000F0A60020D4E103088A7F0020AE4D0846A2
:100670002988F8F7B5FB69882046F8F7B1FB2046D2
:10068000A988F8F7ADFB0120E6E4A84D05F1600666
:10069000A9882046F8F7A4FBE9882046F8F7A0FBD4
:1006A00029892046F8F79CFB2368AA7A591C216007
:1006B0001A702368EA7A591C21601A7055F80C1BCD
:1006C0002046F8F775FBAE42E2D1C4E498495223C4
:1006D0002268501C2060137011F8013F002BF7D1E5
:1006E000B9E4944800232268056803EB4301561CD3
:1006F0006D5C26601570026825680A446E1C52788D
:1007000026602A70026825680A4401339278691CC1
:100710000A2B21602A70E6D19DE4874D0B682A6878
:10072000591C127821601A702B6822689978531C22
:100730002360002311702A6821681A44013352791A
:10074000481C032B20600A70F5D123682A68591CC5
:10075000127A21601A7023682A68591CD2782160A5
:100760001A7023682A68591C127921601A702B6844
:1007700020465989F8F734FB2A682368527A591CB5
:1007800021601A702A680FE000212046F8F710FB5C
:1007900020460021F8F724FB01205DE40B68674A3E
:1007A000581C91782060197023685278591C216078
:1007B00001201A7050E40B6801229918216010463C
:1007C0001A7049E408460021F8F7F2FA012043E4E0
:1007D0005B4D5C4E05F1300795F902105A4B93F9C9
:1007E00006208A4203F1080300F051829E42F6D1AE
:1007F0000835BD42F0D12EE4544B03F15A0522686E
:100800005979501C2060117022681978501C2060A2
:10081000117022685978501C2060117022689978F4
:10082000501C206011702268D978501C2060117013
:10083000226819790633501C9D4220601170DED168
:1008400009E40B68424A591C527D216001201A704C
:1008500002E4404D05F1800655F8041F2046F8F7E4
:10086000A7FAAE42F8D1FFF7F6BB3B4D05F14006C3
:10087000B5F880102046F8F7B3FA236895F882207F
:10088000591C21601A70236895F883200435591C7F
:10089000B54221601A70EBD1FFF7DDBB2C4D0B6820
:1008A0002A7A591C21601A70A98B2046F8F798FA09
:1008B000298B2046F8F794FA698B2046F8F790FACE
:1008C0002368EA7C591C21601A70A98C2046F8F72D
:1008D00087FAE98C2046F8F783FA2368AA7F591C27
:1008E00021601A70236895F82020591C21601A7025
:1008F000698C2046F8F774FA2368EA7A591C21605B
:100900001A70E9682046F8F753FA23682A7C591CC4
:1009100021601A70236895F82120591C216001205C
:100920001A70FFF799BB00BF4C420020044400201E
:10093000A4E103085C5900201C4B0020888400209F
:10094000BC740020487B0020187B002080400020E1
:10095000F0940020307E0020347E00200B68AA4AEC
:10096000581C1178206019701EE7A84D0846298888
:10097000F8F736FAA9882046F8F732FA204629898E
:10098000F8F72EFA0120FFF767BBA14D05F15006DD
:10099000287829F043FA2368027A591C21601A70DA
:1009A00023686A78591C21601A702368AA78591C38
:1009B00021601A702368EA780435591CAE42216020
:1009C0001A70E5D1FFF747BB924B03F1700522681F
:1009D0001978501C2060117022685978501C2060D2
:1009E000117022689978501C206011702268D978A3
:1009F000501C2060117022681979501C2060117001
:100A000022685979501C2060117022689979073347
:100A1000501C9D4220601170D9D1FFF71CBB7E4D48
:100A20000846E989F8F7DCF92046A989F8F7D8F9EA
:100A30000120FFF711BB0B6800255A1C0A601D70CE
:100A40000B685A1C0A601D700B685A1C0A6020460D
:100A500029461D70F8F7ACF920462946F8F7A8F9A1
:100A60000120FFF7F9BA6D4D0846298AF8F7B8F961
:100A7000698A2046F8F7B4F92046A98AF8F7B0F950
:100A80000120FFF7E9BADFF8CCE10027FEB271469A
:100A900000232268501C206016702268501C2060C1
:100AA0001370226811F8010F0133551C062B2560C5
:100AB0001070EED10137062F0EF1060EE6D158491F
:100AC00000232268501C206017702268501C206090
:100AD0001370226811F8010F0133551C0B2B256090
:100AE0001070EED123684F4A581C072120601970FE
:100AF00023680021581C20601970236892F8F020A8
:100B0000591C216001201A70FFF7A6BA0B68464AEB
:100B100041491078454A5D1C256018702368897822
:100B2000581C2060197023689278591C216001209C
:100B30001A70FFF791BA3E4D08462988F8F750F928
:100B400069882046F8F74CF9B5F90430394AD917C5
:100B500082FB0323C1EBA301204689B2F8F740F9D9
:100B60000120FFF779BA344B08461988F8F738F9AD
:100B7000324B20461988F8F733F9314B22681B783D
:100B8000511C03F00103216001201370FFF764BAC8
:100B90000B682C4E01255A1C0A601D700B68B27838
:100BA000591921601A7022F04FF82368264A274904
:100BB0005F1927601870B1F90010B2F90000F8F75A
:100BC00089FA23685A192260187031882046F8F78C
:100BD00007F92846FFF740BA0A681D4B501C1978E0
:100BE0002060117022685978501C206011702268B2
:100BF0009978501C206011702268DB78511C2160AC
:100C000001201370FFF728BAAC5F0020303E0020AF
:100C1000B05F0020F84400206C840020847600201F
:100C2000177F0020347E0020B47900207C840020CF
:100C3000CCA6002067666666D46C0020D66C0020C7
:100C40008E6C0020AA5A0020AC820020AE820020C8
:100C50002C660020F37E00200A68A34BA349187875
:100C6000551C2560107022685878551C256010703E
:100C700022689B78501C206013702046C988F8F7C2
:100C8000AFF80120FFF7E8B90020FFF7E5B92368C6
:100C90005A1C2260197029882046F8F7A1F82368A9
:100CA000EA78591C21601A7023682A79591C21603E
:100CB0001A702368AA79591C21601A7023686A790E
:100CC000591C21601A7093E5DFF844A200254FF00B
:100CD00008080135C5F1200208FA02F2A5F1200347
:100CE0002AFA05F6164328FA03F31E43252D06F0CB
:100CF00001024FF000030BD01343EAD0E8B215F025
:100D000059FF0028E5D0294606A8F8F79FFBE0E741
:100D1000774B1B78DA0700F195800025754E2F463A
:100D200002E00135252D0DD029463046F8F79EFB0F
:100D30000028F6D0294606A8F8F798FB00285CD1D1
:100D40000137EEE76C4B6D4DB3F850102046F8F7C5
:100D500047F800212046F8F743F8694B19684B0122
:100D600003F02002C1F340031343C1F3800243EABE
:100D70004203C1F3C00243EA8203C1F3401243EAD3
:100D8000C20301F0100119432046F8F729F804A91D
:100D900004222046F7F7DCFF23682978594A581CBB
:100DA0002060197011886429A8BF64212046F8F7D3
:100DB00017F8B9F1960F4AD000212046F8F710F83D
:100DC0002168B7F1190348BFA7F11203A3F3C403C5
:100DD0004A1C226020461A460B7005A9F7F7B8FF97
:100DE0002368494A581C1021206019702046118838
:100DF000F7F7DEFF0120FFF72FB9394604A8F8F70F
:100E000025FB9DE7F4EEC87AF1EE10FA4ADA4FF4CA
:100E10007A71FFF728BA0827FFF7F1BA0B68B178A3
:100E20003A4A581C2060197023681278591C2160B6
:100E30001A70FFF77CBB23685A1C226001201E70C9
:100E4000FFF70AB9069B43F00103069365E72368A1
:100E50000322591C21601A7023686A78591C21608A
:100E60001A70ADE70427FFF7CABAF4EEC87AF1EEBC
:100E700010FA3FF515AAF4EEE87AFDEEE77AF1EE06
:100E800010FA17EE901A20D86FF4F973303903FB7B
:100E900001F140F2E73391FBF3F101F2DB5189B24A
:100EA000FFF7E1B9FDEEE77A40F2E73217EE903A4C
:100EB000303B02FB03F388FB0312D917C1EB62211D
:100EC00001F2E93189B2FFF7CEB940F2F313A1F58F
:100ED000836103FB01F140F2E73391FBF3F101F28F
:100EE000DD5189B2FFF7BFB9648400204C42002075
:100EF000747D0020F0A700201C1E0020A07400209C
:100F0000E8A60020EA3E0020B87F00206084002090
:100F100090E33FF408B501210220FCF7A3FA094B46
:100F20001B7803F00503052B08D000210120FCF7F6
:100F300099FA00210846FCF795FAFEE712F0C2F98B
:100F4000F3E700BF043E0020022828BF022010B4AF
:100F5000084C094B207000EB8002C0EBC20207492D
:100F60005DF8044B013003EB4203C0B20B600CF0A0
:100F7000FFB800BFA07400206A5900205C5900200F
:100F800008B524F09FFDF7F7C7FCBDE8084024F042
:100F900081BD00BF38B5484B5A899989914224BF19
:100FA00000225A81198ADA89914224BF0022DA810B
:100FB000DA78CAB1072A41496AD091F85700404D02
:100FC000012400210A282C709C70D9715DD00C2856
:100FD00007D0002A6CD0DFED3B7A072A0ED00A2812
:100FE00062D0DFED397A09E0344A92F857000A28D6
:100FF00056D00C285BD1D979DFED347A344C9FED93
:10100000350AA278002918BFF0EE407A062A04D8E3
:10101000314901EB820191ED0F0A217979B1013A51
:10102000032A0BD8F7EE007A87EE800A2AF0A4FC98
:101030002388984228BF1846208038BD38BD9B7849
:101040001F4A07EE103A1178B8EEC77A67EE277A92
:1010500007EE101AB8EEC77A27EE277AB4EEC70A61
:10106000F1EE10FAEADD80EE277AFDEEC77A17EE90
:10107000903A102BA8BF1023012BB8BF0123DBB27D
:101080008B4238BF0B46137038BDDFED147AA4E7EE
:1010900091F857000A2803D00C28ACD0D9799AE7E8
:1010A000D979DFED0E7AA9E7DFED0D7AA6E7D979D8
:1010B000DFED047AA2E700BFB479002028A8002061
:1010C000608400206F1203396F12833A0AD7A33964
:1010D000847600206F120338A4E103085304E93832
:1010E0000F506E3A2DE9F047AE4FAF4E24F0EAFCB8
:1010F000BE421ED2DFF83C83DFF83C93444625888D
:1011000062197DB14A450DD2052D0BD9338861880E
:10111000C3F30B03994200F0F3801446258862194B
:10112000002DEFD1716830461436FCF7FCFDBE424D
:10113000E4D39E4A1378A3F1170102290FD99C49E1
:1011400011F83300002840F0FD80D80001444978B0
:1011500029B1984911F83330002B00F01B81964CCF
:101160006378022B84BF002363702378022B84BF33
:1011700000232370914B9A78042A00F0028132B93F
:101180001A88B2F5F07F84BF4FF4F0721A808C4D4C
:101190008C4A2B681A40002A00F0FF80D80700F123
:1011A000EB80590400F1E3801A0700F1DB809B0417
:1011B00000F1D180844D2B685A8C998C914224BFC8
:1011C00000225A84FFF7E6FE22F09EFE10B97F4807
:1011D0000AF038FB4FF40070FCF7DCFD4FF40030F0
:1011E000FCF7D8FD4FF40010FCF7D4FD4FF0007071
:1011F000FCF7D0FD4FF08060FCF7CCFD6378022B4C
:1012000006D8734A734903EB430302EB83030B6075
:101210002378022B07D803EB83016F4AC3EBC1038A
:1012200002EB43032B6015F03DFD002130226B489B
:101230002CF0AFFC286813F009FF694B2D6803F10F
:10124000500102E0043399427AD01A78002AF9D189
:101250009C78D8788442F5D26249634B0A7028465C
:101260001D6016F0BDFB614B614A1E796149624801
:10127000624B1160C825642212FB0652604C406B21
:1012800031F8061C5A60002221809A60DA601A61E7
:101290005A619A61DA6183F8202083F8212008B12D
:1012A0001AF066F9574B9FED585A1B88574A9FED25
:1012B000586A5579574C58495848086006EE903A94
:1012C000F8EEE66A1388C5EE265A07EE103A538800
:1012D0001279C4ED005A07EE903AB8EEC77A504B37
:1012E000F8EEE77A1D725A7227EE067A67EE867A72
:1012F000BDE8F04783ED017AC3ED007A24F0CABB64
:1013000063799B077FF409AF716894F804A03046B5
:10131000FCF709FD3388BAEB133F04D01436BE4204
:10132000FFF4ECAE05E773887068AA1FC3F30B03E4
:101330009A4204F10601A8BF1A462AF013F9EDE714
:10134000012289E7D8000C186468002C7FF4FEAEF7
:1013500017241470FAE63348FCF71CFD4020FCF714
:1013600019FD27E73048FCF715FD2B681FE72F48CC
:10137000FCF710FD2B6817E72D48FCF70BFD2B68D9
:101380000FE79A8AB2F57A7FBFF401AF4FF47A7211
:101390009A82FCE618231370E1E643F008032B6001
:1013A000FCE600BF1006000888010008AC5F0020C2
:1013B000D0070408A0FF0308A07400208476002052
:1013C000C05A0020096000025C590020BC74002053
:1013D000725A00201C4B00206A5900208C2A0020E1
:1013E000B05F002048010020C02A00206442002095
:1013F000C8A70020728400207CA60020947F0020D3
:101400004C630020D0280020C0C9FB48EC240020F9
:1014100017B7D138D42800204C4000203661023D57
:10142000284000200940000201600002092000025B
:1014300008600002024000080080000808B524F09F
:1014400041FBF7F769FA24F025FBFFF74BFE01207B
:10145000BDE808400BF08CBE38B50C4C0C4DAC42CE
:1014600006D2616820461434FCF75DFCAC42F8D328
:10147000084A094B094C1460002209491A705A7035
:1014800008480860BDE838401BF0EEB88801000845
:10149000100600085C590020A07400206A59002042
:1014A0001C4B0020725A002008B5FFF7D5FF24F02E
:1014B00009FBF7F731FABDE8084024F0EBBA00BFAA
:1014C000F0B50C2934D8DFE801F0893333335E33CB
:1014D0003333343333330700048C9689B2F802E097
:1014E0001788734D24F480542404240C0484038C42
:1014F0008488818B23F4005321F4E6411B04090402
:101500001B0C46EA0E06090C43EA063341EA0721A2
:10151000A8429BB2A4B289B200F09E8005F5806516
:10152000A84200F0998092688480818302640384D9
:10153000F0BD048C9589B2F802C0B2F800E05C4FAF
:1015400024F480742404240C0484038C8688818B06
:1015500023F400731B0421F073011B0C45EA0C04F7
:10156000090443EA0423090CB8429BB2B6B241EA2B
:101570000E015CD04F4CA04259D092688680818386
:10158000C2630384F0BD048C9589B2F802C0B2F83E
:1015900000E0474E24F010042404240C0484038C3F
:1015A0008788018B23F0200321F4E6411B04090402
:1015B0001B0C45EA0C04090C43EA041341EA0E2112
:1015C000B0429BB2BFB289B25DD03A4CA0425AD071
:1015D00092688780018382630384F0BD048C9789BD
:1015E000B2F802E01688324D24F001042404240CE1
:1015F0000484038C8488018B23F002031B0421F0F4
:1016000073011B0C47EA0E0709043B43090CA8426F
:101610009BB2A4B241EA060125D005F58065A84237
:1016200021D092688480018342630384F0BDD58910
:10163000148A578A23F4006343EA05254FF6FF33E3
:101640002B40958826F440563C4343EA052346EA5E
:1016500004169BB2B6B290E7158A24F4804444EA9B
:101660008514A4B25FE7D689158A578A23F0080348
:10167000334324F4407496883D4323F004032C4301
:101680003343A4B2CDE7D489158A568A23F0800368
:1016900043EA04134FF6BF741C40938827F4406755
:1016A000354344EA031347EA85079BB2BFB28FE78D
:1016B00000000140000401402DE9F04FC822002144
:1016C00083B08B488B4CDFF850928B4D8B4E8C4FF8
:1016D000DFF848822CF05DFA8A488B49DFF840E257
:1016E000DFF840C200221359834200F0D680B3F1E4
:1016F000804F00F0DD80AB4200F0E580B34200F0A7
:10170000E480BB4200F0E380734500F0E280634573
:1017100000F0E180434500F0E080DFF80CA2534583
:1017200000F0DD800AF5806A534500F0DA800AF5A2
:10173000806A534500F0D780AAF5983A534500F0E7
:10174000D4800AF5806A534500F085800AF5806AE6
:10175000534508BF0D237FD01832B2F5907FC2D118
:10176000644C6A4E6A4F6B4D04F5907802E0183471
:10177000A0456DD0A379002BF9D023794FEA131936
:1017800009F1FF39B9F1030F03F00F03EFD836F871
:10179000190040FA03F2D207E9D54FF0010A0AFA1C
:1017A00003F3013B184029F069FC17F8093018448D
:1017B00015EBC002DBD055F83000DFF870E1217A7C
:1017C00000F13F4303F57E039B0A1EF8033003F04C
:1017D0001F0E5B09032B0AFA0EFA60D0042B69D0A6
:1017E000022B07D1DFF820E1DEF844304AEA030398
:1017F000CEF8443093880093B3FA83F3C3F11F0308
:101800009BB2DA0800EB820203F00703D2F820E073
:101810009B004FF00F0C0CFA03FC2EEA0C0EC2F8E2
:1018200020E0D2F820E001FA03F343EA0E0313624A
:1018300069460023022218348DF804208DF8053003
:101840008DF806308DF8073025F04CFCA04591D17D
:1018500003B0BDE8F08F0C2309EBC3034FF0010A7E
:1018600093F85C3003F01F0B5B09032B0AFA0BFAA9
:1018700009D0042B0CD0022B7FF46EAF4B6C4AEADC
:1018800003034B6468E70B6C4AEA03030B6463E7EA
:101890000B6B4AEA03030B635EE70023DCE7DFF828
:1018A00068E0DEF840304AEA0303CEF84030A1E7B2
:1018B0000123D1E7DFF850E0DEF830304AEA0303D5
:1018C000CEF8303096E70223C6E70323C4E70423AB
:1018D000C2E70523C0E70623BEE70723BCE70823CA
:1018E000BAE70923B8E70A23B6E70B23B4E700BF3A
:1018F000C86D0020AC05040800040040000800404A
:10190000000C0040000001400038024000100408B4
:10191000FC0F040810B00020A4E1030800040140FB
:10192000001000400014004000400140D40F0408A3
:1019300001490248FEF734BA686E002000400140B9
:1019400001490248FEF72CBA406E00200004014015
:1019500001490248FEF724BA406E0020000401400D
:1019600001490248FEF71CBA186E0020000C004026
:1019700001490248FEF714BAF06D0020000400404F
:1019800002494FF08040FEF70BBA00BFC86D00203F
:10199000F0B50468474DA30AAB426ED009D8B3F541
:1019A000801F66D0023DAB4258D14FF0480E012651
:1019B00008E0414DAB4264D00F35AB424FD14FF000
:1019C000C00E04264779B0004FEA970C00295CD07E
:1019D00063460227A5899F4083190CEB43032F43DD
:1019E00003F1040C354DBFB245F8231045F82C2007
:1019F000A781EFF31181502282F31288821905EB3F
:101A0000C202136963B313620433821905EBC20285
:101A1000576917B11F6053690433821905EBC2027D
:101A2000976917B11F6093690433821905EBC202ED
:101A3000D76917B11F60D36904330027CAB21F608A
:101A400082F31188304405EBC000036A5BB9A389B7
:101A500023F001031B041B0CA381F0BDF0BDF0BDFE
:101A600005EB0E03D1E7A3899BB243F00103A381E9
:101A7000F0BD4FF0200E0026A4E74FF0700E0226B6
:101A8000A0E74FF0980E03269CE70223BF0803FA55
:101A900007F7A389094D9BB223EA070387190CEBCB
:101AA000470CA3810CF1040345F82C1045F82320C2
:101AB0009FE700BF0300100041001000C86D002028
:101AC00010B5036883480139834282B089B200F0BF
:101AD000CB80A0F58060834200F0C68000F5804096
:101AE000834200F0B88000F58060834200F0B3804C
:101AF00000F58060834200F0AE80774C188824683F
:101B00006408B4FBF2F4013CA4B282B2B3F1804F9A
:101B10000AD07248834207D000F58060834203D028
:101B200000F58060834202D122F0700292B26C48CC
:101B3000834200F0A28000F58060834200F0A7801D
:101B400022F4407200F56C4092B283421A80D9624E
:101B50001C854FD05F4A93424CD001229A821A884A
:101B600092B242F001021A80B3F1804F00F09980E6
:101B70005A4A934200F0978002F58062934200F047
:101B8000948002F58062934200F0918002F58062B9
:101B9000934200F08E8002F58062934200F08B80C9
:101BA00002F57042934200F0888002F57052934231
:101BB00000F0858002F58062934200F0828002F599
:101BC000806293427FD0A2F5983293427DD002F595
:101BD000806293427BD002F58062934208BF0D225F
:101BE00015D002A84FF0012340F8043D1EF0F0FC90
:101BF00002B010BD0122002119869A821A88394844
:101C000092B242F0010283421A80ADD10A46364BAD
:101C100003EBC20301A893F85D408DF80440012353
:101C200000228DF805308DF807308DF806201EF063
:101C3000CFFC1B2C08D02E2CDAD12C4B019301A801
:101C40001EF0C6FC02B010BD294B019301A81EF086
:101C5000BFFC02B010BD204C18882468B4FBF2F41D
:101C6000013CA4B282B251E71B4C18882468B4FB33
:101C7000F2F4013CA4B282B256E701201A80D96284
:101C80001C8598821A8892B202431A8070E701205C
:101C90001A80D9621C8598821A8892B202431A80EF
:101CA00062E70122B3E70222B1E70322AFE7042291
:101CB000ADE70522ABE70622A9E70722A7E708223E
:101CC000A5E70922A3E70A22A1E70B229FE70C223E
:101CD0009DE700BF00040140C075002000040040E3
:101CE0000010004000000140A4E103082C010001A5
:101CF000190100012C4B98423DD0B0F1804F3CD0EF
:101D0000A3F57C4398423AD003F58063984238D0DB
:101D100003F58063984236D003F58063984234D04F
:101D200003F58063984232D003F57043984230D077
:101D300003F5705398422ED003F5806398422CD05F
:101D400003F5806398422AD0A3F59833984228D0AF
:101D500003F58063984207D003F58063984208BF7B
:101D60000D2202D0002070470C22104B03EBC2035F
:101D700093F85C0070470022F7E70122F5E70222A2
:101D8000F3E70322F1E70422EFE70522EDE706225D
:101D9000EBE70722E9E70822E7E70922E5E70A225D
:101DA000E3E70B22E1E700BF00000140A4E10308E4
:101DB0002DE9F04F2DED028B93B0834620F072F9A0
:101DC000914B1D7825B113B0BDEC028BBDE8F08FAF
:101DD0008E4B1B685905F6D58D4B8E4E1B6863B133
:101DE0008D4A31681368CB1A7C2B06D98B48116059
:101DF00003780133037026F029F8894B1B78002BF8
:101E000072D0884C884AD4F81031ABEB030393426C
:101E100001F2548394F81891B9F1000F35D1DFF82D
:101E20003C82D8F80000FAF7EBFEC0B201280FD9C7
:101E300002287E4F42F066803B78002B42F0B18151
:101E4000D4F81C31ABEB0303B3F57A6F82F0EF8269
:101E5000D4F82031002B47D094F81831C3B9744B13
:101E60001B689B7801211E3B00228B4284F81811CD
:101E700084F82C2142F29682D8F800000221043026
:101E800025F096FF94F8243111E0D4F820315BB3AB
:101E9000D4F8283140F6B732ABEB0303934223D991
:101EA00094F82431002B01F0F986DFF8B081013B72
:101EB000DBB284F82431002B01F02684D4F82071A1
:101EC00094F82C2117F8011B94F82D31D8F8000054
:101ED000C4F820710A44013384F82C2184F82D3190
:101EE000FAF792FEC4F828B1524B37681B7853B109
:101EF000DFF86C81D8F8000028B14F4B1B78013B0C
:101F0000012B41F211844D4B1B7873B1DFF85481E2
:101F1000D8F800304BB13368424C02931A46D4F8DB
:101F20004431D31A632B01F2B281DFF83C8198F877
:101F30000030022B01F08A863C4F97F87430032B57
:101F400001F0CC833E4B1B7873B13E4D2B685BB1E7
:101F5000344CFAF79DFBD4F85031029044F61F62DE
:101F6000C31A934200F23081374B1B78002B7DD18E
:101F7000364B1B7843B12B4CD4F8A03203F5C33356
:101F8000A0339B4581F03E82314B1B78002B3FF400
:101F90001AAF244E2F4C304D06F2C1272068FAF7B5
:101FA0002FFE00283FF40FAF2068FAF721FE2B78B0
:101FB00080465A1E33B120682A70FAF721FE0028A5
:101FC000F2D100E703223946781E2BF0C8FD96F8BF
:101FD000C03296F8C12286F8C38283F47F4383F02F
:101FE000FF039B1A1FFA88F89BB2B8EB132FD5D1C9
:101FF00096F8C222DBB29A42D0D1781E1FF0E6F8E2
:102000002B7818442870C9E72F680020D879002061
:10201000A8A40020607C0020C8A60020C4A6002040
:1020200056800020FC2400203F0D030020000020EB
:1020300078A6002058800020608000206880002062
:102040007080002074800020E0800020F18000205B
:102050007A800020808000208480002074A60020E8
:10206000ACA400206CA600207EA30020484C22785F
:10207000A2B1484B9B7A53B1FAF70AFB464B1B6857
:10208000C31AA3F57A73B3F5FA6F07D82278434BD6
:1020900043491868FAF780FD00232370414CD4F8B7
:1020A000983203F5C333A0339B45FFF461AF3E4D37
:1020B000C4F898B22B78002B41F035873B4D2B7834
:1020C000002B41F08D8694F89C2239498D5CEA07FB
:1020D00001F1E787AF0701F1A787680702F12B80BD
:1020E0002A0748D5334B344F0B9312AA1146A3F15C
:1020F0003D0241F8202D0020A3F140020D4603F8D7
:10210000400C0391022311215170937028463968C5
:10211000F6F728FE28467968F6F724FEFB8927495A
:1021200003EBC3039B00053381FB0321DB17C3EBE8
:10213000A101284689B2F6F72DFE3B8A03EB830303
:10214000590089B22846F6F725FE1D4B039D1B78E2
:102150009B0743BF398901F57A7189B24FF47A71CF
:102160002846F6F717FE0A9B3A7D591C0A91284625
:102170001A701FF027FF134A94F89C32117801332C
:1021800093FBF1F201FB123384F89C32F0E600BFBE
:1021900048800020F0940020005F0020E4800020B0
:1021A00008800020FC240020E8800020E980002036
:1021B000EC80002008800020F0A60020676666669C
:1021C000ECA60020F080002094F85631002B41F05E
:1021D0008A85DB4B1A6802F00803002B4AF60B4095
:1021E00048F603414BF60F4349F6074704BF034641
:1021F0000F4612F0040F4FF0190118BF1F4690064A
:1022000084F8561103D547F4804747F02007CD4B9B
:102210005A79C7F30909002A42F031819B79002BD2
:1022200042F03D82984664204FF0FF3A4FF0000C98
:102230000A970B97ADF834C0CDF83AC0CDF83EC040
:10224000CDF842C0CDF83090ADF83680ADF838A06A
:102250008DF846000AAF0FCFDFF800E384F805C021
:10226000AEE80F0097E80F00AEE807002EF8023B3B
:1022700071464FF0010C1B0CFE271F20C82201F8ED
:102280001E39A770A27184F807C0E07094F8660147
:10229000207180F0F10383EA0313DAB2130983F0AB
:1022A000E70343EA022383EAC2031BB283EA031271
:1022B000D2B2C3F3072383EA121343EA022383EA69
:1022C000C2031BB283F0C80282EA0212D2B2C3F385
:1022D000072383EA121343EA022383EAC2031BB2F1
:1022E00083EA0C0787EA0717FFB2C3F3072282EAE3
:1022F000171242EA072200EB0C0382EAC7070EEB33
:102300000C0084F86631278011F8013B7B4083EA9A
:102310000313DBB21A0982EA172242EA032282EA95
:10232000C3031BB29FB281422780EDD183F07C03AF
:1023300083EA0313DBB24FEA131E8EEA172E8EEAEE
:10234000032E8EEAC30E0FFA8EFE1FFA8EF9DFF807
:1023500010C2A4F800905FFA8EFE4FEA192984F8A3
:10236000289084F827E00CF5C77804F1220ADCF8FD
:102370000000DCF80410DCF80820DCF80C304746DC
:102380000FC70CF1100CD445B846F0D1DCF80000B2
:1023900038606D4F9CF8043088F8043007F1270846
:1023A00084F8B5E184F8B69117F8011F2868FAF7A8
:1023B0002BFCB845F8D194F85731002B41F08E84AE
:1023C0006249326809780A2084F85701002901F02F
:1023D00021865F4F01293888069042F257810229F1
:1023E000B7F802E002F06580B8880590032902F092
:1023F0005D81F8880490042902F06E8105293889EE
:1024000002F065810629B7F80A9002F05C8107297D
:10241000B7F80C8002F05481FB89039394F866119D
:102420000A920B4683F0300282EA0212D2B21709F6
:102430004849079387F07A0747EA022709882371FA
:1024400087EAC202444FC1EB012187FB013A069B98
:102450004FF0000C63F30F0C059B6EF31F4C4FF015
:10246000000E63F30F0E049BCDF82CC012B28A4409
:102470000027C91763F31F4EC1EB6A2A039BCDF8EF
:1024800030E082EA021160F30F070020C9B268F35E
:102490000F00C2F3072269F31F4782EA111263F3A8
:1024A0001F404FF000090D978DF83DA00E908DF85C
:1024B0003C9042EA01220DF1280C82EAC107BCE8F7
:1024C0000F003FB287F0C80888EA0818DFF88CE0F0
:1024D00084F805905FFA88F8C7F30727AEE80F0085
:1024E00087EA181747EA08239CE8030083EAC80331
:1024F0001BB283F023024EF8040B82EA0212D2B21E
:10250000C3F30723079F83EA1213704643EA0223AB
:1025100083EAC20207F1010C20F814194FF02308D6
:102520001621FE27C82384F866C1228084F807801C
:102530000EF1020EA770E170A371114612E000BF08
:10254000E8A60020D4A600208B2600207CA2002034
:10255000607F0020887F0020030820800425002061
:10256000FE24002010F8013B4B4083EA0313DBB24A
:102570001A0982EA112242EA032282EAC3031BB249
:1025800099B270452180EDD183F0F40383EA0313FF
:10259000DBB24FEA131E8EEA112E8EEA032E8EEA6C
:1025A000C30E0FFA8EFE1FFA8EF8CA4FA4F80080F1
:1025B0004FEA182C5FFA8EFE84F81EE084F81FC0E4
:1025C0007968BA683868FB6807F5C778A8E80F002B
:1025D00038697969BA6904F28F17A8E8070004F22C
:1025E000AD1884F8ADC184F8ACE117F8011F286874
:1025F000FAF70AFBB845F8D194F85A31002B41F0AC
:102600007783B54B1B681922990684F85A2140F14B
:10261000FC82B24BB24F1B789A0741F128873B7D71
:10262000042B8CBF4FF003084FF00208FAF730F884
:102630003B8A3A890A9003EB83035B00ADF8423092
:102640004FF47A703B680C93F98997F814E07B6833
:102650008DF8448000FB02F24FF0000C0AA84FF006
:10266000FF398DF845E0CDF82CC0CDF83C900E92A6
:102670000D93ADF8401080460390B8E80F00DFF8E6
:1026800070E2AEE80F0098E80F00AEE8070072466F
:10269000182122F81C39E17194F8661184F805C0FC
:1026A00081F0780383EA0313D8B2030983F0F603B9
:1026B00043EA002383EAC0031BB283EA0310C0B2DB
:1026C000C3F3072383EA101343EA002383EAC0031A
:1026D0001BB283F0C80080EA001C5FFA8CFCC3F3D5
:1026E000072080EA1C1040EA0C2080EACC0000B2EF
:1026F00080F0180383EA0313DBB2C0F3072080EAFB
:10270000131040EA032080EAC30301F101081E20F0
:102710004FF0FE0C4FF0C809E0700EF1020E21716F
:1027200084F86681238084F802C084F806901846F5
:1027300012F8011B414081EA0111C9B20B0983EA79
:10274000102343EA012383EAC10109B288B272452A
:102750002080EDD181F0180181EA0111C9B20A0986
:1027600082EA102383EA012383EAC1031BB29AB2EF
:10277000DFF860A12280DBB2120A0592049384F88C
:10278000272084F82630D6460AF5C77904F12208B6
:10279000DEF80000DEF80410DEF80820DEF80C3069
:1027A000CC46ACE80F000EF1100EC645E146EFD165
:1027B000DEF80000CCF800009DF81030DFF834811E
:1027C00084F8B4319DF8143084F8B531C14619F855
:1027D000011F2868FAF718FA424B4B45F7D1F9F771
:1027E00057FF414B414AB3F90410B7F808E03B6882
:1027F0000B930A907B680C9382FB01274FF47A704D
:10280000C9174FF0000C00FB0EF0C1EBA701DDF87B
:102810000CE0ADF83CC0ADF83EC0ADF840C0ADF83E
:1028200042100D900E90BEE80F00314F84F805C0A5
:102830000FC79EE807004FF0210C87E807001C2314
:10284000C8224FF0FE0EE37084F807C084F802E05F
:10285000A27194F86611217181F06A0383EA03136F
:10286000DAB2130983F0D50343EA022383EAC203F1
:102870001BB283EA0312D2B2C3F3072383EA121313
:1028800043EA022383EAC2031BB283F0C80282EA4E
:102890000212D2B2C3F3072383EA121343EA0223DC
:1028A00083EAC2031BB283EA0C0282EA0210C0B2BE
:1028B000C3F3072282EA101242EA0022013182EABF
:1028C000C0020C3784F866112280A7F11C01104663
:1028D00012E000BFFE240020E8A60020ECA60020A5
:1028E000F0A60020B1260020CCA600206766666610
:1028F000042500208B26002011F8013B434083EA89
:102900000313DBB21A0982EA102242EA032282EAA6
:10291000C3031BB298B2B9422080EDD183F06803A3
:1029200083EA0313DBB2190981EA102282EA032247
:1029300082EAC3031BB29AB2DB4F2280DBB24FEABA
:10294000122C049384F8243004F1220384F825C067
:1029500007F5C7790593FB6838687968BA68CE4689
:10296000AEE80F00059B10379F42F146F3D13B883C
:10297000AEF800309DF81030CC4F84F8B231C1462B
:1029800084F8B3C119F8011F2868FAF73DF94F45DB
:10299000F8D194F866C1C64AC64F84F804C08CF0DA
:1029A000EB0383EA0313D9B20B0983F0C50343EAAF
:1029B000012383EAC1031BB283EA0310C0B2C3F34D
:1029C000072181EA101141EA002181EAC0010CCA05
:1029D00009B281F0C80E8EEA0E1E5FFA8EFE4FF02D
:1029E00000090A92C1F30721039A0B93CDF83090A6
:1029F00081EA1E1343EA0E2307CA83EACE031BB201
:102A000083F0310E87E807008EEA0E1E5FFA8EFE15
:102A1000C3F3072383EA1E1343EA0E2383EACE039C
:102A200094F808E0607AA17AE27A277B84F805902E
:102A30001BB28EEA030E8EEA0E1E5FFA8EFEC3F301
:102A4000072383EA1E1343EA0E2383EACE031BB255
:102A5000584080EA0010C0B2C3F3072383EA101382
:102A600043EA002383EAC0031BB2594081EA011004
:102A7000C0B2C3F3072181EA101141EA002181EAC3
:102A8000C00109B24A4082EA0212D2B2C1F307235E
:102A900083EA121343EA022383EAC2031BB25F40B4
:102AA00087EA0717FFB2C3F3072383EA171343EA42
:102AB0000723607BA17BE27B94F810E094F81190EF
:102AC00083EAC7031BB2584080EA0010C0B2C3F3C8
:102AD000072383EA101343EA002383EAC0031BB2EF
:102AE000594081EA0111C9B2C3F3072383EA1113E4
:102AF00043EA012383EAC1031BB25A4082EA02126D
:102B0000D2B2C3F3072383EA121343EA022383EA10
:102B1000C2031BB28EEA030E8EEA0E1E5FFA8EFE11
:102B2000C3F3072383EA1E1343EA0E2383EACE038B
:102B30001BB289EA030989EA09195FFA89F9C3F323
:102B4000072383EA191343EA092383EAC903A17C13
:102B5000E27C594F1BB2594081EA0111C9B2C3F35B
:102B6000072383EA111343EA012383EAC1031BB25B
:102B70005A4082EA0212D2B2C3F3072383EA121345
:102B800043EA022383EAC2031BB283F0270989EADE
:102B90000912D2B2C3F3072989EA121949EA0229B4
:102BA00089EAC2090FFA89F91FFA89F20CF10103C7
:102BB0004FEA122E5FFA89F931204FF0FE0C0C21FA
:102BC00084F86631C8232280E07184F802C0E17085
:102BD000A37184F8149084F815E0DAF80410DAF898
:102BE0000820DAF80C30DAF80000BAF810C00FC785
:102BF00027F803CB84F8A3E184F8A29118F8011F09
:102C00002868FAF701F84745F8D194F85EC1BCF19D
:102C1000000F41F07880294B94F866E1B3F9001079
:102C2000B3F90220B3F904309FED256A214F84F8EF
:102C300005C007EE103A33680A938EF06A0383EA00
:102C4000031306EE901AD9B20B0983F0D50343EAB9
:102C5000012383EAC1031BB283EA03115242C9B2C2
:102C600007EE902AC3F3072383EA111343EA0123F3
:102C7000F8EEE77AF8EEE66AB8EEC77A83EAC103BF
:102C80001BB267EE867A66EE866A27EE067A002029
:102C900083F0C808CDED0C7ACDED0B6A8DED0D7A81
:102CA0000E900F900EE000BFFE240020AF26002003
:102CB000846C0020042500208C260020CCA6002057
:102CC00088C3E43A109088EA08160DF12809F6B294
:102CD000C3F30728B9E80F0088EA161848EA06285F
:102CE00088EAC6080FFA88F80FC788F01E0699E828
:102CF000070086EA0616F6B2C8F3072383EA16131E
:102D000043EA062387E8070083EAC606C8214FF096
:102D100005084FF01E0CFE231C200EF10102A171CC
:102D200084F85E8184F807C0A370E070A7F11001F9
:102D300084F804E00C37268084F8662111F8013B02
:102D4000734083EA0313DBB21A0982EA162242EACD
:102D5000032282EAC3031BB29EB2B9422680EDD1A0
:102D600083F0270383EA0313DBB24FEA131E8EEAD4
:102D7000162E8EEA032E8EEAC30E0FFA8EFE1FFA6F
:102D80008EFCD94FA4F800C05FFA8EFE4FEA1C2CCF
:102D900084F825C084F824E007F5C77804F12209F7
:102DA00038687968BA68FB6846460FC610374F45E1
:102DB000B046F5D1CD4E3B88A8F8003006F1240787
:102DC00084F8B2E184F8B3C116F8011F2868F9F756
:102DD0001BFFB742F8D194F85F81B8F1000F40F0C3
:102DE0008C87C34B1B6805229B0684F85F2141F149
:102DF0000B81C04BDFEDC06ADA891B8907EE902A90
:102E000007EE103AF8EEE77AB8EE477A67EEA67A60
:102E100094F866C1B94BBA4AB3F90410B2F9062066
:102E2000B84EB948CDED0B7A8CF0220383EA031338
:102E3000DFB23B0983F0590343EA072383EAC70360
:102E4000B2F5FA6F1BB2A8BF4FF4FA6283EA031718
:102E5000FFB2B2F57A7FC3F3072383EA1713B8BF33
:102E60004FF47A724FF0640E43EA0723A2F57A72A8
:102E70000EFB02F283EAC70786FB02E680FB01E055
:102E80003FB2C917D217C2EBA612C1EBA0034FF095
:102E900000090AA987F0C8068DED0C7AADF83A2032
:102EA000ADF83830CDF82890CDF834908E4686EACB
:102EB0000616F6B20391C7F30727BEE80F0087EAAC
:102EC000161747EA062787EAC606904FDEF800E0A5
:102ED00084F804C00FC736B286F04A0383EA0313AE
:102EE000DBB2C6F3072181EA13113A4641EA032116
:102EF0000CF1010C81EAC303142042F810E9FE260C
:102F00004FF04A0E002184F866C14FF0C80CE07003
:102F10002380043784F807E0A670617184F806C046
:102F2000184612F8011B414081EA0111C9B20B0990
:102F300083EA102343EA012383EAC10109B288B27C
:102F4000BA422080EDD181F0140181EA0111C9B2A9
:102F50004FEA111E8EEA102E8EEA012E8EEAC10E65
:102F60000FFA8EFE1FFA8EF6DFF87CA126804FEA5C
:102F7000162C5FFA8EFE84F81CE084F81DC0DAF887
:102F80000410DAF80000DAF80820DAF80C30BAF8A1
:102F900018900AF5C7770FC7DAF81000DAF814109E
:102FA00003C704F28F16A7F80090374684F8ABC128
:102FB00084F8AAE104F2AB1917F8011F2868F9F7A1
:102FC00023FEB945F8D1524B524A1B781278013B87
:102FD00012F00100DBB214BFC0214021172B03D82F
:102FE0004D4A134493F830804C4B1A8897071ABF08
:102FF000002341F01001012312F4027F18BF0223C5
:1030000012F0100F18BF062312F0200F18BF102364
:10301000002841F002824FF0030C94F866E10A9315
:103020008EF0460383EA0313DAB2130983F09203A6
:1030300043EA022383EAC2031BB283EA0310C0B24D
:10304000C3F3072282EA101242EA002282EAC00297
:1030500012B282F0C80787EA0717FFB2C2F307224D
:1030600082EA171200238DF82FC0032042EA072CB2
:10307000039A8DF82C808DF82D308DF82E108DF858
:10308000300007CA8CEAC70C0FFA8CFC1F4FE371A3
:103090008CEA0C1803C75FFA88F8CCF3072C8CEA8B
:1030A000181C4CEA082181EAC80894F808C03A7054
:1030B0000FFA88F88CEA080C8CEA0C1C5FFA8CFC7E
:1030C000C8F3072282EA1C1242EA0C22607AA17A33
:1030D00094F80B80637182EACC0212B2504080EA0D
:1030E000001C5FFA8CFC1BE0FE2400208B260020D5
:1030F000E8A60020F0A600200AD7233CCCA600209A
:10310000607F0020D34D621067666666042500204C
:10311000AC5F0020747D00206CE203088A7F0020F1
:10312000C2F3072080EA1C1040EA0C2080EACC00A1
:1031300000B2414081EA0111C9B2C0F3072282EA1C
:10314000111242EA012282EAC10212B288EA02089E
:1031500088EA08185FFA88F8C2F3072282EA181290
:1031600042EA082294F80CC0607BA17B84F804E05A
:1031700082EAC80212B28CEA020C8CEA0C1C5FFADA
:103180008CFCC2F3072282EA1C1242EA0C2282EA79
:10319000CC0212B2504080EA0010C0B2C2F3072243
:1031A00082EA101242EA002282EAC00212B25140C0
:1031B00081EA0111C9B2C2F3072282EA111242EA7E
:1031C000012282EAC102E17B94F8108013B281EA05
:1031D000030282EA0212D2B2C3F3072383EA121374
:1031E00043EA022383EAC2031BB288EA030282EAAB
:1031F0000212D2B2C3F3072383EA121343EA022373
:1032000083EAC2031BB283F0320282EA0212D2B214
:10321000C3F3072383EA121343EA022383EAC203B8
:103220001BB29AB24FF0FE0C0920C8210EF1010E1C
:10323000DBB284F802C04FEA122CE070A17184F86E
:1032400066E1228084F812C06374DAF80000DAF8CC
:103250000410DAF80820BAF80C9007F5C07EAEE842
:10326000070007F5C8778EF80280AEF8009084F862
:10327000A0C184F89F3116F8011F2868F9F7C4FC33
:10328000B742F8D1029BC4F85031FEF76DBEDFF8AB
:1032900024A27C4FDFF82092412024F035FDBAF9BA
:1032A000023087FB0320DB17C3EBA00080B224F0C1
:1032B0000FFDBAF9003087FB0320DB17C3EBA0003A
:1032C00080B224F005FDBAF9043087FB0320DB1738
:1032D000C3EBA00080B224F0FBFC99F80010D8F8F2
:1032E0000000F9F791FC94F848A11AF0010700F0EA
:1032F0001085654B1B689A0672D5644B644F1B782A
:103300009B0741F14B803B7D042B8CBF4FF0030AA0
:103310004FF0020A472024F0F7FC386824F0A4FCA0
:10332000786824F0A1FCFB895A4AD8F80000A2FB77
:103330000323C3F3471319460393F9F765FC3A894E
:1033400099F80010039B64204B4000FB02F089F8C1
:10335000003024F089FC3F7DD8F800004AEA870756
:10336000FFB23946F9F750FC99F80030D8F8000060
:103370005F40394689F80070F9F746FC94F848A197
:10338000BAF1000F2CD1444F4F2024F0BDFC386817
:1033900024F06AFC786824F067FC504624F064FC52
:1033A0000121D8F80000F9F72FFC384A99F80030CD
:1033B0001778D8F8000007F00107394683F00103B9
:1033C00089F80030F9F720FC99F80030D8F80000AF
:1033D0005F40394689F80070F9F716FC94F848A167
:1033E000029B2E4AC4F844310AF10103DBB2A2FB6E
:1033F0000312D20802EB8202A3EB420384F84831A5
:10340000FEF793BD94F8A432254AC4F8A0B202EBAB
:103410008302926C42B312AD04F2AB23214E45F805
:10342000203D002104F2BD2331800B938021152320
:10343000A52784F8AA32284684F8A91284F8A8722D
:10344000904728463188F5F7CBFC0A9D164804F5CD
:103450002A716D1A152DA8BF15252A4628F082F865
:10346000124A94F8A4321570114A013382FB0312F8
:10347000A2EBE37202EB42029B1A84F8A432FEF73D
:1034800083BD00BF67666666E8A60020ECA6002044
:10349000F0A600201F85EB51846C0020CDCCCCCC55
:1034A0006CE20308C47F0020C05D0020D55D0020D1
:1034B00056555555CCA6002070A60020C24AC34BD5
:1034C000D4F8141130681B8892F80BE0C04A401AF7
:1034D0004FF47A71DFB201FB0EF11B0A9777177573
:1034E00088424FF00007D37753759770177180F0BB
:1034F000F784B849DFF808C30B688968B648B74F46
:10350000007897F814A08CFB03E8DB178CFB01EC28
:103510004FEAE17EC3EBA80111770912CEEBAC0EA6
:103520005177F4214FEA2E2C82F820E091764FF06B
:10353000010E302182F81BE082F82210A84B82F89D
:1035400021C04FF0750E782182F823E082F8241014
:10355000820783F81AA040F1BF84D7F800C0A14ABF
:10356000D7F804E0A04882FB0C194FEAEC7182FB0B
:103570000E82C1EBA9514FEAEE79C9EBA25200FBD2
:1035800001C9029200FB02E009EB4909974A4FEAA0
:10359000490982FB0982049200EB4000934A4000F3
:1035A000039082FB0008049A9014029A0490F88910
:1035B0003F8902EB820200EBC00002EB820207F5BA
:1035C000FA770692BAF1050F4FEA80021FFA87FADE
:1035D0000398049F029201EB81014FEAE97201EB2B
:1035E000810105914FEAE071A7EB0200804F83F85B
:1035F00015A0024607FB1292059F4FEAA84840B269
:1036000000EB8709A8EB0100794F0399804607FB7F
:103610001010069F77494FFA88F84FEADC7C4FEA92
:10362000DE7E83F809C083F80EE0DFF8D8C108EB2E
:10363000870E029F81FB07814FEAE778BCF8007094
:103640000397C8EBA1116C4F029187FB021887FB0F
:1036500000170299DFF8B0C11FFA89F91FFA8EFE30
:103660004FEAE2724FEAE070C2EB681883F80A9002
:10367000C0EB671283F80FE04FEA19274FEA1E29C3
:10368000C1F3072E0399BCF80000DF7283F8109095
:103690004FEA222783F80C805A749DF80820DA71CB
:1036A0004FEA282C4FEA1A2A4FEA112934BF4FF06B
:1036B00032084FF033089DF80C2083F80DC09F743A
:1036C00083F816A083F808E0DA7483F8149083F87E
:1036D0001B801877C4F810B1FEF79CBBDFF82C9163
:1036E000D9F80000F9F77CFA00283EF42BACD9F8A1
:1036F00000000121F9F770FA0222002387F87420F4
:1037000088F80030FEF71EBC94F82C1194F82D3187
:10371000D8F800004A1C013384F82C2184F82D319C
:10372000F9F772FAFEF7DEBB344CDFF8E4904FF0A5
:10373000000A0BE01B2B00F09F820D2B00F079811B
:103740004FF0010389F80130D8F80000F9F758FA72
:1037500000285FD0D8F80000F9F74AFA83B27E2B30
:1037600032682AD099F801100029EDD194F82E2161
:10377000002ADFD07D2B00F0648294F83CE1BEF19A
:10378000000F04D080F02003DBB284F83C11511C00
:10379000C9B22244092984F82E1182F8303100F090
:1037A00044820829D0D8B4F83A21134403EB1323F8
:1037B00003F0FF03A4F83A31C6E784F82EA184F899
:1037C0002FA189F801A0BFE7F07D0020E87D00204F
:1037D00088800020B4A40020ECA60020F0A60020E1
:1037E000B48000206BCA5F6B806967FF83DE1B4378
:1037F00040420F00D34D62101F85EB51FC24002086
:1038000067666666D46C0020D66C00200CA400208D
:103810002000002094F83D3133B194F8313184F820
:103820003D01302B00F0D78594F82F21BA4BBB49CE
:10383000DFF818A3DFF8189302954FF0010E9046B9
:103840004246002A00F05B833268D21B012A00F254
:103850001F8294F83E21002A40F0348294F83FC140
:1038600033F81C00F0B984F83FE10A689506E7D503
:103870009AF800209007E3D5A94FAA49FA89029D3A
:103880004FF4F36303FB02F381FB0321DB17C3EB6C
:1038900061114FF4036024F071FA002384F82F3192
:1038A000FEF731BB0CF1010C5FFA8CFCB0F5E06F58
:1038B00084F83FC100F09A801BD8B0F5047F00F077
:1038C000498136D8B0F5887F00F0D380B0F5007F0D
:1038D00000F0B880B0F5807FB2D10A685207AFD54A
:1038E0000021029D24F04AFA002384F82F31FEF7CC
:1038F0000ABBB0F5026F00F05E816CD8B0F5E46FE2
:1039000000F08480B0F5006F00F0DD80B0F5E26F6C
:1039100096D1854B029DDA6B998A642303FB02F3EF
:1039200093FBF1F124F02AFA002384F82F31FEF7FB
:10393000EABAB0F5826F00F05581B0F5C06F00F0C3
:103940002981B0F5806F7FF47BAF94F84031029D00
:103950000133DBB2032B00F2AF8142F2107184F825
:10396000403101FB03F1714B1B88002B40F0A28119
:1039700001316F4B1B78DB076E4B1B8848BF04314E
:10398000DF0748BF0A31980748BF14311A0648BFFD
:103990002831DF0548BF2831580748BF64311A076E
:1039A00048BFC8319F0548BF01F5C871980648BF98
:1039B00001F57A71DA0648BF01F5FA615F0648BF82
:1039C00001F57A614FF4806024F0D8F9002384F87F
:1039D0002F31FEF798BAB0F5046F1CD0B0F5116F17
:1039E00056D0B0F5036F7FF42BAF3EE74E4B029DF0
:1039F00090469A6B998A642303FB02F393FBF1F1DF
:103A000024F0BCF984F82F81FEF77DBA464B029D65
:103A100090461A6CEEE7484B029DB3F9041001EB97
:103A200081019046490024F0A9F984F82F81FEF71E
:103A30006ABA4FF0010184F82E1184F83031A4F8ED
:103A40003A2181E699F80620002A3FF4F9AE3B4B73
:103A50003B491B68029D81FB0321DB17C3EBA101DE
:103A60004FF4007024F08AF9002384F82F31FEF718
:103A70004ABA0A6852077FF5E3AE00214FF4887016
:103A8000029D24F07BF9002384F82F31FEF73BBA26
:103A900099F80520002A3FF4D3AE2A4A107800286E
:103AA0003FF4CEAE284B029D1B8803EB83035900E5
:103AB00091FBF0F14FF4116024F060F9002384F8D9
:103AC0002F31FEF720BA0A6895067FF5B9AE9AF84D
:103AD000002090077FF5B4AE1CF0010F029D104F3F
:103AE000104900F068847A6882EAE273A3EBE2731B
:103AF00003EB5303A1FB0331C908002AACBF41F01B
:103B0000004141F040414FF4006024F037F90023B8
:103B100084F82F31FEF7F7B96CE20308E8A600201D
:103B2000F0A600201F85EB517CA60020B87F002066
:103B3000747D00208A7F0020CCA60020B4A4002041
:103B400067666666FE7D0020E87D0020ECA600200A
:103B5000D4A6002099F80520002A3FF471AEC64A89
:103B6000107800283FF46CAEC44B029D5B7B002BA9
:103B700000F08184C24B1B8893FBF0F000EB8000C7
:103B800041004FF4047024F0F9F8002384F82F3139
:103B9000FEF7B9B999F80620002A3FF451AEB94BA7
:103BA000029D99684FF4C06024F0E8F8002384F87F
:103BB0002F31FEF7A8B90D68AD067FF541AE9AF832
:103BC00000C01CF0020F3FF43BAEAF4F029D3B899B
:103BD0006421904601FB03F124F0D0F884F82F8192
:103BE000FEF791B90A68900640F10181A74BA64FF4
:103BF0001878397D029D00F00203002B0CBF0023D2
:103C00004FF47A7340F6B83208BF4FF4FA6210F0FE
:103C1000010F18BF134619444FF4826024F0AEF828
:103C2000002384F82F31FEF76EB9B4F83A21C2F1BF
:103C3000FF0293427FF484AD4FF0010384F83D31DD
:103C40007EE54FF0010384F83C317DE5F8F720FD77
:103C50008F4B1B68C01A40F6B833984200F2588167
:103C6000DFF858A29AF804303A2B00F0C7820023FC
:103C700088F80030FEF766B9D8F80000F8F7C0FF02
:103C800000287FF45DAD4FF0010384F82F315BE530
:103C90000023029D84F82F31FEF735B9C4F8203196
:103CA00084F81831DFF8188224F0B6F894F824313B
:103CB000FEF7FDB802315CE6012384F8403142F2A0
:103CC000107150E67349029D062023F041FE002347
:103CD00084F83E0184F82F31FEF715B9013B84F8D2
:103CE0005731FEF789BC013B84F85631FEF763BBC0
:103CF000013B84F85A31FEF788BF08F1FF3884F899
:103D00005F81FFF7BFBA0CF1FF3C84F85EC1FFF79B
:103D100062B8614B1B88D80513D4D90600F17B83A8
:103D20009A0600F1DA83580600F1DC83190700F1E6
:103D3000DB83DA0700F1EC8313F0020F0CBF0427DA
:103D40000C27564B564A1B78D27803F001030AB170
:103D500043F002035320039323F0D6FF484A12880E
:103D600002EB820202EB8202900080B223F0B0FFED
:103D7000002023F0ADFF4B4A4B491288D8F80000D1
:103D8000C2EBC212520081FB023111444FEAE27AC7
:103D9000CAEB612A5FFA8AFA5146F8F735FF99F8BB
:103DA0000020039BD8F800001F438AEA020A002182
:103DB00089F800A0F8F728FF3946D8F80000F8F78E
:103DC00023FF99F80030D8F800007B40DBB2194699
:103DD00089F80030F8F718FF94F848A1FFF7D0BA37
:103DE00032493A2023F0B4FD2870FEF7C1B8304ABA
:103DF0001268120600F1F782204A127B002A3FF473
:103E00001FAD94F84111029D032900F28383DFE87E
:103E100001F059281902274B1B6859799A79DB79E7
:103E200001F1407101EB022101EB0341002384F811
:103E300041314FF4826023F0A1FF002384F82F3139
:103E4000FEF761B81C4B1A68137A507992781B04FC
:103E500003EB002313444A1C84F8412103EB016166
:103E6000E7E7154B1A68D379107952781B0403EBF6
:103E700000231344EFE700BFFE7D0020F07D00200B
:103E8000E87D0020B4A40020F0A60020ECA60020CD
:103E900084A30020757D03088A7F0020747D0020A4
:103EA000947F0020887F00200308208025200308BD
:103EB000D87900201C4B00205C5900206CA3002006
:103EC00074A60020BA4B1A689379D07812781B0434
:103ED00003EB00231344BEE72D22DA76FFF7FABB8B
:103EE000B44B31681B78C4F81411013B012B3FF629
:103EF00000AB1021022391701371FFF7FABA029DF3
:103F0000FEF701B823F078FF01233B70FDF7A0BF57
:103F1000A94AB2F84A3100210133A2F84A3188F89F
:103F20000010FEF70FB8A54EA54B00930024A6F194
:103F30003F01A44BA44A089106F8404CA3490996B6
:103F40000AA8F5F725F8089E731C08933470089B9F
:103F50002922591C08911A70089BEA22591C0891C1
:103F60001A70089BC822591C08910AA81A7026F0DA
:103F7000BBFB471C0AA93A46089827F0F3FA089AAF
:103F8000D31901330893D455089B5A1C08921C700E
:103F9000089B5A1C08921C70089B5A1C08921C70A3
:103FA000089B5A1C08921C70089B5A1C08921C7093
:103FB000089B5A1C08921C70089B5A1C08921C7083
:103FC000089B5A1C08921C70089B5A1C08921C7073
:103FD000089B5A1C08921C70089B5A1C08921C7063
:103FE000089BFF22591C08911A70089B01229918FE
:103FF00012A808911A7050F8283D9B1B33701DF0D1
:10400000E1FF2C70FDF7B4BFDFED717AB0EE677A97
:10401000FEF7FEBE884689460846049105918E4605
:1040200006910391FEF7FAB9644A6A4B0B9212AEFD
:10403000A2F13D0046F8200D1988674FA2F1400318
:1040400000204FF00A0E02F8400C082283F801E02D
:1040500030469A70F4F79EFE3B686049DA1781FBA0
:104060000313C2EBA30399B23046F4F793FE0CF0AE
:10407000BDF8BF680A9B3A0C591C0A911A700A9B3A
:104080003A0A591C0A911A700A9B5A1C0A921F700C
:104090000A9B5A1C0A92187030461DF093FFFEF7D7
:1040A0001CB84F4F9FED4F8AB7F9022043480B9041
:1040B00007EE902AF8EEE77A12AE67EE887AA0F162
:1040C0003D01FDEEE77A46F8201D00F8403C08234C
:1040D000CDED027A00F83F3C1E23BDF8081000F831
:1040E0003E3C3046F4F756FEB7F9003007EE903A02
:1040F000F8EEE77A304667EE887AFDEEE77ACDEDA6
:10410000027ABDF80810F4F745FEB7F9043007EE5F
:10411000903AF8EEE77A304667EE887AFDEEE77A75
:10412000CDED027ABDF80810F4F734FE30461DF0EC
:1041300049FFFDF7CFBF2C4A204B12680B93A3F128
:104140004007002103F8401C2123D100BB7040F13F
:10415000B88126490326264B1B885A0500F1A68103
:10416000D80700F1BC8103F00203224A002B1CBFD8
:1041700003261146DFF880803246404627F0F2F9E8
:1041800006EB080312A80133A8F1020140F8203D14
:1041900000225B1A06F808207B701DF013FFFDF764
:1041A0009FBFC4F81CB187F80090FDF751BE00BF57
:1041B0005C590020907F0020FC2400200880002013
:1041C000A674002044120408A8120408B4120408BB
:1041D00000000000E87D0020B4A400206766666649
:1041E000CCA6002058A08B41208400203410040865
:1041F0008A7F002050100408CB7F00209AF80240EC
:10420000C4B1013CE4B2013454445146002211F8D7
:10421000013B534083EA0313DBB2120ADF0042EA98
:1042200003228C4287EA131382EA0302EFD1002AA9
:104230007FF41DADBC4ABD4FBD4B1288BD4CFA6129
:10424000DFF824931A68FA629B68B4F84A21F8668A
:104250000021FB64D9F80000F963FA65F7F7D6FD91
:10426000029000287DF469AE0221D9F80000F8F729
:10427000B3FC94F84C319AF803200392642B4FF06E
:10428000040287F8742040F0738194F84D31072BB5
:1042900004BF9DF8083084F84D3194F84D310693F1
:1042A00007EB031ADAF804100291084626F01CFA0C
:1042B000DAF8081005915FFA80FA084626F014FA39
:1042C000C0B204900AEB0002069B9B480299029040
:1042D0000832C27123F00F0286468272049803F0FE
:1042E0000F0300EBCA008EF80D3052468EF80E0018
:1042F0000EF10F0027F036F9904B049A05990AF158
:104300000900184427F02EF90298C37903F1010A35
:10431000CBB1013B5FFA83FC0CF1080CDFF84CE2F7
:1043200084440023073010F8011B59408B00CA0851
:1043300083EA410302F018024B404EFA02F2534066
:104340008445DBB2EFD17D4A03980AF8023020F0B1
:10435000A3FC94F84D310022013384F84D3184F8E8
:104360004C21029BDDF808A09B785BB11AF8051080
:10437000D9F80000F8F748FC01359AF80230EDB2A0
:10438000AB42F3D894F84C310322013384F84C311A
:1043900087F8742088F80020FFF7A2B94FF0010ACF
:1043A000FEF7B8BF0221D8F80000F8F715FC94F822
:1043B0002431FDF77CBD3A6882EAE273A3EBE27335
:1043C00003EB5303A1FB0331C908002AB8BF41F036
:1043D0008041FFF798BB5A49881F23F05DFB84F8A2
:1043E0003E01FFF721BA10230027042218460AA92C
:1043F000029D8DF828308DF829208DF82A708DF8CF
:104400002B708DF82C708DF82D7023F097FC84F8AC
:104410002F71FDF778BD342793E44A4AD278002AF9
:104420000CBF4FF0040C4FF0050CFEF7F6BD012356
:10443000D8F800003B70F8F7DBFB0746D8F800001F
:10444000F8F7D6FB7B067DF403AD8A284ED08E2884
:104450007DF4FEAC94F81831002B7DF416AD3A4B88
:10446000C4F820312D2384F82431FDF7F8BC4FF037
:104470000108FEF7DBB82C4B1888FFF77FBB2A49F1
:104480009A790B8803EB830303EB83034FEA8308DA
:104490001FFA88F8002A00F01081254B1B680FFADC
:1044A00083FA0BF0A3FE40B2FDF7C0BE03262749F6
:1044B00060E6984699461846049305930393FDF7E2
:1044C000ADBF234B234A1B68234903F48003002B11
:1044D00016BF1146042603263DE6242731E41F4972
:1044E000042647E610272CE420272AE41C4B1B68EF
:1044F0009F067DF5ADAC94F81831002B7DF4C5AC6A
:10450000184BC4F820312D2384F82431FDF7A7BCC3
:10451000082716E44B1CDBB2042B84F841314FEA28
:1045200001613FF483AC84E4E87D0020200000209A
:10453000B4A40020FC240020889D00208E9D002033
:1045400034260020947F002088800020A4120408D4
:10455000D8790020341004083810040848100408E2
:10456000E8A60020B48000200CA400200007090E5B
:1045700097F875A05B4904951AF00F0F04BF0AF174
:10458000010A5FFA8AFABAF1070F28BF4FF0010A51
:104590004FEA0A1C07EB0C03187C534B02930A18D2
:1045A000002392F82410504A93725FFA8CF31A4653
:1045B0004E4B964607EB0C024EEA0000012918709C
:1045C000D26803F101000CD90239C9B28D1C1D4417
:1045D000034603F8012BAB424FEA1222F9D1013115
:1045E0000844BC4422F060030AF1010A9CF811203F
:1045F0005FFA8AFA1343BAF1080F037000F101035E
:1046000040D04FEA0A1C07EB0C01384A087C3549B8
:1046100001449A1A91F8241055180EF1100E132D1A
:104620005FFA8EFEC6DD049D0298DFF8CCE0D2B2C0
:10463000931DDBB243F04001C17103F1010CCBB11A
:104640000532D3B20833C31804930EF101000023DE
:1046500010F8011B59408B0083EA4103CA084B4004
:10466000234902F0180241FA02F25340049A8242AE
:10467000DBB2EDD103980CF80E3087F875A020F06E
:104680000BFB6EE6194A049D9A1ACDE798469946A7
:104690001846049305939E460393FDF7BFBE154B42
:1046A0009046B3F900A06420FDF7C0BD9846994636
:1046B000184604930393FDF7B1BE4FF0FF33EEE6C7
:1046C0000393FDF7ABBE98460393FDF7A7BE98464C
:1046D00099460393FDF7A2BE984699461846039360
:1046E000FDF79CBE6CE20308889D0020959D00208C
:1046F0000007090EB4A400208E9D00202DE9F04F84
:104700002DED0A8B3C4B1B7895B0012B089001F0E6
:1047100086863A4C94F80021002A41F0CB80072B82
:10472000374D01F07786002304936B68344898472F
:10473000002800F06981B5F8B470002285F8552092
:10474000002F40F04387B5F93E00AA6AB5F93C60F6
:10475000696AB5F94030DFF8B4B0821AE86A6A6372
:10476000711A1B1A2963274895F85610AB6316F087
:1047700081FEDBF80030990040F1F080D5ED0D5A54
:10478000D5ED0C7A204A94ED676AD4ED686A94ED11
:10479000697AD4F8A8311268B8EEE58AD5ED0E5AD8
:1047A000F8EEE77AF8EEE58A013377EE867A38EEAE
:1047B000268A78EE878A9342C4ED677A84ED688A08
:1047C000C4ED698AC4F8A83101F0DC830A4B1F7874
:1047D000142F02F02F870023D4F8B0610593062E22
:1047E00000F2AF80DFE816F0E215A7168714BB16BB
:1047F00014005215EB1400BF047D0020C0270020D8
:1048000028A8002058A8002014600020D879002093
:10481000D94B1A78D4F8B4E1DFF8CCC39FEDD77A3E
:104820004FEACE000CEB000383ED007A002A7DD026
:10483000D349B0EE476AF0EE476A0023F1EC017A03
:10484000013367EEA77A05EE903AB4EEE77AF1EE1F
:1048500010FAF8EEE55AB8BFB0EE677A934276EEFA
:10486000A76AA7EEA56AE9D1F5EEC06A0CEB0003D2
:10487000F1EE10FA83ED007A58DDC6EE265AC14BF0
:10488000C14A1288F7EE007A75EEE75AD3ED007A46
:1048900065EEA77AFDEEE77A17EE903A812B43F3A7
:1048A000DA859342A8BF134607EE903AF8EEE77A0E
:1048B000B64B00EB0E0103EB810393ED057AD3EDCC
:1048C000003A93ED066A93ED014AD3ED046AD3ED05
:1048D000034A93ED025AA3EEA77AA4EE276A66EE86
:1048E000C76AA7EE646ABDEEC77AE5EE276A17EEDF
:1048F000101A812983ED056AC3ED066A43F3A88582
:104900008A42A8BF0A4607EE902AF8EEE77AFCEE44
:10491000E77ACDED067ABDF818300CEB00029380F3
:10492000BEF1000F02D1132F04F04882152F42F080
:1049300037846044DFF8B482838828F81E30D4F8C6
:10494000B061934B013683FB06239A19F317C3EB2F
:10495000A203C3EBC303F61AC4F8B0618D4B1B78F6
:10496000002B01F0AE808C4EDFF88492DFF87CA241
:1049700006F2DC680027894BD5ED087A1B78172BE7
:1049800001F09A8396ED007AB8EEC78A082B28EEDC
:10499000278A07D1B0EE480A059326F0EDFF059B64
:1049A0002AF81700DBF8002092000BD5002F04F046
:1049B0005B85B0EE480AD5F8783708F17000984763
:1049C000B0EE408AB0EE480AD5F89836A8F17000EB
:1049D0009847D5F8083740469847704B1B78032B0B
:1049E000B0EE408A01F06283D6F85C06D5F8B830A4
:1049F000B0EE480A98470137032F08F12408A9ECC4
:104A0000010A06F10406B6D1644B93F80090B9F19F
:104A1000070F00F0988694F8C031002B40F0A08674
:104A20005F4B5B79002B40F0CB8501235B4A84F818
:104A3000C0311278072A02F0428000230B93594BB1
:104A400094ED729A93ED007A574BDFF8A881D3F872
:104A500000A0564B0593F7EE007A37EEC9BA544BD7
:104A600007932BEE07BA534B0993534B0693B4EEBF
:104A7000E7BA08F168030025F1EE10FA0A93D4EDC5
:104A800071BA4E4BDFF870B1DFED4D8A9FED4DAA44
:104A9000DFED3AAADFED4C9ADFF860914B4F0493BB
:104AA00088BFB0EE67BA2E46494B98ED008A2B447A
:104AB000D3ED007AF5EE407AF1EE10FA17D0454BBF
:104AC0002B44D3ED006A38EE667AB0EEC76AF4EE96
:104AD000C67AF1EE10FA08D5B5EEC07AF1EE10FA0A
:104AE000CCBF37EEA68A36EEE78A83ED008A059BB7
:104AF0001A88930700F08680022E00F08380364BE0
:104B00009AF82E1033F9163007EE103A0A9B07EE8A
:104B1000901A2B44F8EEE76AB8EEC77AD3ED007A24
:104B20004B42A6EEA77A700007EE903AF8EEE77ACD
:104B3000B4EEE77AF1EE10FA0AD407EE901AF8EE26
:104B4000677AF4EEC77AF1EE10FA88BFF0EE477A92
:104B5000224B23490344085EB3F90C30C01A07EE18
:104B6000100AB8EEC77AD007E7EE687A40F10086FF
:104B70001C4B93ED008A43E01A6000200000000007
:104B8000C02700201C600020186000205062002018
:104B9000932449920D60002058A80020047D002035
:104BA000B4790020184A00205C5900208A7F002038
:104BB00098000020747D0020C87900204C5F002000
:104BC000CDCCCC3DAE47813F0000C842585F0020AD
:104BD0000C4A00208C290020502900206C840020E1
:104BE000CCA60020F449002038620020087D002077
:104BF000CC790020C42800206C450020645F002090
:104C000027EE888A069B94F8D8212B44D3ED01CA5D
:104C100038EE6CCA002A3DD0D24BD4F8DC2108997A
:104C20001B688A1A9A4235DD9AF84830022B01F047
:104C3000BA87022E04F08583CB4B1B68990740F19D
:104C40002787CA4BCA49DFF890E331F916C09EEDB9
:104C5000008ADFF888E3C7ED00AA03EB460028EEE0
:104C6000288AB0F90C00A0EB0C0007EE900AF8EED1
:104C7000E77ADEF8000027EE888A904238EE6CCAA8
:104C8000C1F23281F7EE007AB4EEE79AF1EE10FA53
:104C900001F10181B74B2B4493ED000A049B2BEEED
:104CA000800A022E20EE0C0AA3EC010A049304F001
:104CB0006283079BDBED007A93ED007AAE4BD7ED74
:104CC000006A93ED006AAD4B67EE277A2B4427EE1E
:104CD0008B7AD3ED007A67EE277AF0EE665AE7EE2C
:104CE0008C5AB1EE467AB4EEE57AF1EE10FA08DCB1
:104CF000B4EEE56AF1EE10FA8CBFB0EE657AB0EE74
:104D0000467A94ED726AF7EE007AB4EEE76AF1EE55
:104D100010FAACBF0123002343B1F0EEE66AF0EED7
:104D2000C77AF4EEE67AF1EE10FA01D587ED007A53
:104D3000022E04F0F082924A924B52F826001B6831
:104D4000B0EE6C0A9847904A904B52F826001B68C8
:104D500098479AF8373023B1059B1B88002B00F049
:104D60007185B0EE6A8A8A4B9BED007A38EE400A74
:104D70002B4493ED008A83ED000A9AF8483030EE18
:104D8000480AC0EE077A2BB3099B1B78DB0721D5B5
:104D9000B7EE007AB4EEC79AF1EE10FA04DB94F89D
:104DA000D831002B00F05F87D4F8DC31089AD31A91
:104DB0006C4A12689A420DDD764B93ED007AB0EEA4
:104DC000CCCAB4EEC7CAF1EE10FA41F1A9800023B3
:104DD00084F8D831704B94F8E8212B4493ED007A95
:104DE0002BEE877A67EE277AC9ED007A32B9049BF9
:104DF000C7ED00AA43ED01AAC9ED00AA0136032EB2
:104E000008F1040809F1040907F1040705F1040594
:104E10007FF44AAE614B1B78072B01F05283012BC4
:104E200001F03A86002794F8F031002B40F0FA8523
:104E30005B4A5C4B10681B6810F4805A93F82C3066
:104E400040F06886584A594992ED006A498B584AA1
:104E500084ED806A92ED007A564A84ED817A07EEFD
:104E6000901AF8EEE76AD2ED037A534A84ED7E6A2F
:104E700037EE467A77EEE67AD2ED006A84ED7D7AF7
:104E8000012284F80822C7EEA65A4C494C4A91EDFB
:104E9000005A4C499FED4C6A91ED004A4B49DFEDB9
:104EA0004C6AD1ED004A92ED007A35EE045AF7EEE5
:104EB000007AF4EEE75A35EE245AF1EE10FA88BF84
:104EC000F0EE675A25EE065AF4EEE65AB1EE476A5E
:104ED000F1EE10FAB4EEC65AB8BFF0EE665AF1EE33
:104EE00010FAC4ED835A01F1DA80B4EEC75AF1EE3C
:104EF00010FA88BFB0EE475A304ADFED336AD2ED80
:104F0000017A304A92ED014A304A77EE847AD2ED46
:104F1000014A77EEA47A67EEA67AB4EEE76AF1EE7C
:104F200010FA08DCB4EEE77AF1EE10FA8CBFB0EEBE
:104F3000676AB0EE476A214ADFED236AD2ED027A52
:104F4000204AD2ED024A234A77EEA47A92ED007A03
:104F500067EEA67AB1EE473AF4EEC37AF1EE10FAB4
:104F600047D43DE0204A0020E8A600206C840020C1
:104F7000CCA60020C84900203C4A0020D44900208B
:104F80007445002070450020C8450020C44500201D
:104F9000A02900202C4A0020E0490020047D0020A8
:104FA000D87900205C590020C8820020F0940020AD
:104FB0003C840020007E0020544200204C5F0020F2
:104FC000404A0020585F00206F12833A645F00203F
:104FD00000000000444A0020F44900201C4A002040
:104FE000F4EEC77AF1EE10FA8CBFB0EE473AB0EEAD
:104FF000673AF04A52780AB9B1EE433A002B41F0D1
:105000008183F7EE003AEC4D2A78002A02F0B6864A
:10501000EA4BDFEDEB6AD3ED024A93ED017AD3ED73
:10502000037A66EE244AE5EE074AE3EE274A63EE8A
:10503000A44AF4EEE64AF1EE10FAB4BFB0EE664AC6
:10504000B0EE644A98BFF0EE646A012ACDED0C4AD6
:1050500002F0B98693ED067AD3ED052AD3ED077AEF
:1050600026EE077AA5EE227AA3EE277A23EE877A38
:10507000B4EEE67AF1EE10FAB4EEC47A8CBFF0EE3C
:10508000667AF0EE477AF1EE10FA98BFF0EE676AB2
:10509000B4BFF0EE447AF0EE477A022A8DED0D7A35
:1050A00000F0DE8093ED0A7AD3ED092A93ED0B4AE6
:1050B00026EE077AA5EE227AA3EE047A23EE877A0B
:1050C000B4EEE67AF1EE10FAB4EEE77A8CBFB0EE09
:1050D000664AB0EE474AF1EE10FA98BFF0EE446A25
:1050E000A8BFF0EE477A032A8DED0E7A00F0B88063
:1050F00093ED0E7AD3ED0D2A93ED0F4A26EE077A43
:10510000A5EE227AA3EE047A23EE877AB4EEE67A4D
:10511000F1EE10FAB4EEE77A8CBFB0EE664AB0EE6C
:10512000474AF1EE10FA98BFF0EE446AA8BFF0EEDD
:10513000477A042A8DED0F7A00F0928093ED124A9F
:10514000D3ED112A93ED137A26EE044AA5EE224AF6
:10515000A3EE074A23EE844AB4EEE64AF1EE10FAD3
:10516000B4EEE74A8CBFB0EE667AB0EE447AF1EE68
:1051700010FA98BFF0EE476AA8BFF0EE447A052A0D
:105180008DED104A6CD093ED164AD3ED152A93EDB0
:10519000177A26EE044AA5EE224AA3EE074A23EE2A
:1051A000844AB4EEE64AF1EE10FAB4EEE74A8CBF58
:1051B000B0EE667AB0EE447AF1EE10FA98BFF0EEF7
:1051C000476AA8BFF0EE447A062A8DED114A47D00F
:1051D00093ED1A4AD3ED192A93ED1B7A26EE044A71
:1051E000A5EE224AA3EE074A23EE844AB4EEE64A2D
:1051F000F1EE10FAB4EEE74A8CBFB0EE667AB0EE8C
:10520000447AF1EE10FA98BFF0EE476AA8BFF0EECC
:10521000447A072A8DED124A22D093ED1E7AD3EDFF
:105220001D2A93ED1F4A26EE077AA5EE227AA4EEF8
:10523000037A27EE237AB4EEE67AF1EE10FAB4EEB2
:10524000E77A8CBFB0EE666AB0EE476AF1EE10FA0C
:105250008DED137A98BFF0EE466AA8BFF0EE477A5C
:1052600077EEE67AF7EE006AF4EEE67AF1EE10FAFF
:10527000C4ED727A43F3878586EEA77A022ADDEDC4
:105280000D7A67EE244A67EE877ACDED0C4ACDEDB4
:105290000D7A2DD0DDED0E7A67EE877A032ACDEDFB
:1052A0000E7A25D0DDED0F7A67EE877A042ACDEDF0
:1052B0000F7A1DD0DDED107A67EE877A052ACDEDE5
:1052C000107A15D0DDED117A67EE877A062ACDEDDA
:1052D000117A0DD0DDED127A67EE877A072ACDEDCF
:1052E000127A05D0DDED137A27EE877A8DED137AE9
:1052F000344B1E6816F0805601F0AA80F6EE005A74
:10530000C4ED835A002A02F011852F4BD4ED814A57
:1053100093F8038094F908320999D4ED806A91F8E2
:1053200000E0DFF8B0C02949DFF8AC90B1F9061011
:105330009CED007A049106EE103AFDEEE44A244B0F
:1053400099F80090B3F81AB094ED7D5AD4ED7E7AB6
:1053500014EE903AFDEEE64A00F0100C00F48000E6
:105360000EF0010EB8EEC66A14EE901A0590B8F170
:10537000000F41F00982DFF84480BCF1000F41F0DA
:10538000B58098ED007ADDED0C6ADFF850C025EEAF
:10539000877AA6EE267AF0EE676AE5EE076ABDEE3A
:1053A000E67A17EE106A17EE100A9E42A8BF18465A
:1053B00016E000BFAC5F0020E57C0020C441002067
:1053C0000000000020840020947F0020607F0020E7
:1053D000F0940020A0410020A8760020805F0020EB
:1053E000B142C8BF084607EE100AB8EEC77A012AD4
:1053F0008CED007A00F0DC8098ED047ADDED0D6A2A
:1054000025EE877AA6EE267AF0EE676AE5EE076A61
:10541000BDEEE67A17EE106A17EE100A9E42A8BF9C
:105420001846B142C8BF084607EE100AB8EEC77A60
:10543000022A8CED017A00F0BB8098ED087ADDED50
:105440000E6A25EE877AA6EE267AF0EE676AE5EE1A
:10545000076ABDEEE67A17EE106A17EE100A9E4252
:10546000A8BF1846B142C8BF084607EE100AB8EEFA
:10547000C77A032A8CED027A00F09A8098ED0C7AB4
:10548000DDED0F6A25EE877AA6EE267AF0EE676AE2
:10549000E5EE076ABDEEE67A17EE106A17EE100A1F
:1054A0009E42A8BF1846B142C8BF084607EE100A80
:1054B000B8EEC77A042A8CED037A79D098ED107A89
:1054C000DDED106A25EE877AA6EE267AF0EE676AA1
:1054D000E5EE076ABDEEE67A17EE106A17EE100ADF
:1054E0009E42A8BF1846B142C8BF084607EE100A40
:1054F000B8EEC77A052A8CED047A59D098ED147A63
:10550000DDED116A25EE877AA6EE267AF0EE676A5F
:10551000E7EE056ABDEEE67A17EE106A17EE100A9E
:105520009E42A8BF1846B142C8BF084607EE100AFF
:10553000B8EEC77A062A8CED057A39D098ED187A3C
:10554000DDED126A25EE877AA6EE867AF0EE676ABE
:10555000E7EE056ABDEEE67A17EE106A17EE100A5E
:105560009E42A8BF1846B142C8BF084607EE100ABF
:10557000B8EEC77A072A8CED067A19D098ED1C7A16
:10558000DDED136A65EE875AE6EE265AE5EE257ADA
:10559000FDEEE77A17EE900A8342A8BF03468142E8
:1055A000C8BF0B4607EE903AF8EEE77ACCED077AE3
:1055B000BEF1000F40F04382002A40F03B823EE201
:1055C000AE4B1B78013BDBB2FFF730BAAC4B069316
:1055D0004FF47A761B68B6FBF3F3C3EB4316A94985
:1055E000DFF8CC8291F801A0A749B8F9060091F83C
:1055F000009003EB8603DE00B6B2B74202F0FD80F6
:10560000D5F88810B5F93CE0EB6E4A1C07EE90EA3D
:105610007344012AC5F88820EB66F8EEE77A02F0B9
:10562000F780D5ED1E5AD5ED206A07EE102A37EE29
:10563000E56AB8EEC75A012F86EE057A37EE257A6D
:1056400077EEC77A85ED1F7AE7EE866A85ED1E7ADA
:10565000F0EE667AC5ED216AC5ED206A02F0D384CA
:10566000D5F89C10B5F93EE02B6F4A1C07EE90EA86
:105670007344012AC5F89C202B67F8EEE77A02F004
:10568000E080D5ED235AD5ED256A07EE102A37EED6
:10569000E56AB8EEC75A012F86EE057A37EE257A0D
:1056A00077EEC77A85ED247AE7EE866A85ED237A70
:1056B000F0EE667AC5ED266AC5ED256A02F0D8845B
:1056C000D5F8B010B5F940E06B6F4A1C07EE90EAD0
:1056D0007344012AC5F8B0206B67F8EEE77A02F050
:1056E000C980D5ED285AD5ED2A6A07EE102A37EE83
:1056F000E56AB8EEC75A012F86EE057A37EE257AAD
:1057000077EEC77A85ED297AE6EE276A85ED287A65
:10571000F0EE667AC5ED2B6AC5ED2A6A02F09C842C
:10572000A8F80600B5F8B430574A013B92F800904B
:10573000A5F8B43006990023B9F1070F4B608B60D0
:10574000CB607FF468A9F6F7A3FF049BDFF86081C4
:10575000C01A94F8C031A8F80000002B3FF460A9EB
:10576000013B84F8C03115B0BDEC0A8BBDE8F08F69
:1057700094ED5E7AB1F90000D4ED5F6AB1F902E010
:10578000424AF4EEC76A80EAE0738EEAEE71A3EB58
:10579000E073F1EE10FAA1EBEE71B4BFB0EE476A20
:1057A000B0EE666A8B42B8BF0B4607EE103A13782C
:1057B000B8EEC77A27EE287A002B40F02582344BCA
:1057C000D3ED005AF4EECA5AF1EE10FA41F1F88026
:1057D000B7EE005A75EE654ADFED2E6A9FED2E5A40
:1057E0002E4B36EEC77A24EE855AD3ED006AE7EEEB
:1057F000055A65EEA65AF5EEC05AF1EE10FA40F2DF
:105800002386C9EEA56AB7EE007AF0EE475AE6EEB7
:10581000665AF0EE656AF4EEC76AF1EE10FA88BFD8
:10582000F0EE476AF5EEC06AF1EE10FAB8BFF0EE9E
:105830006A6A1B4B93ED007A67EE877AA7EEA68A19
:10584000FFF7E0B9174B184A2B4493ED007AD2EDDD
:10585000007A164B67EE277AF7EE006AF4EEE67AE6
:10586000F1EE10FA93ED007A88BFF0EE667A67EEFB
:10587000877A27EE888AFFF776BA00BF6084002017
:10588000C8790020B4790020047D0020004A00205F
:10589000084A002000003443610BB63BFC4900205D
:1058A000F849002038290020F0490020EC49002068
:1058B000087D0020072B02F081820026DFF83CB330
:1058C000B64DDBF800305F0501F17F80B44B1B78EB
:1058D000002B40F0F381DFF80C9394F8127127B19C
:1058E000B04B1B88980742F0348094F81821002AA6
:1058F00041F0758099F81E70002F00F0F383022F9D
:1059000002F02080032F01F0D082A74B598899F82C
:105910001F300233DBB2002A02F00880002902F0B7
:105920000580A2480768B1FBF7F10FB2A4F84871EF
:10593000002B03F0308207EE907AF8EEE77AF7EE6C
:10594000006A86EEA77A9A49012BD4ED576AD1ED09
:10595000007A77EEE67A67EE877AC4ED537A21D043
:10596000D1ED017AD4ED586A77EEE67A022B67EE34
:10597000877AC4ED547A15D0D1ED027AD4ED596A04
:1059800077EEE67A032B67EE877AC4ED557A09D075
:10599000D1ED037AD4ED5A6A77EEE67A67EE877A2C
:1059A000C4ED567A83480078092803F0A082002FBE
:1059B00040F39E8393B394ED577AD4ED537A77EE08
:1059C000877A012BC4ED577AC1ED007A21D094ED8E
:1059D000587AD4ED547A77EE877A022BC4ED587A50
:1059E000C1ED017A15D094ED597AD4ED557A77EE60
:1059F000877A032BC4ED597AC1ED027A09D0D4ED30
:105A00005A7A94ED567A77EE877AC4ED5A7AC1EDD8
:105A1000037A013B022BB8BF0223DBB2002A18BF76
:105A2000022366E3099B644D1B78DE0700F1648165
:105A30002A7822B192006149614825F093FD614BBB
:105A40001B68002B40F02F835F4B1B789BB128789D
:105A500070B1DFF86C81DFF8A8910026F0B2D9F8B8
:105A60000030B8EC010A9847287801368642F5DB09
:105A7000564B1B6898474F4B1B78072B00F01A8535
:105A8000012384F8003115B0BDEC0A8BBDE8F08F1E
:105A90004F4BC7ED00AA1B689342BFF6F3A84D4BCE
:105AA0001A88002384F8D831002A41F09C864A4A9B
:105AB0004A4B1178186881F00101F7F7A1FCFFF754
:105AC000E9B8474FDFF83C9107F24C7607F5F768E5
:105AD000F7EC017A95ED080AD5F87837F8EEE77A11
:105AE000304627EE800A9847A6F1E000D5F89836B0
:105AF0009847A6F17000D5F808379847D7F85806A8
:105B0000D5F8B83098472436B045A9EC010ADFD162
:105B1000FEF77ABF099A1278D50703D4314A128B5F
:105B2000A4F8FC21304A2249128891ED037A07EE4D
:105B3000902AF8EEE77AB4EEE77AF1EE10FA41F245
:105B400096802A49098807EE901AF8EEE77AB4EEB3
:105B5000E77AF1EE10FAC0F2FC872549254AD1ED2B
:105B6000006A92ED006A2449C4ED806ABCEEC75A0F
:105B700076EE665A15EE102AC4ED7E6AC4ED7D5AA3
:105B800084ED816AA4F8FC210122D1ED006A84F839
:105B9000082277EE677AFFF776B900BF28A80020C1
:105BA000480100208A7F00207CA20020A45F002002
:105BB000007E0020047D0020E57C0020A441002020
:105BC000805F002068450020B0790020A476002086
:105BD0001C4A0020387C00203A7C00203C7C0020BD
:105BE00058A80020F0940020584200205A4200207B
:105BF000444200203C84002060420020D8790020EC
:105C00009C760020CC790020CD4B93ED005AB5EE68
:105C1000C05AF1EE10FA40F31784CA4BD3ED006A74
:105C2000F5EEC06AF1EE10FA40F30E8436EEC77A54
:105C300066EE695A87EE266AC5EE856AB7EE007A87
:105C4000B4EEC76AF1EE10FA88BFB0EE476AB5EE5F
:105C5000C06AF1EE10FA76EE876AB8BFB0EE6A6AF3
:105C600066EE266AD7E5B84A92ED007AF0EEE76A6A
:105C7000F4EEC76AF1EE10FA7FF796A8B34A92EDF8
:105C8000007AF0EECC6AF4EEC76AF1EE10FA7FF714
:105C90008BA8AF4A98ED007AD2ED006AB0EEC77AD1
:105CA000B4EEE67AF1EE10FA7FF57EA801220899AB
:105CB000C4F8DC1184F8D821FFF77AB8A54BDFF8D7
:105CC000B892B3F90620B9F81A309A423FF705AEF8
:105CD000A14B1B78012B01F01486192B01F01186C2
:105CE0000E2B3FF4FAAD082B3FF4F7AD9B49002390
:105CF0008B60C4F80C31F0E52B78002B3FF49FAE9D
:105D0000D4ED5F3A94ED5E6AD4ED7E7A944A94EDD8
:105D10007D7AD2ED005A94ED5C4AD4ED5B4ADFF80F
:105D20005C82DFF85CC2F4EEC63AF3EE046AF1EE90
:105D300010FA37EEA65A01F1098098ED026A26EEB4
:105D4000446AF0EE674AE6EE074AF4EEC54A34EEDE
:105D5000E66AF1EE10FA48BFB0EE656A012B8CEDF1
:105D6000006A3FF46CAE98ED066A26EE446AF0EEE7
:105D7000674AE6EE074AB4EEE45A34EEE66AF1EE1C
:105D800010FA88BFB0EE656A022B8CED016A3FF411
:105D900056AE98ED0A6A26EE446AF0EE674AE6EEE1
:105DA000074AF4EEC54A34EEE66AF1EE10FA48BF4F
:105DB000B0EE656A032B8CED026A3FF440AE98EDBD
:105DC0000E6A26EE446AF0EE674AE6EE074AB4EE43
:105DD000E45A34EEE66AF1EE10FAC8BFB0EE656A36
:105DE000042B8CED036A3FF42AAE98ED126A26EE7E
:105DF000446AF0EE674AE6EE074AB4EEE45A34EE3F
:105E0000E66AF1EE10FAC8BFB0EE656A052B8CEDBC
:105E1000046A3FF414AE98ED166A26EE446AF0EE7A
:105E2000674AE6EE074AF4EEC54A74EEE66AF1EE1A
:105E300010FAB8BFF0EE656A062BCCED056A3FF4A8
:105E4000FEADD8ED1A6A66EEC46AF0EE674AE6EE79
:105E5000874AB3EE046AB4EEE45A74EEC66AF1EE11
:105E600010FAC8BFF0EE656A072BCCED066A3FF466
:105E7000E6ADD8ED1E6A26EEC44AE4EE077AB4EE2B
:105E8000E75A77EEC67AF1EE10FAC8BFF0EE657AFF
:105E9000CCED077AD3E50699324BD1ED017A93ED3B
:105EA000007AF0EEE77AF4EEC77AF1EE10FA7EF5BA
:105EB000F1AED1ED027AF0EEE77AB4EEE77AF1EEE8
:105EC00010FA7EF7E7AED1ED037AF0EEE77AB4EEA2
:105ED000E77AF1EE10FA7EF7DDAE234B1B689A07E6
:105EE0007FF5DDAD2149224BB3F90C20B1F900E07B
:105EF0002048AEEB020E00688EEAEE72A2EBEE7264
:105F00008242BEF6C7AEB3F90E30B1F90220D21A02
:105F100082EAE273A3EBE27398427EF7BBAEBEE582
:105F20000B4B98ED007AD3ED006AB0EEC77AB4EE71
:105F3000E67AF1EE10FA7EF74DAFFEF748BF00BFEC
:105F4000FC490020044A0020304A00202C4A00204E
:105F5000344A0020607F0020AC5F0020007E0020DB
:105F6000A0410020284A0020E8A60020CCA600205E
:105F70006C840020244A0020F0940020C4410020BA
:105F8000805F002007EE103A524BDFF854811B78F7
:105F9000C4F8A871B8EEC77AF7EE006A132B86EE44
:105FA000879AB8F90400B4F8AC7195ED080A01F0CD
:105FB000A583494B494A93ED001A93ED053A93EDB9
:105FC000122A93ED176AD3ED091A93ED0E4AD3ED19
:105FD000015AD3ED063A93ED0A7A93ED0F5AD3EDB9
:105FE000132AD3ED186AD3ED044AD3ED030A67EE02
:105FF000897A69EE288A29EE088AA1EE273A02EB0F
:1060000087060021A2EE286AC4F89C11C4F8A011EA
:10601000A1EE884AE5EEA73AA7EE085A93ED167A64
:10602000D3ED0D5A93ED021AD3ED0C1A86ED003A1A
:10603000E2EEA86A64EEC34A27EE467A93ED0B2A95
:10604000D3ED152A86ED204AE0EEC33A65EEC45A38
:1060500093ED143AC3ED053AE1EE274AF0EE477AA4
:10606000A1EEC45AE2EE085AE2EEC66AE3EE287ADE
:10607000C3ED064A83ED0E5AC3ED0F5A86ED406A12
:10608000C3ED176AC3ED187AC4F8A4117B1C03F0A2
:106090001F03A4F8AC31A8F80400FEF797BBB0EEDC
:1060A000465AFEF729BF0EF0A9F9CDE425F064FCAD
:1060B0002AF81700FEF798BC96ED007A05EB470228
:1060C000B8EEC78A928F2AF8172028EE278AFEF7A3
:1060D00069BC00BF047D0020BC6200203860002045
:1060E000087D0020A4F84871002A00F07281DB4985
:1060F0000223DB4ADFEDDB6A1068DB4A90F802E03E
:1061000092F800C0027807EE902AF8EEE77AB0EE37
:10611000007A67EEA67AF4EEC77AF1EE10FA40F351
:10612000228337EEC77ADFEDD16AB0EE676AA7EE59
:10613000266AB0EE467A9FEDCE6AD1ED006A66EE31
:10614000866AB0EEE66AC4ED5B6A84ED5E6ABEF113
:10615000000F13D005EE90EAB8EEE55ADFEDC15A14
:1061600066EEA64A25EE255AF7EE005A75EEC55A98
:1061700064EE864AE4EE855A66EEA56ADFEDBD5A06
:10618000427927EE257A27EE267ACAB1DFEDB56A85
:10619000DFEDB95A26EE266A06EE902AF8EEE66A98
:1061A00026EE266AB4EEE56AF1EE10FA00F3868573
:1061B000F7EE005A35EEC66AC5EE866A27EE267AF5
:1061C000BCF10C0F9FEDAD8ADFEDAD6A00F02785C5
:1061D000B4EEC87AF1EE10FA98BFB0EE478AB4EE8A
:1061E000E68AF1EE10FAB8BFB0EE668A84ED418A15
:1061F000002B00F0E280B0EE007AF4EEC77AF1EE08
:1062000010FA05DD37EEC77ADFED986AE7EE267AF9
:1062100091ED017ADFED966A27EE267AB0EEC76A35
:1062200084ED5C7A84ED5F6ABEF1000F13D006EE58
:1062300090EADFED8C5AF8EEE66A27EE075A66EE32
:10624000A56AF7EE005A75EEE65A25EE065AE5EE17
:10625000265A27EE257ADFED876A827967EEA67ADD
:1062600067EE877AAAB107EE102AB8EEC77ADFED9B
:106270007D5ADFED816A27EE067A27EE257AB4EEA5
:10628000E67AF1EE10FA40F31D85DFED7E6A67EEE7
:10629000A67ABCF10C0F00F0A184DFED786A9FEDC7
:1062A000787AF4EEE67AF1EE10FA88BFF0EE667ACC
:1062B000F4EEC77AF1EE10FAB8BFF0EE477A012B90
:1062C000C4ED427A79DD4378DFED666A07EE903AF5
:1062D000F8EEE77AB0EE007A67EEA67A437AF4EE4B
:1062E000C77AF1EE10FA05DD37EEC77ADFED5F6AA7
:1062F000E7EE267A91ED027ADFED5D6A27EE267AE7
:10630000B0EEC76A84ED5D7A84ED606A9BB106EEFB
:10631000903ADFED545AF8EEE66A27EE075A66EE39
:10632000A56AF7EE005A75EEE65A25EE065AE6EE35
:10633000855A27EE257ADFED4F6AC37967EEA67A94
:1063400067EE877A0BB307EE103AB8EEC77ADFED47
:10635000455ADFED496A27EE067A27EE257AB4EE34
:10636000E67AF1EE10FA0CDCB5EEC07AF1EE10FA36
:1063700001F1D282B7EE006A36EE477AC6EE076ABE
:1063800001E0DFED406A67EEA67ABCF10C0F00F089
:106390001B84DFED3A6A9FED3A7AF4EEE67AF1EE8D
:1063A00010FA88BFF0EE667AF4EEC77AF1EE10FAD2
:1063B000B8BFF0EE477AC4ED437ABCF1090F00F0A4
:1063C000E78399F82170002F40F07E83002384F842
:1063D00018312D4B1B68990609D52C4B1B8803F0EF
:1063E000300323B12A4B1B78DA0701F1BA87294B16
:1063F0001B7823B9284FBB78002B41F0E7821A4B5A
:106400001B78072B00F028840022072B84F800213A
:106410007EF489A9F6F73CF90490FEF786B91F4B84
:106420001F4C1A681F4BDFF8888094F80001D2696E
:106430001B88A8F80020A8F8023000287FF43DAAA5
:106440000490194DFEF771B9DFED186AFFF7F1B945
:1064500041023EF553AFFEF755BF00BF007E00205E
:106460001C4B00200AD7233C047D0020D7A36841A1
:106470006F12033B00004843A4707D3F00C0F94405
:1064800000C0F9C40000C842E8A600208A7F0020AE
:10649000ECA600202F680020AA5A002010820020BD
:1064A000C0270020EA3E002028A8002000000000AD
:1064B000087D0020F6F7ECF8AC4BC01BD880FFF746
:1064C000DFBAF6F7E5F8AA4B0B9A1B78DFF89C8247
:1064D000801A012BA8F8020000F0E082072B7EF45E
:1064E000A1ACF6F7D5F80746FEF79DBCBEF1000F4C
:1064F00041F07B8498ED007ADDED0C6ADFF884C210
:1065000025EE877AA6EE867AF0EE676AE7EE056AF0
:10651000BDEEE67A17EE106A17EE100A9E42A8BF8B
:106520001846B142C8BF084607EE100AB8EEC77A4F
:10653000012A8CED007A3FF47DAA98ED047ADDED16
:106540000D6A25EE877AA6EE867AF0EE676AE7EEA8
:10655000056ABDEEE67A17EE106A17EE100A9E4243
:10656000A8BF1846B142C8BF084607EE100AB8EEE9
:10657000C77A022A8CED017A3FF45CAA98ED087A7A
:10658000DDED0E6A25EE877AA6EE867AF0EE676A72
:10659000E7EE056ABDEEE67A17EE106A17EE100A0E
:1065A0009E42A8BF1846B142C8BF084607EE100A6F
:1065B000B8EEC77A032A8CED027A3FF43BAA98ED35
:1065C0000C7ADDED0F6A25EE877AA6EE867AF0EE7C
:1065D000676AE7EE056ABDEEE67A17EE106A17EE17
:1065E000100A9E42A8BF1846B142C8BF084607EE2F
:1065F000100AB8EEC77A042A8CED037A3FF41AAA7F
:1066000098ED107ADDED106A25EE877AA6EE867A8F
:10661000F0EE676AE7EE056ABDEEE67A17EE106AFD
:1066200017EE100A9E42A8BF1846B142C8BF0846DE
:1066300007EE100AB8EEC77A052A8CED047A3FF40B
:10664000F9A998ED147ADDED116A25EE877AA6EEA8
:10665000867AF0EE676AE7EE056ABDEEE67A17EE37
:10666000106A17EE100A9E42A8BF1846B142C8BF72
:10667000084607EE100AB8EEC77A062A8CED057AAE
:106680003FF4D8A998ED187ADDED126A25EE877AE5
:10669000A6EE867AF0EE676AE7EE056ABDEEE67A68
:1066A00017EE106A17EE100A9E42A8BF1846B142B4
:1066B000C8BF084607EE100AB8EEC77A072A8CED65
:1066C000067A3FF4B7A998ED1C7ADDED136A65EE02
:1066D000875AE6EE265AE5EE257AFDEEE77A17EEC2
:1066E000900A8342A8BF03468142C8BF0B4607EE0B
:1066F000903AF8EEE77ACCED077A002A7FF49AA96F
:10670000FFF79DB91B4B5A79002A3EF47AAC1A4A1E
:106710001278002A3EF475AC1B78DFED184A07EEBC
:10672000903A174BB8EE677A1B8807EE902A06EE70
:10673000903AF8EEE77AF8EE666A67EE277AB7EEF7
:10674000007AC7EEA63AF4EEE43AF1EE10FA88BF0A
:10675000F0EE643AF4EEC73AF1EE10FAB8BFF0EE9C
:10676000473AFEF750BCB0EE677AE4E4087D0020BB
:10677000047D0020D4A60020FE7D0020713DAA3FAC
:10678000E87D0020805F0020BCF1000F00F09783BF
:10679000BEF1000F42F04780DFF8A085B9F1000F8D
:1067A00041F09286D8ED006ADDED0C4ADFF890C525
:1067B00065EEA66ABDEEC77A17EE101AB0EE667ADD
:1067C000A4EE867AF0EE676AE7EE056ABDEEE67A39
:1067D00017EE106A17EE100A9E42A8BF1846B14283
:1067E000C8BF084607EE100AB8EEC77A012A8CED3A
:1067F000007A3FF41FA998ED047ADDED0D6A25EECD
:10680000877AA6EE867AF0EE676AE7EE056ABDEE55
:10681000E67A17EE106A17EE100A9E42A8BF1846D5
:106820008E42B8BF084607EE100AB8EEC77A022AB1
:106830008CED017A3FF4FEA898ED087ADDED0E6A42
:1068400025EE877AA6EE867AF0EE676AE7EE056AAD
:10685000BDEEE67A17EE106A17EE100A9E42A8BF48
:1068600018468E42B8BF084607EE100AB8EEC77A3F
:10687000032A8CED027A3FF4DDA898ED0C7ADDED69
:106880000F6A25EE877AA6EE867AF0EE676AE7EE63
:10689000056ABDEEE67A17EE106A17EE100A9E4200
:1068A000A8BF18468E42B8BF084607EE100AB8EED9
:1068B000C77A042A8CED037A3FF4BCA898ED107ACD
:1068C000DDED106A25EE877AA6EE867AF0EE676A2D
:1068D000E7EE056ABDEEE67A17EE106A17EE100ACB
:1068E0009E42A8BF18468E42B8BF084607EE100A5F
:1068F000B8EEC77A052A8CED047A3FF49BA898ED90
:10690000147ADDED116A25EE877AA6EE867AF0EE2E
:10691000676AE7EE056ABDEEE67A17EE106A17EED3
:10692000100A9E42A8BF18468E42B8BF084607EE1E
:10693000100AB8EEC77A062A8CED057A3FF47AA8D9
:1069400098ED187ADDED126A25EE877AA6EE867A42
:10695000F0EE676AE7EE056ABDEEE67A17EE106ABA
:1069600017EE100A9E42A8BF18468E42B8BF0846CE
:1069700007EE100AB8EEC77A072A8CED067A3FF4C4
:1069800059A898ED1C7ADDED136A65EE875AE6EE9C
:10699000265AE5EE257AFDEEE77A17EE900A834255
:1069A000A8BF03468142D8BF194607EE901AF8EEF9
:1069B000E77ACCED077A002A7FF43CA8FFF73FB8CE
:1069C000C74BD3ED005AFEF716BFAB68002B3EF461
:1069D0007DAF05F1500128469847FEF777BFC14BC0
:1069E000C149D3F8EC30096844F620608342A8BF5F
:1069F0000346B3F57A7FB8BF4FF47A7398B2C906ED
:106A0000A4F81A01DBF8003041F1F882DB0400F150
:106A10006B83B64BD3F800E0BEF93270B449DFF8AF
:106A200024C3D1ED037AD4F81C31ACFB00108009EB
:106A3000642191FBF0F11429BDEEE77A04EB430CDD
:106A4000A8BF142101338B42C4F81C3117EE108A01
:106A5000A4BF0023C4F81C3104EB4303ACF820812D
:106A6000B3F9203107EE103AB8EEC77A77EEC77A5D
:106A7000FDEEE77ACDED047ABDF9101081EAE173FD
:106A8000A3EBE173BB4202F36F819A4B19464FF0BF
:106A90007E530B60FEF72EBFDFF8AC82F5F7F8FDF2
:106AA000954AD4F8EC311268C4F8EC01C31A9A1A6A
:106AB0000746A8F80430A8F80620FEF7B4B9F5F7A1
:106AC000E7FD0B90FDF7BBBF1E218748F2F7CEFC18
:106AD00000283FF47BAC894B1B8858063FF576AC09
:106AE00094F88431BB4242F08B81824BD4ED627AC0
:106AF000D3ED016A94ED435ADFED815A9FED816A2F
:106B000027EEC57A68EE277AA8EE267AE5EE267A91
:106B1000B4EEE57AF1EE10FA88BFB0EE657AB4EE25
:106B2000C67AF1EE10FAF4EEE57AB8BFB0EE467A26
:106B3000F1EE10FA88BFF0EE657AF4EEC67AF1EE67
:106B400010FAB8BFF0EE467A84ED417AC4ED437A8C
:106B50003CE4B4F8FC11914240F281856A496B4AE9
:106B6000D1ED007A92ED007A6949C4ED807A77EE32
:106B7000676AC4ED7E7A0122C4ED7D6A84ED817A74
:106B8000D1ED006ADFED637A84F80822FEF77BB965
:106B9000FDEEC87ADFF8B08117EE903AA8F80470DD
:106BA000A8F806300DE45C4B1B88002B40F076857E
:106BB0005A4A5B4B11781868F6F722FCD4F8DC21AE
:106BC000089B9A1AFEF735B8BDEEE77ADFF87881B0
:106BD00017EE103AA8F80430FFF7DBBB9FED487AB8
:106BE000DFED486ADFF86081F4EEC77AF1EE10FA63
:106BF00098BFB0EE677AFDEEE77AB4EEE67AF1EE92
:106C000010FA17EE902AB8BFB0EE667A012B84ED29
:106C1000427AA8F802203FF756ABFFF7D2BBB4EE9A
:106C2000C87AF1EE10FA98BFB0EE478ABDEEC77A87
:106C3000B4EEE68ADFF81081F1EE10FA17EE102AB2
:106C4000B8BFB0EE668A84ED418AA8F80020002B18
:106C50007FF4D1AAFFF7B5BBF5F71AFDDFF8E8809E
:106C6000304B801B1B78A8F80400FFF7CDBB2E4AE1
:106C70002E49D2ED006A2E4A91ED006A1278C4EDD9
:106C8000806A84ED816A002A40F0E58476EEC65A77
:106C9000F0EE466ABCEEC76A2649C4ED7D5A16EE90
:106CA000102AC4ED7E6AA4F8FC21FF22D1ED006A0F
:106CB00084F8082277EEC77AFEF7E5B8DFED1E6AA2
:106CC000FFF77CBAB5EEC07AF1EE10FA00F120863B
:106CD000B7EE006A36EE477AC6EE076AFFF7D7BA14
:106CE000FC4900201C1E0020208400205C5900204C
:106CF000007E002098000020A45F00208A7F0020F2
:106D000000C0F94400C0F9C4444200203C84002083
:106D10006042002000000000387C00203A7C002007
:106D20003C7C0020047D0020C882002048420020D6
:106D3000A87600205C4200200000C842C441002028
:106D4000805F0020D34D6210087D002098ED016A1D
:106D500026EE646AB0EE674AA6EE074AB4EEC45A5D
:106D600034EE666AF1EE10FAC8BFB0EE656A012B28
:106D70008CED006A3EF463AE98ED056A26EE646A17
:106D8000B0EE674AA6EE074AB4EEC45A34EE666A1D
:106D9000F1EE10FAC8BFB0EE656A022B8CED016A05
:106DA0003EF44DAE98ED096A26EE646AB0EE674A8D
:106DB000A6EE074AB4EEC45A34EE666AF1EE10FA53
:106DC000C8BFB0EE656A032B8CED026A3EF437AEA5
:106DD00098ED0D6A26EE646AB0EE674AA6EE074AA1
:106DE000B4EEC45A34EE666AF1EE10FAC8BFB0EEE3
:106DF000656A042B8CED036A3EF421AE98ED116AAE
:106E000026EE646AB0EE674AA6EE074AB4EEC45AAC
:106E100034EE666AF1EE10FAC8BFB0EE656A052B73
:106E20008CED046A3EF40BAE98ED156A26EE646AAA
:106E3000B0EE674AA6EE074AB4EEC45A74EE666A2C
:106E4000F1EE10FAC8BFF0EE656A062BCCED056ACC
:106E50003EF4F5ADD8ED196A66EEE46AB0EE674A25
:106E6000A6EE874AB3EE046AB4EEC45A74EE466ADC
:106E7000F1EE10FAC8BFF0EE656A072BCCED066A9A
:106E80003EF4DDADD8ED1D6A66EEE44AE4EE877AA5
:106E9000F4EEC57A77EEC67AF1EE10FAB8BFF0EEEE
:106EA000657ACCED077AFEF7CABD99F82030C3EBBE
:106EB000431103EB8101C90089B2FEF728BDDFF859
:106EC000DC84B9F1000F41F00D81D8ED006ADDEDF1
:106ED0000C4ADFF8CCC465EEA66ABDEEC77A17EEA1
:106EE000101AB0EE667AA4EE867AF0EE676AE7EEE4
:106EF000056ABDEEE67A17EE106A17EE100A9E429A
:106F0000A8BF1846B142C8BF084607EE100AB8EE3F
:106F1000C77A012A8CED007A3EF44AAB98ED047AE8
:106F2000DDED0D6A25EE877AA6EE867AF0EE676AC9
:106F3000E7EE056ABDEEE67A17EE106A17EE100A64
:106F40009E42A8BF18468E42B8BF084607EE100AF8
:106F5000B8EEC77A022A8CED017A3EF429AB98ED9F
:106F6000087ADDED0E6A25EE877AA6EE867AF0EED7
:106F7000676AE7EE056ABDEEE67A17EE106A17EE6D
:106F8000100A9E42A8BF18468E42B8BF084607EEB8
:106F9000100AB8EEC77A032A8CED027A3EF408ABE9
:106FA00098ED0C7ADDED0F6A25EE877AA6EE867AEB
:106FB000F0EE676AE7EE056ABDEEE67A17EE106A54
:106FC00017EE100A9E42A8BF18468E42B8BF084668
:106FD00007EE100AB8EEC77A042A8CED037A3EF465
:106FE000E7AA98ED107ADDED106A25EE877AA6EE15
:106FF000867AF0EE676AE7EE056ABDEEE67A17EE8E
:10700000106A17EE100A9E42A8BF18468E42B8BFFB
:10701000084607EE100AB8EEC77A052A8CED047A06
:107020003EF4C6AA98ED147ADDED116A25EE877A52
